******************************************************************************
               TMS320C6x Linker Unix v7.4.0                    
******************************************************************************
>> Linked Mon Nov 19 16:54:04 2012

OUTPUT FILE NAME:   <shmIpcBenchmark_c6657.out>
ENTRY POINT SYMBOL: "_c_int00"  address: 0082a700


MEMORY CONFIGURATION

         name            origin    length      used     unused   attr    fill
----------------------  --------  ---------  --------  --------  ----  --------
  L2SRAM                00800000   00100000  00052e72  000ad18e  RW X
  MSMCSRAM              0c000000   00100000  00100000  00000000  RW X
  DDR3                  80000000   20000000  00000000  20000000  RWIX


SEGMENT ALLOCATION MAP

run origin  load origin   length   init length attrs members
----------  ----------- ---------- ----------- ----- -------
00800000    00800000    000315c0   000315c0    r-x
  00800000    00800000    000315c0   000315c0    r-x .text
008315c0    008315c0    00019008   00000000    rw-
  008315c0    008315c0    0000fa00   00000000    rw- .msgQ_ptrs
  00840fc0    00840fc0    00009608   00000000    rw- .far
0084a5c8    0084a5c8    00000008   00000008    rw-
  0084a5c8    0084a5c8    00000008   00000008    rw- .fardata.1
0084a5d0    0084a5d0    0000497e   0000497e    r--
  0084a5d0    0084a5d0    0000497e   0000497e    r-- .const
0084ef50    0084ef50    0000153c   0000153c    rw-
  0084ef50    0084ef50    0000153c   0000153c    rw- .fardata.2
00850490    00850490    00001000   00000000    rw-
  00850490    00850490    00001000   00000000    rw- .stack
00851490    00851490    00000ec0   00000da0    rw-
  00851490    00851490    00000da0   00000da0    rw- platform_lib
  00852230    00852230    00000120   00000000    rw- .cio
00852350    00852350    00000080   00000080    r--
  00852350    00852350    00000080   00000080    r-- .switch
00852400    00852400    00000200   00000200    r-x
  00852400    00852400    00000200   00000200    r-x .vecs
00852600    00852600    00000018   00000000    rw-
  00852600    00852600    00000018   00000000    rw- .bss
00852618    00852618    00000050   00000050    rw-
  00852618    00852618    00000050   00000050    rw- .neardata
00852668    00852668    00000840   00000840    r--
  00852668    00852668    00000840   00000840    r-- .cinit


SECTION ALLOCATION MAP

 output                                  attributes/
section   page    origin      length       input sections
--------  ----  ----------  ----------   ----------------
.init_array 
*          0    00800000    00000000     UNINITIALIZED

xdc.meta   0    00800000    00000120     COPY SECTION
                  00800000    00000120     bench_shm_pe66.oe66 (xdc.meta)

.text      0    00800000    000315c0     
                  00800000    00001ea0     ti.platform.evm6657l.ae66 : platform.obj (.text)
                  00801ea0    00001900                               : evmc6657.obj (.text)
                  008037a0    000011c0     ipc.lib : Ipc.obj (.text:ti_sdo_ipc_GateMP_Instance_init__F)
                  00804960    000010c0     ti.platform.evm6657l.ae66 : evmc665x_nand.obj (.text)
                  00805a20    00000d80                               : evmc665x_i2c_eeprom.obj (.text)
                  008067a0    00000bc0     bench_common.obj (.text)
                  00807360    00000a80     bench_shm.obj (.text)
                  00807de0    00000a60     ipc.lib : Ipc.obj (.text:ti_sdo_ipc_heaps_HeapMemMP_alloc__E)
                  00808840    000009e0             : Ipc.obj (.text:ti_sdo_ipc_heaps_HeapMemMP_free__E)
                  00809220    000009a0             : Ipc.obj (.text:Ipc_attach)
                  00809bc0    000009a0     ti.targets.rts6000.ae66 : System.oe66 (.text:xdc_runtime_System_doPrint__I)
                  0080a560    00000920     ipc.lib : Ipc.obj (.text:Ipc_detach)
                  0080ae80    00000920     bench_osal.obj (.text)
                  0080b7a0    00000860     ipc.lib : Ipc.obj (.text:ti_sdo_ipc_GateMP_Instance_finalize__F)
                  0080c000    00000840             : Ipc.obj (.text:MessageQ_put)
                  0080c840    00000780             : Ipc.obj (.text:ti_sdo_ipc_heaps_HeapMemMP_Instance_init__F)
                  0080cfc0    00000780     sysbios.lib : BIOS.obj (.text:ti_sysbios_family_c64p_Exception_handler__I)
                  0080d740    00000700     rts6600_elf.lib : pow.obj (.text:pow)
                  0080de40    000006c0     ti.platform.evm6657l.ae66 : evmc665x_uart.obj (.text)
                  0080e500    000006c0     ipc.lib : Ipc.obj (.text:ti_sdo_ipc_nsremote_NameServerRemoteNotify_Instance_init__F)
                  0080ebc0    000006a0             : Ipc.obj (.text:NameServer_add)
                  0080f260    00000660     sysbios.lib : BIOS.obj (.text:ti_sysbios_heaps_HeapMem_free__E)
                  0080f8c0    00000620     ipc.lib : Ipc.obj (.text:Notify_sendEvent)
                  0080fee0    00000620     sysbios.lib : BIOS.obj (.text:ti_sysbios_heaps_HeapMem_alloc__E)
                  00810500    000005e0     ipc.lib : Ipc.obj (.text:Notify_registerEventSingle)
                  00810ae0    000005c0             : Ipc.obj (.text:Notify_unregisterEventSingle)
                  008110a0    000005c0     rts6600_elf.lib : divd.obj (.text:__c6xabi_divd)
                  00811660    000005c0                     : _printfi.obj (.text:_getarg_diouxp)
                  00811c20    000005c0     ti.platform.evm6657l.ae66 : evmc665x_spi.obj (.text)
                  008121e0    000005c0     ipc.lib : Ipc.obj (.text:ti_sdo_ipc_SharedRegion_start__F)
                  008127a0    000005c0     sysbios.lib : BIOS.obj (.text:ti_sysbios_timers_timer64_Timer_Module_startup__F)
                  00812d60    00000580     ipc.lib : Ipc.obj (.text:ti_sdo_ipc_nsremote_NameServerRemoteNotify_get__F)
                  008132e0    00000560             : Ipc.obj (.text:MessageQ_free)
                  00813840    00000560             : Ipc.obj (.text:NameServer_get)
                  00813da0    00000540             : Ipc.obj (.text:ti_sdo_ipc_Ipc_procSyncStart__I)
                  008142e0    00000520     ti.platform.evm6657l.ae66 : evmc665x_nor.obj (.text)
                  00814800    000004e0     ipc.lib : Ipc.obj (.text:ti_sdo_ipc_notifyDrivers_NotifyDriverCirc_Instance_init__F)
                  00814ce0    000004c0     ti.platform.evm6657l.ae66 : evmc665x_fpga.obj (.text)
                  008151a0    000004a0     ipc.lib : Ipc.obj (.text:ti_sdo_ipc_gates_GatePeterson_Instance_init__F)
                  00815640    00000460     rts6600_elf.lib : _printfi.obj (.text:_printfi)
                  00815aa0    00000460                     : _printfi.obj (.text:_setfield)
                  00815f00    00000460     ipc.lib : Ipc.obj (.text:ti_sdo_ipc_GateMP_setRegion0Reserved__F)
                  00816360    00000460             : Ipc.obj (.text:ti_sdo_ipc_Ipc_procSyncFinish__I)
                  008167c0    00000460             : Ipc.obj (.text:ti_sdo_ipc_MessageQ_Instance_init__F)
                  00816c20    00000440             : Ipc.obj (.text:ti_sdo_ipc_heaps_HeapMemMP_getStats__E)
                  00817060    00000440             : Ipc.obj (.text:ti_sdo_ipc_heaps_HeapMemMP_postInit__I)
                  008174a0    00000400             : Ipc.obj (.text:ti_sdo_ipc_Notify_Instance_init__F)
                  008178a0    00000400     sysbios.lib : BIOS.obj (.text:ti_sysbios_knl_Semaphore_pend__E)
                  00817ca0    000003c0     ipc.lib : Ipc.obj (.text:ti_sdo_ipc_SharedRegion_reserveMemory__F)
                  00818060    000003c0     sysbios.lib : BIOS.obj (.text:ti_sysbios_knl_Task_setPri__E)
                  00818420    000003a0     rts6600_elf.lib : fputs.obj (.text:fputs)
                  008187c0    00000380     ipc.lib : Ipc.obj (.text:HeapMemMP_sharedMemReq)
                  00818b40    00000380             : Ipc.obj (.text:MessageQ_alloc)
                  00818ec0    00000340             : Ipc.obj (.text:GateMP_sharedMemReq)
                  00819200    00000340             : Ipc.obj (.text:ti_sdo_ipc_nsremote_NameServerRemoteNotify_swiFxn__I)
                  00819540    00000340     bench_shm_pe66.oe66 (.text:xdc_runtime_System_printfExtend__I)
                  00819880    00000320     rts6600_elf.lib : _printfi.obj (.text:_pproc_fge)
                  00819ba0    00000300     ipc.lib : Ipc.obj (.text:GateMP_openByAddr)
                  00819ea0    00000300     sysbios.lib : BIOS.obj (.text:ti_sysbios_family_c64p_Hwi_dispatchC__I)
                  0081a1a0    000002e0     ipc.lib : Ipc.obj (.text:SharedRegion_getEntry)
                  0081a480    000002e0             : Ipc.obj (.text:SharedRegion_getPtr)
                  0081a760    000002e0     rts6600_elf.lib : _printfi.obj (.text:_pproc_fwp)
                  0081aa40    000002e0     ipc.lib : Ipc.obj (.text:ti_sdo_ipc_notifyDrivers_NotifyDriverCirc_isr__I)
                  0081ad20    000002e0     sysbios.lib : BIOS.obj (.text:ti_sysbios_gates_GateMutexPri_enter__E)
                  0081b000    000002e0                 : BIOS.obj (.text:ti_sysbios_knl_Task_Module_startup__F)
                  0081b2e0    000002c0     ipc.lib : Ipc.obj (.text:MessageQ_open)
                  0081b5a0    000002a0             : Ipc.obj (.text:Ipc_start)
                  0081b840    000002a0             : Ipc.obj (.text:NameServer_getLocal)
                  0081bae0    000002a0     rts6600_elf.lib : _printfi.obj (.text:fcvt)
                  0081bd80    000002a0     sysbios.lib : BIOS.obj (.text:ti_sysbios_knl_Clock_workFunc__E)
                  0081c020    00000280     ipc.lib : Ipc.obj (.text:SharedRegion_getSRPtr)
                  0081c2a0    00000280     rts6600_elf.lib : divf.obj (.text:__c6xabi_divf)
                  0081c520    00000280     sysbios.lib : BIOS.obj (.text:deviceConfig$44)
                  0081c7a0    00000280     rts6600_elf.lib : _printfi.obj (.text:ecvt)
                  0081ca20    00000280     ipc.lib : Ipc.obj (.text:ti_sdo_ipc_notifyDrivers_NotifyDriverCirc_sharedMemReq__F)
                  0081cca0    00000280     sysbios.lib : BIOS.obj (.text:ti_sysbios_knl_Clock_Instance_init__F)
                  0081cf20    00000280                 : BIOS.obj (.text:ti_sysbios_knl_Task_exit__E)
                  0081d1a0    00000280     ti.targets.rts6000.ae66 : Core-mem.oe66 (.text:xdc_runtime_Core_createObject__I)
                  0081d420    00000280                             : Error.oe66 (.text:xdc_runtime_Error_raiseX__F)
                  0081d6a0    00000260     ipc.lib : Ipc.obj (.text:ti_sdo_ipc_heaps_HeapMemMP_Instance_finalize__F)
                  0081d900    00000260     ti.targets.rts6000.ae66 : Startup.oe66 (.text:xdc_runtime_Startup_startMods__I)
                  0081db60    00000240     rts6600_elf.lib : imath64.obj (.text:__c6xabi_divull)
                  0081dda0    00000240                     : _printfi.obj (.text:_pconv_e)
                  0081dfe0    00000240                     : _printfi.obj (.text:_pproc_diouxp)
                  0081e220    00000240     ipc.lib : Ipc.obj (.text:ti_sdo_ipc_MessageQ_Instance_finalize__F)
                  0081e460    00000240             : Ipc.obj (.text:ti_sdo_ipc_notifyDrivers_NotifyDriverCirc_sendEvent__E)
                  0081e6a0    00000240     sysbios.lib : BIOS.obj (.text:ti_sysbios_family_c64p_Exception_internalHandler__I)
                  0081e8e0    00000240                 : BIOS.obj (.text:ti_sysbios_knl_Semaphore_post__E)
                  0081eb20    00000220     ipc.lib : Ipc.obj (.text:MessageQ_get)
                  0081ed40    00000220     rts6600_elf.lib : _printfi.obj (.text:_pproc_str)
                  0081ef60    00000220                     : fputc.obj (.text:fputc)
                  0081f180    00000220     sysbios.lib : BIOS.obj (.text:ti_sysbios_family_c64p_Hwi_reconfig__E)
                  0081f3a0    00000220                 : BIOS.obj (.text:ti_sysbios_knl_Swi_run__I)
                  0081f5c0    00000220                 : BIOS.obj (.text:ti_sysbios_knl_Task_schedule__I)
                  0081f7e0    00000220                 : BIOS.obj (.text:ti_sysbios_knl_Task_startup__E)
                  0081fa00    00000200     ipc.lib : Ipc.obj (.text:GateMP_enter)
                  0081fc00    00000200             : Ipc.obj (.text:GateMP_leave)
                  0081fe00    00000200     rts6600_elf.lib : _printfi.obj (.text:_pconv_g)
                  00820000    00000200     sysbios.lib : c64p_Hwi_disp_always.obj (.text:_ti_sysbios_family_c64p_Hwi_dispatchAlways)
                  00820200    00000200                 : BIOS.obj (.text:block$56)
                  00820400    00000200     rts6600_elf.lib : setvbuf.obj (.text:setvbuf)
                  00820600    00000200     ipc.lib : Ipc.obj (.text:ti_sdo_ipc_family_c647x_MultiProcSetup_init__I)
                  00820800    000001e0             : Ipc.obj (.text:ti_sdo_ipc_GateMP_attach__F)
                  008209e0    000001e0             : Ipc.obj (.text:ti_sdo_ipc_GateMP_getFreeResource__I)
                  00820bc0    000001e0     sysbios.lib : BIOS.obj (.text:ti_sysbios_knl_Task_postInit__I)
                  00820da0    000001e0                 : BIOS.obj (.text:ti_sysbios_timers_timer64_Timer_getFreq__E)
                  00820f80    000001c0     ipc.lib : Ipc.obj (.text:HeapMemMP_openByAddr)
                  00821140    000001c0     rts6600_elf.lib : _printfi.obj (.text:_mcpy)
                  00821300    000001c0     sysbios.lib : BIOS.obj (.text:ti_sysbios_knl_Swi_Instance_init__F)
                  008214c0    000001c0                 : BIOS.obj (.text:ti_sysbios_knl_Task_checkStacks__E)
                  00821680    000001c0                 : BIOS.obj (.text:ti_sysbios_timers_timer64_Timer_setPeriodMicroSecs__E)
                  00821840    000001a0     rts6600_elf.lib : trgdrv.obj (.text:HOSTrename)
                  008219e0    000001a0     ipc.lib : Ipc.obj (.text:SharedRegion_getCacheLineSize)
                  00821b80    000001a0             : Ipc.obj (.text:SharedRegion_getHeap)
                  00821d20    000001a0             : Ipc.obj (.text:SharedRegion_isCacheEnabled)
                  00821ec0    000001a0     rts6600_elf.lib : imath40.obj (.text:__c6xabi_divul)
                  00822060    000001a0     ipc.lib : Ipc.obj (.text:ti_sdo_ipc_GateMP_openRegion0Reserved__F)
                  00822200    000001a0             : Ipc.obj (.text:ti_sdo_ipc_nsremote_NameServerRemoteNotify_attach__E)
                  008223a0    000001a0             : Ipc.obj (.text:ti_sdo_ipc_transports_TransportShmNotify_put__E)
                  00822540    000001a0     sysbios.lib : BIOS.obj (.text:ti_sysbios_gates_GateMutex_enter__E)
                  008226e0    000001a0                 : BIOS.obj (.text:ti_sysbios_timers_timer64_Timer_start__E)
                  00822880    00000180     ipc.lib : Ipc.obj (.text:MultiProc_getName)
                  00822a00    00000180             : Ipc.obj (.text:MultiProc_setLocalId)
                  00822b80    00000180             : Ipc.obj (.text:NameServer_getHandle)
                  00822d00    00000180             : Ipc.obj (.text:Notify_intLineRegistered)
                  00822e80    00000180     rts6600_elf.lib : copy_decompress_rle.obj (.text:__TI_decompress_rle_core)
                  00823000    00000180                     : frexp.obj (.text:frexp)
                  00823180    00000180     sysbios.lib : c64p_Exception_asm.obj (.text)
                  00823300    00000180     ipc.lib : Ipc.obj (.text:ti_sdo_ipc_MessageQ_registerTransport__F)
                  00823480    00000180             : Ipc.obj (.text:ti_sdo_ipc_Notify_Module_startup__F)
                  00823600    00000180             : Ipc.obj (.text:ti_sdo_ipc_gates_GatePeterson_enter__E)
                  00823780    00000180             : Ipc.obj (.text:ti_sdo_utils_NameServer_Module_startup__F)
                  00823900    00000180     sysbios.lib : BIOS.obj (.text:ti_sysbios_heaps_HeapMem_Instance_init__F)
                  00823a80    00000180                 : BIOS.obj (.text:ti_sysbios_knl_Swi_schedule__I)
                  00823c00    00000180                 : BIOS.obj (.text:ti_sysbios_knl_Task_unblockI__E)
                  00823d80    00000180     ti.targets.rts6000.ae66 : Text.oe66 (.text:xdc_runtime_Text_putSite__F)
                  00823f00    00000160     rts6600_elf.lib : ldexp.obj (.text:ldexp)
                  00824060    00000160                     : sqrt.obj (.text:sqrt)
                  008241c0    00000160     ti.platform.evm6657l.ae66 : evmc665x_phy.obj (.text)
                  00824320    00000160     ipc.lib : Ipc.obj (.text:ti_sdo_ipc_GateMP_createLocal__F)
                  00824480    00000160             : Ipc.obj (.text:ti_sdo_ipc_MessageQ_unregisterTransport__F)
                  008245e0    00000160             : Ipc.obj (.text:ti_sdo_ipc_gates_GateHWSem_Instance_init__F)
                  00824740    00000160             : Ipc.obj (.text:ti_sdo_utils_NameServer_isRegistered__E)
                  008248a0    00000160             : Ipc.obj (.text:ti_sdo_utils_NameServer_registerRemoteDriver__E)
                  00824a00    00000160             : Ipc.obj (.text:ti_sdo_utils_NameServer_unregisterRemoteDriver__E)
                  00824b60    00000160     sysbios.lib : BIOS.obj (.text:ti_sysbios_syncs_SyncSem_Instance_init__F)
                  00824cc0    00000140     ti.csl.ae66 : csl_chip.oe66 (.text:CSL_chipReadReg)
                  00824e00    00000140     ipc.lib : Ipc.obj (.text:GateMP_close)
                  00824f40    00000140             : Ipc.obj (.text:MessageQ_registerHeap)
                  00825080    00000140             : Ipc.obj (.text:Notify_attach)
                  008251c0    00000140     boot.ae66 : autoinit.oe66 (.text:_auto_init_elf)
                  00825300    00000140     rts6600_elf.lib : _printfi.obj (.text:_pproc_fflags)
                  00825440    00000140                     : lowlev.obj (.text:getdevice)
                  00825580    00000140     ipc.lib : Ipc.obj (.text:ti_sdo_ipc_Notify_exec__F)
                  008256c0    00000140     sysbios.lib : BIOS.obj (.text:ti_sysbios_family_c64p_Hwi_Module_startup__F)
                  00825800    00000140                 : BIOS.obj (.text:ti_sysbios_family_c66_Cache_Module_startup__F)
                  00825940    00000140                 : BIOS.obj (.text:ti_sysbios_gates_GateSwi_enter__E)
                  00825a80    00000140                 : BIOS.obj (.text:ti_sysbios_knl_Clock_Instance_finalize__F)
                  00825bc0    00000140                 : BIOS.obj (.text:ti_sysbios_knl_Semaphore_Instance_init__F)
                  00825d00    00000140                 : BIOS.obj (.text:ti_sysbios_knl_Swi_post__E)
                  00825e40    00000140                 : BIOS.obj (.text:ti_sysbios_knl_Task_blockI__E)
                  00825f80    00000140                 : BIOS.obj (.text:ti_sysbios_knl_Task_yield__E)
                  008260c0    00000120     rts6600_elf.lib : fclose.obj (.text:_closefile)
                  008261e0    00000120                     : _printfi.obj (.text:_ltostr)
                  00826300    00000120                     : fseek.obj (.text:fseek)
                  00826420    00000120     sysbios.lib : BIOS.obj (.text:rtsUnlock$0)
                  00826540    00000120     ipc.lib : Ipc.obj (.text:ti_sdo_ipc_MessageQ_Module_startup__F)
                  00826660    00000120             : Ipc.obj (.text:ti_sdo_ipc_family_c647x_Interrupt_intRegister__E)
                  00826780    00000120             : Ipc.obj (.text:ti_sdo_ipc_nsremote_NameServerRemoteNotify_Instance_finalize__F)
                  008268a0    00000100     rts6600_elf.lib : trgdrv.obj (.text:HOSTlseek)
                  008269a0    00000100                     : _io_perm.obj (.text:_wrt_ok)
                  00826aa0    00000100     sysbios.lib : BIOS.obj (.text:initDevice$44)
                  00826ba0    00000100     ipc.lib : Ipc.obj (.text:ti_sdo_ipc_GateMP_start__F)
                  00826ca0    00000100             : Ipc.obj (.text:ti_sdo_ipc_Notify_Instance_finalize__F)
                  00826da0    00000100             : Ipc.obj (.text:ti_sdo_ipc_SharedRegion_attach__F)
                  00826ea0    00000100             : Ipc.obj (.text:ti_sdo_ipc_SharedRegion_clearReservedMemory__F)
                  00826fa0    00000100             : Ipc.obj (.text:ti_sdo_ipc_family_c647x_Interrupt_Module_startup__F)
                  008270a0    00000100             : Ipc.obj (.text:ti_sdo_ipc_gates_GateHWSem_Module_startup__F)
                  008271a0    00000100             : Ipc.obj (.text:ti_sdo_ipc_gates_GateMPSupportNull_enter__E)
                  008272a0    00000100             : Ipc.obj (.text:ti_sdo_ipc_gates_GateMPSupportNull_leave__E)
                  008273a0    00000100             : Ipc.obj (.text:ti_sdo_ipc_transports_TransportShmNotify_Instance_init__F)
                  008274a0    00000100     sysbios.lib : BIOS.obj (.text:ti_sysbios_gates_GateMutexPri_leave__E)
                  008275a0    00000100                 : BIOS.obj (.text:ti_sysbios_knl_Clock_startI__E)
                  008276a0    00000100                 : BIOS.obj (.text:ti_sysbios_knl_Swi_restoreHwi__E)
                  008277a0    00000100     ti.targets.rts6000.ae66 : Core-mem.oe66 (.text:xdc_runtime_Core_deleteObject__I)
                  008278a0    00000100                             : Startup.oe66 (.text:xdc_runtime_Startup_exec__F)
                  008279a0    00000100                             : Text.oe66 (.text:xdc_runtime_Text_putMod__F)
                  00827aa0    00000100                             : Text.oe66 (.text:xdc_runtime_Text_visitRope2__I)
                  00827ba0    000000e0     rts6600_elf.lib : trgdrv.obj (.text:HOSTopen)
                  00827c80    000000e0                     : _printfi.obj (.text:_div)
                  00827d60    000000e0                     : atoi.obj (.text:atoi)
                  00827e40    000000e0                     : lowlev.obj (.text:close)
                  00827f20    000000e0                     : copy_zero_init.obj (.text:decompress:ZI:__TI_zero_init)
                  00828000    000000e0                     : fflush.obj (.text:fflush)
                  008280e0    000000e0                     : ltoa.obj (.text:ltoa)
                  008281c0    000000e0                     : memset.obj (.text:memset)
                  008282a0    000000e0                     : printf.obj (.text:printf)
                  00828380    000000e0     bench_shm_pe66.oe66 (.text:ti_sdo_ipc_Notify_Object__create__S)
                  00828460    000000e0     ipc.lib : Ipc.obj (.text:ti_sdo_ipc_Notify_detach__F)
                  00828540    000000e0             : Ipc.obj (.text:ti_sdo_ipc_family_c647x_NotifyCircSetup_attach__E)
                  00828620    000000e0             : Ipc.obj (.text:ti_sdo_ipc_gates_GateHWSem_enter__E)
                  00828700    000000e0             : Ipc.obj (.text:ti_sdo_ipc_notifyDrivers_NotifyDriverCirc_disableEvent__E)
                  008287e0    000000e0             : Ipc.obj (.text:ti_sdo_ipc_notifyDrivers_NotifyDriverCirc_enable__E)
                  008288c0    000000e0     sysbios.lib : BIOS.obj (.text:ti_sysbios_family_c64p_Hwi_Instance_finalize__F)
                  008289a0    000000e0                 : BIOS.obj (.text:ti_sysbios_family_c64p_Hwi_Instance_init__F)
                  00828a80    000000e0     bench_shm_pe66.oe66 (.text:ti_sysbios_family_c64p_Hwi_Object__create__S)
                  00828b60    000000e0     sysbios.lib : BIOS.obj (.text:ti_sysbios_knl_Clock_start__E)
                  00828c40    000000e0                 : BIOS.obj (.text:ti_sysbios_timers_timer64_Timer_startup__E)
                  00828d20    000000e0     ti.targets.rts6000.ae66 : Error.oe66 (.text:xdc_runtime_Error_print__F)
                  00828e00    000000e0                             : Memory.oe66 (.text:xdc_runtime_Memory_alloc__F)
                  00828ee0    000000c0     rts6600_elf.lib : trgdrv.obj (.text:HOSTread)
                  00828fa0    000000c0                     : trgdrv.obj (.text:HOSTunlink)
                  00829060    000000c0                     : trgdrv.obj (.text:HOSTwrite)
                  00829120    000000c0     ipc.lib : Ipc.obj (.text:HeapMemMP_create)
                  008291e0    000000c0     rts6600_elf.lib : dtor_list.obj (.text:_Z11__TI_atexitPFYvPvES_S_)
                  008292a0    000000c0                     : dtor_list.obj (.text:__cxa_finalize)
                  00829360    000000c0                     : divu.obj (.text:__divu)
                  00829420    000000c0                     : fflush.obj (.text:_doflush)
                  008294e0    000000c0                     : exit.obj (.text:exit)
                  008295a0    000000c0     bench_shm_pe66.oe66 (.text:ti_sdo_ipc_GateMP_Object__create__S)
                  00829660    000000c0     ipc.lib : Ipc.obj (.text:ti_sdo_ipc_GateMP_getRegion0ReservedSize__F)
                  00829720    000000c0     bench_shm_pe66.oe66 (.text:ti_sdo_ipc_MessageQ_Object__create__S)
                  008297e0    000000c0     ipc.lib : Ipc.obj (.text:ti_sdo_ipc_family_c647x_Interrupt_intShmStub__I)
                  008298a0    000000c0     bench_shm_pe66.oe66 (.text:ti_sdo_ipc_gates_GatePeterson_Object__create__S)
                  00829960    000000c0     bench_shm_pe66.oe66 (.text:ti_sdo_ipc_heaps_HeapMemMP_Object__create__S)
                  00829a20    000000c0     bench_shm_pe66.oe66 (.text:ti_sdo_ipc_nsremote_NameServerRemoteNotify_Object__create__S)
                  00829ae0    000000c0     ipc.lib : Ipc.obj (.text:ti_sdo_ipc_transports_TransportShmNotifySetup_attach__E)
                  00829ba0    000000c0     bench_shm_pe66.oe66 (.text:ti_sdo_ipc_transports_TransportShmNotify_Object__create__S)
                  00829c60    000000c0     sysbios.lib : BIOS.obj (.text:ti_sysbios_BIOS_errorRaiseHook__I)
                  00829d20    000000c0                 : BIOS.obj (.text:ti_sysbios_gates_GateAll_leave__E)
                  00829de0    000000c0                 : BIOS.obj (.text:ti_sysbios_heaps_HeapMem_getStats__E)
                  00829ea0    000000c0                 : BIOS.obj (.text:ti_sysbios_knl_Clock_logTick__E)
                  00829f60    000000c0                 : BIOS.obj (.text:ti_sysbios_knl_Swi_Instance_finalize__F)
                  0082a020    000000c0     bench_shm_pe66.oe66 (.text:ti_sysbios_knl_Swi_Object__create__S)
                  0082a0e0    000000c0     bench_shm_pe66.oe66 (.text:ti_sysbios_syncs_SyncSem_Object__create__S)
                  0082a1a0    000000c0     sysbios.lib : BIOS.obj (.text:ti_sysbios_timers_timer64_Timer_stop__E)
                  0082a260    000000c0     ti.targets.rts6000.ae66 : System.oe66 (.text:xdc_runtime_System_formatNum__I)
                  0082a320    000000c0     bench_shm_pe66.oe66 (.text:xdc_runtime_knl_GateThread_Object__create__S)
                  0082a3e0    000000a0     rts6600_elf.lib : trgdrv.obj (.text:HOSTclose)
                  0082a480    000000a0     ipc.lib : Ipc.obj (.text:MessageQ_create)
                  0082a520    000000a0     rts6600_elf.lib : fltulld.obj (.text:__c6xabi_fltulld)
                  0082a5c0    000000a0                     : round.obj (.text:__c6xabi_nround)
                  0082a660    000000a0                     : remu.obj (.text:__remu)
                  0082a700    000000a0     boot.ae66 : boot.oe66 (.text:_c_int00)
                  0082a7a0    000000a0     rts6600_elf.lib : fopen.obj (.text:_cleanup)
                  0082a840    000000a0                     : _printfi.obj (.text:_ecpy)
                  0082a8e0    000000a0                     : _printfi.obj (.text:_fcpy)
                  0082a980    000000a0                     : _printfi.obj (.text:_pconv_f)
                  0082aa20    000000a0     sysbios.lib : c64p_Hwi_asm.obj (.text:_ti_sysbios_family_c64p_Hwi_plug__E)
                  0082aac0    000000a0     rts6600_elf.lib : lowlev.obj (.text:finddevice)
                  0082ab60    000000a0                     : lowlev.obj (.text:lseek)
                  0082ac00    000000a0                     : memcpy64.obj (.text:memcpy)
                  0082aca0    000000a0                     : modf.obj (.text:modf)
                  0082ad40    000000a0     ipc.lib : Ipc.obj (.text:ti_sdo_ipc_family_c647x_Interrupt_intUnregister__E)
                  0082ade0    000000a0             : Ipc.obj (.text:ti_sdo_ipc_gates_GatePeterson_leave__E)
                  0082ae80    000000a0             : Ipc.obj (.text:ti_sdo_ipc_notifyDrivers_NotifyDriverCirc_Instance_finalize__F)
                  0082af20    000000a0     sysbios.lib : BIOS.obj (.text:ti_sysbios_heaps_HeapMem_init__I)
                  0082afc0    000000a0                 : BIOS.obj (.text:ti_sysbios_syncs_SyncSem_wait__F)
                  0082b060    000000a0     rts6600_elf.lib : lowlev.obj (.text:write)
                  0082b100    000000a0     ti.targets.rts6000.ae66 : Assert.oe66 (.text:xdc_runtime_Assert_raise__I)
                  0082b1a0    00000080     rts6600_elf.lib : fixdu.obj (.text:__c6xabi_fixdu)
                  0082b220    00000080                     : fixfu.obj (.text:__c6xabi_fixfu)
                  0082b2a0    00000080                     : llshift.obj (.text:__c6xabi_llshl)
                  0082b320    00000080     sysbios.lib : c62_TaskSupport_asm.obj (.text:_ti_sysbios_family_c62_TaskSupport_swap__E)
                  0082b3a0    00000080     bench_shm_pe66.oe66 (.text:malloc)
                  0082b420    00000080     rts6600_elf.lib : trgmsg.obj (.text:readmsg)
                  0082b4a0    00000080                     : strncpy.obj (.text:strncpy)
                  0082b520    00000080     ti.platform.evm6657l.ae66 : evm665x_i2c.obj (.text)
                  0082b5a0    00000080     bench_shm_pe66.oe66 (.text:ti_sdo_ipc_gates_GateHWSem_Object__create__S)
                  0082b620    00000080     bench_shm_pe66.oe66 (.text:ti_sdo_ipc_gates_GateMPSupportNull_Object__create__S)
                  0082b6a0    00000080     bench_shm_pe66.oe66 (.text:ti_sdo_ipc_notifyDrivers_NotifyDriverCirc_Object__create__S)
                  0082b720    00000080     ipc.lib : Ipc.obj (.text:ti_sdo_ipc_nsremote_NameServerRemoteNotify_detach__E)
                  0082b7a0    00000080             : Ipc.obj (.text:ti_sdo_ipc_transports_TransportShmNotify_Instance_finalize__F)
                  0082b820    00000080     bench_shm_pe66.oe66 (.text:ti_sdo_utils_List_Object__create__S)
                  0082b8a0    00000080     sysbios.lib : BIOS.obj (.text:ti_sysbios_family_c62_TaskSupport_start__E)
                  0082b920    00000080                 : BIOS.obj (.text:ti_sysbios_family_c64p_Exception_Module_startup__F)
                  0082b9a0    00000080                 : BIOS.obj (.text:ti_sysbios_family_c64p_Hwi_eventMap__E)
                  0082ba20    00000080                 : BIOS.obj (.text:ti_sysbios_family_c66_Cache_invL1pAll__E)
                  0082baa0    00000080     bench_shm_pe66.oe66 (.text:ti_sysbios_gates_GateAll_Object__create__S)
                  0082bb20    00000080     bench_shm_pe66.oe66 (.text:ti_sysbios_gates_GateHwi_Object__create__S)
                  0082bba0    00000080     bench_shm_pe66.oe66 (.text:ti_sysbios_gates_GateMutexPri_Object__create__S)
                  0082bc20    00000080     bench_shm_pe66.oe66 (.text:ti_sysbios_gates_GateMutex_Object__create__S)
                  0082bca0    00000080     bench_shm_pe66.oe66 (.text:ti_sysbios_gates_GateSwi_Object__create__S)
                  0082bd20    00000080     sysbios.lib : BIOS.obj (.text:ti_sysbios_gates_GateSwi_leave__E)
                  0082bda0    00000080                 : BIOS.obj (.text:ti_sysbios_hal_Hwi_checkStack:ti_sysbios_hal_Hwi_checkStack)
                  0082be20    00000080     bench_shm_pe66.oe66 (.text:ti_sysbios_heaps_HeapMem_Object__create__S)
                  0082bea0    00000080     sysbios.lib : BIOS.obj (.text:ti_sysbios_knl_Clock_Module_startup__F)
                  0082bf20    00000080     bench_shm_pe66.oe66 (.text:ti_sysbios_knl_Clock_Object__create__S)
                  0082bfa0    00000080     sysbios.lib : BIOS.obj (.text:ti_sysbios_knl_Clock_getTicks__E)
                  0082c020    00000080                 : BIOS.obj (.text:ti_sysbios_knl_Idle_loop__E)
                  0082c0a0    00000080     bench_shm_pe66.oe66 (.text:ti_sysbios_knl_Queue_Object__create__S)
                  0082c120    00000080     bench_shm_pe66.oe66 (.text:ti_sysbios_knl_Semaphore_Object__create__S)
                  0082c1a0    00000080     sysbios.lib : BIOS.obj (.text:ti_sysbios_knl_Semaphore_pendTimeout__I)
                  0082c220    00000080                 : BIOS.obj (.text:ti_sysbios_knl_Swi_startup__E)
                  0082c2a0    00000080                 : BIOS.obj (.text:ti_sysbios_knl_Task_restore__E)
                  0082c320    00000080                 : BIOS.obj (.text:ti_sysbios_timers_timer64_Timer_getCount__E)
                  0082c3a0    00000080                 : BIOS.obj (.text:ti_sysbios_timers_timer64_Timer_getPeriod__E)
                  0082c420    00000080     bench_shm_pe66.oe66 (.text:ti_sysbios_xdcruntime_GateThreadSupport_Object__create__S)
                  0082c4a0    00000080     rts6600_elf.lib : lowlev.obj (.text:unlink)
                  0082c520    00000080     ti.targets.rts6000.ae66 : Core-label.oe66 (.text:xdc_runtime_Core_assignLabel__I)
                  0082c5a0    00000080                             : Core-params.oe66 (.text:xdc_runtime_Core_assignParams__I)
                  0082c620    00000080                             : System.oe66 (.text:xdc_runtime_System_atexit__F)
                  0082c6a0    00000080                             : System.oe66 (.text:xdc_runtime_System_rtsExit__I)
                  0082c720    00000080                             : Text.oe66 (.text:xdc_runtime_Text_printVisFxn__I)
                  0082c7a0    00000080                             : Text.oe66 (.text:xdc_runtime_Text_xprintf__I)
                  0082c820    00000060     ipc.lib : Ipc.obj (.text:GateMP_Params_init)
                  0082c880    00000060             : Ipc.obj (.text:HeapMemMP_Params_init)
                  0082c8e0    00000060             : Ipc.obj (.text:Notify_numIntLines)
                  0082c940    00000060     rts6600_elf.lib : frcmpyd_div.obj (.text:__c6xabi_frcmpyd_div)
                  0082c9a0    00000060                     : llshift.obj (.text:__c6xabi_llshru)
                  0082ca00    00000060                     : imath64.obj (.text:_subcull)
                  0082ca60    00000060                     : memccpy.obj (.text:memccpy)
                  0082cac0    00000060     bench_shm_pe66.oe66 (.text:ti_sdo_ipc_MessageQ_Object__get__S)
                  0082cb20    00000060     ipc.lib : Ipc.obj (.text:ti_sdo_ipc_family_c647x_NotifyCircSetup_sharedMemReq__E)
                  0082cb80    00000060             : Ipc.obj (.text:ti_sdo_ipc_gates_GateHWSem_leave__E)
                  0082cbe0    00000060             : Ipc.obj (.text:ti_sdo_ipc_gates_GatePeterson_Instance_finalize__F)
                  0082cc40    00000060             : Ipc.obj (.text:ti_sdo_ipc_gates_GatePeterson_sharedMemReq__E)
                  0082cca0    00000060             : Ipc.obj (.text:ti_sdo_ipc_transports_TransportShmNotifySetup_detach__E)
                  0082cd00    00000060             : Ipc.obj (.text:ti_sdo_ipc_transports_TransportShmNotify_notifyFxn__I)
                  0082cd60    00000060     bench_shm_pe66.oe66 (.text:ti_sdo_utils_List_Object__get__S)
                  0082cdc0    00000060     bench_shm_pe66.oe66 (.text:ti_sdo_utils_NameServer_Object__get__S)
                  0082ce20    00000060     bench_shm_pe66.oe66 (.text:ti_sysbios_BIOS_exitFunc__I)
                  0082ce80    00000060     sysbios.lib : BIOS.obj (.text:ti_sysbios_BIOS_registerRTSLock__I)
                  0082cee0    00000060                 : BIOS.obj (.text:ti_sysbios_gates_GateAll_enter__E)
                  0082cf40    00000060                 : BIOS.obj (.text:ti_sysbios_gates_GateMutex_Instance_init__F)
                  0082cfa0    00000060                 : BIOS.obj (.text:ti_sysbios_hal_Hwi_initStack:ti_sysbios_hal_Hwi_initStack)
                  0082d000    00000060     bench_shm_pe66.oe66 (.text:ti_sysbios_heaps_HeapMem_Object__get__S)
                  0082d060    00000060     bench_shm_pe66.oe66 (.text:ti_sysbios_knl_Clock_doTick__I)
                  0082d0c0    00000060     bench_shm_pe66.oe66 (.text:ti_sysbios_knl_Queue_Object__get__S)
                  0082d120    00000060     sysbios.lib : BIOS.obj (.text:ti_sysbios_knl_Swi_Module_startup__F)
                  0082d180    00000060     bench_shm_pe66.oe66 (.text:ti_sysbios_knl_Swi_Object__get__S)
                  0082d1e0    00000060     bench_shm_pe66.oe66 (.text:ti_sysbios_knl_Task_Object__get__S)
                  0082d240    00000060     sysbios.lib : BIOS.obj (.text:ti_sysbios_knl_Task_allBlockedFunction__I)
                  0082d2a0    00000060                 : BIOS.obj (.text:ti_sysbios_knl_Task_enter__I)
                  0082d300    00000060     rts6600_elf.lib : vsprintf.obj (.text:vsprintf)
                  0082d360    00000060                     : trgmsg.obj (.text:writemsg)
                  0082d3c0    00000060     bench_shm_pe66.oe66 (.text:xdc_runtime_GateNull_Object__create__S)
                  0082d420    00000060     ti.targets.rts6000.ae66 : Memory.oe66 (.text:xdc_runtime_Memory_calloc__F)
                  0082d480    00000060                             : SysStd.oe66 (.text:xdc_runtime_SysStd_abort__F)
                  0082d4e0    00000060                             : System.oe66 (.text:xdc_runtime_System_avprintf__F)
                  0082d540    00000060                             : System.oe66 (.text:xdc_runtime_System_vprintf__F)
                  0082d5a0    00000060                             : Text.oe66 (.text:xdc_runtime_Text_cordText__F)
                  0082d600    00000040     rts6600_elf.lib : isinf.obj (.text:__c6xabi_isinf)
                  0082d640    00000040                     : _printfi.obj (.text:__c6xabi_isnan)
                  0082d680    00000040                     : args_main.obj (.text:_args_main)
                  0082d6c0    00000040                     : vsprintf.obj (.text:_outs)
                  0082d700    00000040     sysbios.lib : c62_TaskSupport_asm.obj (.text:_ti_sysbios_family_c62_TaskSupport_buildTaskStack)
                  0082d740    00000040                 : c64p_Hwi_asm_switch.obj (.text:_ti_sysbios_family_xxx_Hwi_switchToIsrStack)
                  0082d780    00000040     bench_shm_pe66.oe66 (.text:free)
                  0082d7c0    00000040     bench_osal.obj (.text:l2_global_address)
                  0082d800    00000040     sysbios.lib : BIOS.obj (.text:rtsLock$0)
                  0082d840    00000040     rts6600_elf.lib : strlen.obj (.text:strlen)
                  0082d880    00000040     bench_shm_pe66.oe66 (.text:ti_sdo_ipc_GateMP_Object__delete__S)
                  0082d8c0    00000040     bench_shm_pe66.oe66 (.text:ti_sdo_ipc_GateMP_Params__init__S)
                  0082d900    00000040     bench_shm_pe66.oe66 (.text:ti_sdo_ipc_GateMP_RemoteCustom1Proxy_Object__create__S)
                  0082d940    00000040     bench_shm_pe66.oe66 (.text:ti_sdo_ipc_GateMP_RemoteCustom2Proxy_Object__create__S)
                  0082d980    00000040     bench_shm_pe66.oe66 (.text:ti_sdo_ipc_GateMP_RemoteSystemProxy_Object__create__S)
                  0082d9c0    00000040     bench_shm_pe66.oe66 (.text:ti_sdo_ipc_MessageQ_Params__init__S)
                  0082da00    00000040     bench_shm_pe66.oe66 (.text:ti_sdo_ipc_MessageQ_registerTransport__E)
                  0082da40    00000040     bench_shm_pe66.oe66 (.text:ti_sdo_ipc_Notify_Object__delete__S)
                  0082da80    00000040     ipc.lib : Ipc.obj (.text:ti_sdo_ipc_family_c647x_Interrupt_intClear__E)
                  0082dac0    00000040             : Ipc.obj (.text:ti_sdo_ipc_family_c647x_Interrupt_intSend__E)
                  0082db00    00000040     bench_shm_pe66.oe66 (.text:ti_sdo_ipc_gates_GateHWSem_Handle__label__S)
                  0082db40    00000040     bench_shm_pe66.oe66 (.text:ti_sdo_ipc_gates_GateHWSem_Object__delete__S)
                  0082db80    00000040     bench_shm_pe66.oe66 (.text:ti_sdo_ipc_gates_GateHWSem_Params__init__S)
                  0082dbc0    00000040     bench_shm_pe66.oe66 (.text:ti_sdo_ipc_gates_GateMPSupportNull_Handle__label__S)
                  0082dc00    00000040     bench_shm_pe66.oe66 (.text:ti_sdo_ipc_gates_GateMPSupportNull_Object__delete__S)
                  0082dc40    00000040     bench_shm_pe66.oe66 (.text:ti_sdo_ipc_gates_GateMPSupportNull_Params__init__S)
                  0082dc80    00000040     bench_shm_pe66.oe66 (.text:ti_sdo_ipc_gates_GatePeterson_Handle__label__S)
                  0082dcc0    00000040     bench_shm_pe66.oe66 (.text:ti_sdo_ipc_gates_GatePeterson_Object__delete__S)
                  0082dd00    00000040     bench_shm_pe66.oe66 (.text:ti_sdo_ipc_gates_GatePeterson_Params__init__S)
                  0082dd40    00000040     bench_shm_pe66.oe66 (.text:ti_sdo_ipc_heaps_HeapMemMP_Handle__label__S)
                  0082dd80    00000040     bench_shm_pe66.oe66 (.text:ti_sdo_ipc_heaps_HeapMemMP_Object__delete__S)
                  0082ddc0    00000040     bench_shm_pe66.oe66 (.text:ti_sdo_ipc_heaps_HeapMemMP_Params__init__S)
                  0082de00    00000040     bench_shm_pe66.oe66 (.text:ti_sdo_ipc_notifyDrivers_NotifyDriverCirc_Handle__label__S)
                  0082de40    00000040     bench_shm_pe66.oe66 (.text:ti_sdo_ipc_notifyDrivers_NotifyDriverCirc_InterruptProxy_intRegister__E)
                  0082de80    00000040     bench_shm_pe66.oe66 (.text:ti_sdo_ipc_notifyDrivers_NotifyDriverCirc_Object__delete__S)
                  0082dec0    00000040     bench_shm_pe66.oe66 (.text:ti_sdo_ipc_notifyDrivers_NotifyDriverCirc_Params__init__S)
                  0082df00    00000040     ipc.lib : Ipc.obj (.text:ti_sdo_ipc_notifyDrivers_NotifyDriverCirc_disable__E)
                  0082df40    00000040             : Ipc.obj (.text:ti_sdo_ipc_notifyDrivers_NotifyDriverCirc_enableEvent__E)
                  0082df80    00000040             : Ipc.obj (.text:ti_sdo_ipc_notifyDrivers_NotifyDriverCirc_registerEvent__E)
                  0082dfc0    00000040             : Ipc.obj (.text:ti_sdo_ipc_notifyDrivers_NotifyDriverCirc_unregisterEvent__E)
                  0082e000    00000040     bench_shm_pe66.oe66 (.text:ti_sdo_ipc_nsremote_NameServerRemoteNotify_Handle__label__S)
                  0082e040    00000040     bench_shm_pe66.oe66 (.text:ti_sdo_ipc_nsremote_NameServerRemoteNotify_Object__delete__S)
                  0082e080    00000040     bench_shm_pe66.oe66 (.text:ti_sdo_ipc_nsremote_NameServerRemoteNotify_Object__first__S)
                  0082e0c0    00000040     bench_shm_pe66.oe66 (.text:ti_sdo_ipc_nsremote_NameServerRemoteNotify_Object__next__S)
                  0082e100    00000040     bench_shm_pe66.oe66 (.text:ti_sdo_ipc_nsremote_NameServerRemoteNotify_Params__init__S)
                  0082e140    00000040     bench_shm_pe66.oe66 (.text:ti_sdo_ipc_nsremote_NameServerRemoteNotify_get__E)
                  0082e180    00000040     ipc.lib : Ipc.obj (.text:ti_sdo_ipc_nsremote_NameServerRemoteNotify_sharedMemReq__E)
                  0082e1c0    00000040     bench_shm_pe66.oe66 (.text:ti_sdo_ipc_transports_TransportShmNotify_Handle__label__S)
                  0082e200    00000040     bench_shm_pe66.oe66 (.text:ti_sdo_ipc_transports_TransportShmNotify_Object__delete__S)
                  0082e240    00000040     bench_shm_pe66.oe66 (.text:ti_sdo_ipc_transports_TransportShmNotify_Params__init__S)
                  0082e280    00000040     bench_shm_pe66.oe66 (.text:ti_sdo_utils_List_Object__destruct__S)
                  0082e2c0    00000040     bench_shm_pe66.oe66 (.text:ti_sdo_utils_NameServer_Module__startupDone__F)
                  0082e300    00000040     bench_shm_pe66.oe66 (.text:ti_sdo_utils_NameServer_Object__first__S)
                  0082e340    00000040     bench_shm_pe66.oe66 (.text:ti_sdo_utils_NameServer_Object__next__S)
                  0082e380    00000040     bench_shm_pe66.oe66 (.text:ti_sysbios_BIOS_startFunc__I)
                  0082e3c0    00000040     sysbios.lib : BIOS.obj (.text:ti_sysbios_BIOS_start__E)
                  0082e400    00000040     bench_shm_pe66.oe66 (.text:ti_sysbios_family_c64p_Hwi_Module__startupDone__F)
                  0082e440    00000040     bench_shm_pe66.oe66 (.text:ti_sysbios_family_c64p_Hwi_Object__delete__S)
                  0082e480    00000040     bench_shm_pe66.oe66 (.text:ti_sysbios_family_c64p_Hwi_Params__init__S)
                  0082e4c0    00000040     sysbios.lib : BIOS.obj (.text:ti_sysbios_family_c64p_Hwi_disableInterrupt__E)
                  0082e500    00000040                 : BIOS.obj (.text:ti_sysbios_family_c64p_Hwi_enableInterrupt__E)
                  0082e540    00000040                 : BIOS.obj (.text:ti_sysbios_family_c66_Cache_wait__E)
                  0082e580    00000040     bench_shm_pe66.oe66 (.text:ti_sysbios_gates_GateAll_Handle__label__S)
                  0082e5c0    00000040     bench_shm_pe66.oe66 (.text:ti_sysbios_gates_GateAll_Object__delete__S)
                  0082e600    00000040     bench_shm_pe66.oe66 (.text:ti_sysbios_gates_GateHwi_Handle__label__S)
                  0082e640    00000040     bench_shm_pe66.oe66 (.text:ti_sysbios_gates_GateHwi_Object__delete__S)
                  0082e680    00000040     bench_shm_pe66.oe66 (.text:ti_sysbios_gates_GateMutexPri_Handle__label__S)
                  0082e6c0    00000040     sysbios.lib : BIOS.obj (.text:ti_sysbios_gates_GateMutexPri_Instance_finalize__F)
                  0082e700    00000040                 : BIOS.obj (.text:ti_sysbios_gates_GateMutexPri_Instance_init__F)
                  0082e740    00000040     bench_shm_pe66.oe66 (.text:ti_sysbios_gates_GateMutexPri_Object__delete__S)
                  0082e780    00000040     bench_shm_pe66.oe66 (.text:ti_sysbios_gates_GateMutexPri_Object__destruct__S)
                  0082e7c0    00000040     bench_shm_pe66.oe66 (.text:ti_sysbios_gates_GateMutex_Handle__label__S)
                  0082e800    00000040     sysbios.lib : BIOS.obj (.text:ti_sysbios_gates_GateMutex_Instance_finalize__F)
                  0082e840    00000040     bench_shm_pe66.oe66 (.text:ti_sysbios_gates_GateMutex_Object__delete__S)
                  0082e880    00000040     sysbios.lib : BIOS.obj (.text:ti_sysbios_gates_GateMutex_leave__E)
                  0082e8c0    00000040     bench_shm_pe66.oe66 (.text:ti_sysbios_gates_GateSwi_Handle__label__S)
                  0082e900    00000040     bench_shm_pe66.oe66 (.text:ti_sysbios_gates_GateSwi_Object__delete__S)
                  0082e940    00000040     bench_shm_pe66.oe66 (.text:ti_sysbios_hal_Cache_CacheProxy_inv__E)
                  0082e980    00000040     bench_shm_pe66.oe66 (.text:ti_sysbios_hal_Cache_CacheProxy_wbInv__E)
                  0082e9c0    00000040     bench_shm_pe66.oe66 (.text:ti_sysbios_hal_Cache_CacheProxy_wb__E)
                  0082ea00    00000040     bench_shm_pe66.oe66 (.text:ti_sysbios_hal_Timer_Module__startupDone__F)
                  0082ea40    00000040     bench_shm_pe66.oe66 (.text:ti_sysbios_heaps_HeapMem_Handle__label__S)
                  0082ea80    00000040     bench_shm_pe66.oe66 (.text:ti_sysbios_heaps_HeapMem_Object__delete__S)
                  0082eac0    00000040     bench_shm_pe66.oe66 (.text:ti_sysbios_knl_Clock_Object__destruct__S)
                  0082eb00    00000040     bench_shm_pe66.oe66 (.text:ti_sysbios_knl_Clock_Params__init__S)
                  0082eb40    00000040     bench_shm_pe66.oe66 (.text:ti_sysbios_knl_Queue_Object__destruct__S)
                  0082eb80    00000040     sysbios.lib : BIOS.obj (.text:ti_sysbios_knl_Semaphore_Instance_finalize__F)
                  0082ebc0    00000040     bench_shm_pe66.oe66 (.text:ti_sysbios_knl_Semaphore_Object__delete__S)
                  0082ec00    00000040     bench_shm_pe66.oe66 (.text:ti_sysbios_knl_Semaphore_Object__destruct__S)
                  0082ec40    00000040     bench_shm_pe66.oe66 (.text:ti_sysbios_knl_Semaphore_Params__init__S)
                  0082ec80    00000040     bench_shm_pe66.oe66 (.text:ti_sysbios_knl_Swi_Object__destruct__S)
                  0082ecc0    00000040     bench_shm_pe66.oe66 (.text:ti_sysbios_knl_Swi_Params__init__S)
                  0082ed00    00000040     bench_shm_pe66.oe66 (.text:ti_sysbios_knl_Task_Object__first__S)
                  0082ed40    00000040     bench_shm_pe66.oe66 (.text:ti_sysbios_knl_Task_Object__next__S)
                  0082ed80    00000040     bench_shm_pe66.oe66 (.text:ti_sysbios_syncs_SyncSem_Handle__label__S)
                  0082edc0    00000040     sysbios.lib : BIOS.obj (.text:ti_sysbios_syncs_SyncSem_Instance_finalize__F)
                  0082ee00    00000040     bench_shm_pe66.oe66 (.text:ti_sysbios_syncs_SyncSem_Object__delete__S)
                  0082ee40    00000040     bench_shm_pe66.oe66 (.text:ti_sysbios_timers_timer64_Timer_Module__startupDone__F)
                  0082ee80    00000040     sysbios.lib : BIOS.obj (.text:ti_sysbios_xdcruntime_GateThreadSupport_Instance_finalize__F)
                  0082eec0    00000040                 : BIOS.obj (.text:ti_sysbios_xdcruntime_GateThreadSupport_Instance_init__F)
                  0082ef00    00000040     bench_shm_pe66.oe66 (.text:ti_sysbios_xdcruntime_GateThreadSupport_Object__delete__S)
                  0082ef40    00000040     sysbios.lib : BIOS.obj (.text:ti_sysbios_xdcruntime_GateThreadSupport_enter__F)
                  0082ef80    00000040                 : BIOS.obj (.text:ti_sysbios_xdcruntime_GateThreadSupport_leave__F)
                  0082efc0    00000040     ti.targets.rts6000.ae66 : Error.oe66 (.text:xdc_runtime_Error_check__F)
                  0082f000    00000040                             : Error.oe66 (.text:xdc_runtime_Error_init__F)
                  0082f040    00000040     bench_shm_pe66.oe66 (.text:xdc_runtime_Error_raiseX__E)
                  0082f080    00000040     bench_shm_pe66.oe66 (.text:xdc_runtime_GateNull_Handle__label__S)
                  0082f0c0    00000040     bench_shm_pe66.oe66 (.text:xdc_runtime_GateNull_Object__delete__S)
                  0082f100    00000040     ti.targets.rts6000.ae66 : Gate.oe66 (.text:xdc_runtime_Gate_leaveSystem__F)
                  0082f140    00000040     bench_shm_pe66.oe66 (.text:xdc_runtime_IHeap_alloc)
                  0082f180    00000040     bench_shm_pe66.oe66 (.text:xdc_runtime_IHeap_free)
                  0082f1c0    00000040     ti.targets.rts6000.ae66 : Memory.oe66 (.text:xdc_runtime_Memory_free__F)
                  0082f200    00000040                             : Registry.oe66 (.text:xdc_runtime_Registry_findById__F)
                  0082f240    00000040     bench_shm_pe66.oe66 (.text:xdc_runtime_Startup_exec__I)
                  0082f280    00000040     ti.targets.rts6000.ae66 : System.oe66 (.text:xdc_runtime_System_abort__F)
                  0082f2c0    00000040     bench_shm_pe66.oe66 (.text:xdc_runtime_System_aprintf__E)
                  0082f300    00000040     bench_shm_pe66.oe66 (.text:xdc_runtime_System_printf__E)
                  0082f340    00000040     bench_shm_pe66.oe66 (.text:xdc_runtime_System_sprintf__E)
                  0082f380    00000040     ti.targets.rts6000.ae66 : Text.oe66 (.text:xdc_runtime_Text_ropeText__F)
                  0082f3c0    00000040     bench_shm_pe66.oe66 (.text:xdc_runtime_Text_visitRope__I)
                  0082f400    00000040     bench_shm_pe66.oe66 (.text:xdc_runtime_knl_GateThread_Handle__label__S)
                  0082f440    00000040     ti.targets.rts6000.ae66 : GateThread.oe66 (.text:xdc_runtime_knl_GateThread_Instance_finalize__F)
                  0082f480    00000040                             : GateThread.oe66 (.text:xdc_runtime_knl_GateThread_Instance_init__F)
                  0082f4c0    00000040     bench_shm_pe66.oe66 (.text:xdc_runtime_knl_GateThread_Object__delete__S)
                  0082f500    00000040     bench_shm_pe66.oe66 (.text:xdc_runtime_knl_GateThread_Proxy_Object__create__S)
                  0082f540    00000020     ipc.lib : Ipc.obj (.text:GateMP_getDefaultRemote)
                  0082f560    00000020             : Ipc.obj (.text:MultiProc_getBaseIdOfCluster)
                  0082f580    00000020             : Ipc.obj (.text:MultiProc_getNumProcessors)
                  0082f5a0    00000020             : Ipc.obj (.text:MultiProc_self)
                  0082f5c0    00000020     rts6600_elf.lib : errno.obj (.text:__c6xabi_errno_addr)
                  0082f5e0    00000020                     : negll.obj (.text:__c6xabi_negll)
                  0082f600    00000020                     : trunc.obj (.text:__c6xabi_trunc)
                  0082f620    00000020                     : dtor_list.obj (.text:__cxa_atexit)
                  0082f640    00000020                     : dtor_list.obj (.text:__cxa_ia64_exit)
                  0082f660    00000020     ti.targets.rts6000.ae66 : xdc_noinit.oe66 (.text:__xdc__init)
                  0082f680    00000020     rts6600_elf.lib : _lock.obj (.text:_nop)
                  0082f6a0    00000020                     : printf.obj (.text:_outc)
                  0082f6c0    00000020                     : vsprintf.obj (.text:_outc)
                  0082f6e0    00000020                     : printf.obj (.text:_outs)
                  0082f700    00000020                     : _lock.obj (.text:_register_lock)
                  0082f720    00000020                     : _lock.obj (.text:_register_unlock)
                  0082f740    00000020     sysbios.lib : c62_TaskSupport_asm.obj (.text:_ti_sysbios_family_c62_TaskSupport_glue)
                  0082f760    00000020                 : c64p_Hwi_asm_switch.obj (.text:_ti_sysbios_family_xxx_Hwi_switchToTaskStack)
                  0082f780    00000020     rts6600_elf.lib : exit.obj (.text:abort)
                  0082f7a0    00000020                     : dtor_list.obj (.text:atexit)
                  0082f7c0    00000020                     : copy_decompress_none.obj (.text:decompress:none:__TI_decompress_none)
                  0082f7e0    00000020                     : copy_decompress_rle.obj (.text:decompress:rle24:__TI_decompress_rle24)
                  0082f800    00000020     sysbios.lib : BIOS.obj (.text:nullFunc$0)
                  0082f820    00000020     rts6600_elf.lib : fputc.obj (.text:putc)
                  0082f840    00000020                     : fputc.obj (.text:putchar)
                  0082f860    00000020     bench_shm_pe66.oe66 (.text:ti_sdo_ipc_GateMP_RemoteCustom1Proxy_Object__delete__S)
                  0082f880    00000020     bench_shm_pe66.oe66 (.text:ti_sdo_ipc_GateMP_RemoteCustom1Proxy_Params__init__S)
                  0082f8a0    00000020     bench_shm_pe66.oe66 (.text:ti_sdo_ipc_GateMP_RemoteCustom1Proxy_Proxy__abstract__S)
                  0082f8c0    00000020     bench_shm_pe66.oe66 (.text:ti_sdo_ipc_GateMP_RemoteCustom1Proxy_Proxy__delegate__S)
                  0082f8e0    00000020     bench_shm_pe66.oe66 (.text:ti_sdo_ipc_GateMP_RemoteCustom1Proxy_getReservedMask__E)
                  0082f900    00000020     bench_shm_pe66.oe66 (.text:ti_sdo_ipc_GateMP_RemoteCustom1Proxy_sharedMemReq__E)
                  0082f920    00000020     bench_shm_pe66.oe66 (.text:ti_sdo_ipc_GateMP_RemoteCustom2Proxy_Object__delete__S)
                  0082f940    00000020     bench_shm_pe66.oe66 (.text:ti_sdo_ipc_GateMP_RemoteCustom2Proxy_Params__init__S)
                  0082f960    00000020     bench_shm_pe66.oe66 (.text:ti_sdo_ipc_GateMP_RemoteCustom2Proxy_Proxy__abstract__S)
                  0082f980    00000020     bench_shm_pe66.oe66 (.text:ti_sdo_ipc_GateMP_RemoteCustom2Proxy_Proxy__delegate__S)
                  0082f9a0    00000020     bench_shm_pe66.oe66 (.text:ti_sdo_ipc_GateMP_RemoteCustom2Proxy_getReservedMask__E)
                  0082f9c0    00000020     bench_shm_pe66.oe66 (.text:ti_sdo_ipc_GateMP_RemoteCustom2Proxy_sharedMemReq__E)
                  0082f9e0    00000020     bench_shm_pe66.oe66 (.text:ti_sdo_ipc_GateMP_RemoteSystemProxy_Object__delete__S)
                  0082fa00    00000020     bench_shm_pe66.oe66 (.text:ti_sdo_ipc_GateMP_RemoteSystemProxy_Params__init__S)
                  0082fa20    00000020     bench_shm_pe66.oe66 (.text:ti_sdo_ipc_GateMP_RemoteSystemProxy_Proxy__abstract__S)
                  0082fa40    00000020     bench_shm_pe66.oe66 (.text:ti_sdo_ipc_GateMP_RemoteSystemProxy_Proxy__delegate__S)
                  0082fa60    00000020     bench_shm_pe66.oe66 (.text:ti_sdo_ipc_GateMP_RemoteSystemProxy_getReservedMask__E)
                  0082fa80    00000020     bench_shm_pe66.oe66 (.text:ti_sdo_ipc_GateMP_RemoteSystemProxy_sharedMemReq__E)
                  0082faa0    00000020     bench_shm_pe66.oe66 (.text:ti_sdo_ipc_GateMP_attach__E)
                  0082fac0    00000020     bench_shm_pe66.oe66 (.text:ti_sdo_ipc_GateMP_getRegion0ReservedSize__E)
                  0082fae0    00000020     bench_shm_pe66.oe66 (.text:ti_sdo_ipc_GateMP_getSharedAddr__E)
                  0082fb00    00000020     ipc.lib : Ipc.obj (.text:ti_sdo_ipc_GateMP_getSharedAddr__F)
                  0082fb20    00000020     bench_shm_pe66.oe66 (.text:ti_sdo_ipc_GateMP_start__E)
                  0082fb40    00000020     bench_shm_pe66.oe66 (.text:ti_sdo_ipc_MessageQ_Module_startup__E)
                  0082fb60    00000020     bench_shm_pe66.oe66 (.text:ti_sdo_ipc_MessageQ_SetupTransportProxy_attach__E)
                  0082fb80    00000020     bench_shm_pe66.oe66 (.text:ti_sdo_ipc_MessageQ_SetupTransportProxy_detach__E)
                  0082fba0    00000020     bench_shm_pe66.oe66 (.text:ti_sdo_ipc_MessageQ_SetupTransportProxy_isRegistered__E)
                  0082fbc0    00000020     bench_shm_pe66.oe66 (.text:ti_sdo_ipc_MessageQ_SetupTransportProxy_sharedMemReq__E)
                  0082fbe0    00000020     bench_shm_pe66.oe66 (.text:ti_sdo_ipc_MessageQ_unregisterTransport__E)
                  0082fc00    00000020     bench_shm_pe66.oe66 (.text:ti_sdo_ipc_Notify_Module_GateProxy_enter__E)
                  0082fc20    00000020     bench_shm_pe66.oe66 (.text:ti_sdo_ipc_Notify_Module_GateProxy_leave__E)
                  0082fc40    00000020     bench_shm_pe66.oe66 (.text:ti_sdo_ipc_Notify_Module_startup__E)
                  0082fc60    00000020     bench_shm_pe66.oe66 (.text:ti_sdo_ipc_Notify_SetupProxy_attach__E)
                  0082fc80    00000020     bench_shm_pe66.oe66 (.text:ti_sdo_ipc_Notify_SetupProxy_numIntLines__E)
                  0082fca0    00000020     bench_shm_pe66.oe66 (.text:ti_sdo_ipc_Notify_SetupProxy_sharedMemReq__E)
                  0082fcc0    00000020     bench_shm_pe66.oe66 (.text:ti_sdo_ipc_Notify_detach__E)
                  0082fce0    00000020     bench_shm_pe66.oe66 (.text:ti_sdo_ipc_Notify_exec__E)
                  0082fd00    00000020     bench_shm_pe66.oe66 (.text:ti_sdo_ipc_SharedRegion_attach__E)
                  0082fd20    00000020     bench_shm_pe66.oe66 (.text:ti_sdo_ipc_SharedRegion_clearReservedMemory__E)
                  0082fd40    00000020     bench_shm_pe66.oe66 (.text:ti_sdo_ipc_SharedRegion_reserveMemory__E)
                  0082fd60    00000020     bench_shm_pe66.oe66 (.text:ti_sdo_ipc_SharedRegion_start__E)
                  0082fd80    00000020     bench_shm_pe66.oe66 (.text:ti_sdo_ipc_family_c647x_Interrupt_Module_startup__E)
                  0082fda0    00000020     ipc.lib : Ipc.obj (.text:ti_sdo_ipc_family_c647x_Interrupt_intDisable__E)
                  0082fdc0    00000020             : Ipc.obj (.text:ti_sdo_ipc_family_c647x_Interrupt_intEnable__E)
                  0082fde0    00000020             : Ipc.obj (.text:ti_sdo_ipc_family_c647x_NotifyCircSetup_numIntLines__E)
                  0082fe00    00000020     bench_shm_pe66.oe66 (.text:ti_sdo_ipc_gates_GateHWSem_Module_startup__E)
                  0082fe20    00000020     ipc.lib : Ipc.obj (.text:ti_sdo_ipc_gates_GateHWSem_getReservedMask__E)
                  0082fe40    00000020     bench_shm_pe66.oe66 (.text:ti_sdo_ipc_gates_GateHWSem_query__E)
                  0082fe60    00000020     ipc.lib : Ipc.obj (.text:ti_sdo_ipc_gates_GateHWSem_query__F)
                  0082fe80    00000020             : Ipc.obj (.text:ti_sdo_ipc_gates_GateHWSem_sharedMemReq__E)
                  0082fea0    00000020             : Ipc.obj (.text:ti_sdo_ipc_gates_GateMPSupportNull_Instance_init__F)
                  0082fec0    00000020             : Ipc.obj (.text:ti_sdo_ipc_gates_GateMPSupportNull_getReservedMask__E)
                  0082fee0    00000020     bench_shm_pe66.oe66 (.text:ti_sdo_ipc_gates_GateMPSupportNull_query__E)
                  0082ff00    00000020     ipc.lib : Ipc.obj (.text:ti_sdo_ipc_gates_GateMPSupportNull_query__F)
                  0082ff20    00000020             : Ipc.obj (.text:ti_sdo_ipc_gates_GateMPSupportNull_sharedMemReq__E)
                  0082ff40    00000020             : Ipc.obj (.text:ti_sdo_ipc_gates_GatePeterson_getReservedMask__E)
                  0082ff60    00000020     bench_shm_pe66.oe66 (.text:ti_sdo_ipc_gates_GatePeterson_query__E)
                  0082ff80    00000020     ipc.lib : Ipc.obj (.text:ti_sdo_ipc_gates_GatePeterson_query__F)
                  0082ffa0    00000020     bench_shm_pe66.oe66 (.text:ti_sdo_ipc_heaps_HeapMemMP_isBlocking__E)
                  0082ffc0    00000020     ipc.lib : Ipc.obj (.text:ti_sdo_ipc_heaps_HeapMemMP_isBlocking__F)
                  0082ffe0    00000020     bench_shm_pe66.oe66 (.text:ti_sdo_ipc_notifyDrivers_NotifyDriverCirc_InterruptProxy_intClear__E)
                  00830000    00000020     bench_shm_pe66.oe66 (.text:ti_sdo_ipc_notifyDrivers_NotifyDriverCirc_InterruptProxy_intDisable__E)
                  00830020    00000020     bench_shm_pe66.oe66 (.text:ti_sdo_ipc_notifyDrivers_NotifyDriverCirc_InterruptProxy_intEnable__E)
                  00830040    00000020     bench_shm_pe66.oe66 (.text:ti_sdo_ipc_notifyDrivers_NotifyDriverCirc_InterruptProxy_intSend__E)
                  00830060    00000020     bench_shm_pe66.oe66 (.text:ti_sdo_ipc_notifyDrivers_NotifyDriverCirc_InterruptProxy_intUnregister__E)
                  00830080    00000020     ipc.lib : Ipc.obj (.text:ti_sdo_ipc_notifyDrivers_NotifyDriverCirc_setNotifyHandle__E)
                  008300a0    00000020     bench_shm_pe66.oe66 (.text:ti_sdo_ipc_notifyDrivers_NotifyDriverCirc_sharedMemReq__E)
                  008300c0    00000020     ipc.lib : Ipc.obj (.text:ti_sdo_ipc_nsremote_NameServerRemoteNotify_cbFxn__I)
                  008300e0    00000020             : Ipc.obj (.text:ti_sdo_ipc_transports_TransportShmNotifySetup_isRegistered__E)
                  00830100    00000020             : Ipc.obj (.text:ti_sdo_ipc_transports_TransportShmNotifySetup_sharedMemReq__E)
                  00830120    00000020             : Ipc.obj (.text:ti_sdo_ipc_transports_TransportShmNotify_control__E)
                  00830140    00000020             : Ipc.obj (.text:ti_sdo_ipc_transports_TransportShmNotify_getStatus__E)
                  00830160    00000020     bench_shm_pe66.oe66 (.text:ti_sdo_ipc_transports_TransportShmNotify_setErrFxn__E)
                  00830180    00000020     ipc.lib : Ipc.obj (.text:ti_sdo_ipc_transports_TransportShmNotify_setErrFxn__F)
                  008301a0    00000020             : Ipc.obj (.text:ti_sdo_utils_List_Instance_init__F)
                  008301c0    00000020     bench_shm_pe66.oe66 (.text:ti_sdo_utils_MultiProc_getClusterId__E)
                  008301e0    00000020     ipc.lib : Ipc.obj (.text:ti_sdo_utils_MultiProc_getClusterId__F)
                  00830200    00000020     bench_shm_pe66.oe66 (.text:ti_sdo_utils_NameServer_Module__startupDone__S)
                  00830220    00000020     bench_shm_pe66.oe66 (.text:ti_sdo_utils_NameServer_Module_startup__E)
                  00830240    00000020     bench_shm_pe66.oe66 (.text:ti_sdo_utils_NameServer_SetupProxy_attach__E)
                  00830260    00000020     bench_shm_pe66.oe66 (.text:ti_sdo_utils_NameServer_SetupProxy_detach__E)
                  00830280    00000020     bench_shm_pe66.oe66 (.text:ti_sdo_utils_NameServer_SetupProxy_sharedMemReq__E)
                  008302a0    00000020     bench_shm_pe66.oe66 (.text:ti_sysbios_BIOS_RtsGateProxy_enter__E)
                  008302c0    00000020     bench_shm_pe66.oe66 (.text:ti_sysbios_BIOS_RtsGateProxy_leave__E)
                  008302e0    00000020     sysbios.lib : BIOS.obj (.text:ti_sysbios_BIOS_getCpuFreq__E)
                  00830300    00000020                 : BIOS.obj (.text:ti_sysbios_BIOS_getThreadType__E)
                  00830320    00000020                 : BIOS.obj (.text:ti_sysbios_BIOS_setThreadType__E)
                  00830340    00000020     bench_shm_pe66.oe66 (.text:ti_sysbios_family_c62_TaskSupport_Module__startupDone__S)
                  00830360    00000020     sysbios.lib : BIOS.obj (.text:ti_sysbios_family_c62_TaskSupport_checkStack__E)
                  00830380    00000020     bench_shm_pe66.oe66 (.text:ti_sysbios_family_c64p_Exception_Module_startup__E)
                  008303a0    00000020     bench_shm_pe66.oe66 (.text:ti_sysbios_family_c64p_Hwi_Module__startupDone__S)
                  008303c0    00000020     bench_shm_pe66.oe66 (.text:ti_sysbios_family_c64p_Hwi_Module_startup__E)
                  008303e0    00000020     sysbios.lib : BIOS.obj (.text:ti_sysbios_family_c64p_Hwi_clearInterrupt__E)
                  00830400    00000020                 : BIOS.obj (.text:ti_sysbios_family_c64p_Hwi_getHandle__E)
                  00830420    00000020                 : BIOS.obj (.text:ti_sysbios_family_c64p_Hwi_startup__E)
                  00830440    00000020                 : BIOS.obj (.text:ti_sysbios_family_c64p_Hwi_switchFromBootStack__E)
                  00830460    00000020                 : BIOS.obj (.text:ti_sysbios_family_c64p_Hwi_unPluggedInterrupt__I)
                  00830480    00000020     bench_shm_pe66.oe66 (.text:ti_sysbios_family_c64p_TimestampProvider_Module_startup__E)
                  008304a0    00000020     sysbios.lib : BIOS.obj (.text:ti_sysbios_family_c64p_TimestampProvider_Module_startup__F)
                  008304c0    00000020                 : BIOS.obj (.text:ti_sysbios_family_c64p_TimestampProvider_get32__E)
                  008304e0    00000020                 : BIOS.obj (.text:ti_sysbios_family_c64p_TimestampProvider_get64__E)
                  00830500    00000020                 : BIOS.obj (.text:ti_sysbios_family_c64p_tci6488_TimerSupport_enable__E)
                  00830520    00000020     bench_shm_pe66.oe66 (.text:ti_sysbios_family_c66_Cache_Module_startup__E)
                  00830540    00000020     sysbios.lib : BIOS.obj (.text:ti_sysbios_family_c66_Cache_inv__E)
                  00830560    00000020                 : BIOS.obj (.text:ti_sysbios_family_c66_Cache_wbInv__E)
                  00830580    00000020                 : BIOS.obj (.text:ti_sysbios_family_c66_Cache_wb__E)
                  008305a0    00000020                 : BIOS.obj (.text:ti_sysbios_gates_GateAll_Instance_init__F)
                  008305c0    00000020     bench_shm_pe66.oe66 (.text:ti_sysbios_gates_GateAll_query__E)
                  008305e0    00000020     sysbios.lib : BIOS.obj (.text:ti_sysbios_gates_GateAll_query__F)
                  00830600    00000020                 : BIOS.obj (.text:ti_sysbios_gates_GateHwi_Instance_init__F)
                  00830620    00000020                 : BIOS.obj (.text:ti_sysbios_gates_GateHwi_enter__E)
                  00830640    00000020                 : BIOS.obj (.text:ti_sysbios_gates_GateHwi_leave__E)
                  00830660    00000020     bench_shm_pe66.oe66 (.text:ti_sysbios_gates_GateHwi_query__E)
                  00830680    00000020     sysbios.lib : BIOS.obj (.text:ti_sysbios_gates_GateHwi_query__F)
                  008306a0    00000020     bench_shm_pe66.oe66 (.text:ti_sysbios_gates_GateMutexPri_query__E)
                  008306c0    00000020     sysbios.lib : BIOS.obj (.text:ti_sysbios_gates_GateMutexPri_query__F)
                  008306e0    00000020     bench_shm_pe66.oe66 (.text:ti_sysbios_gates_GateMutex_query__E)
                  00830700    00000020     sysbios.lib : BIOS.obj (.text:ti_sysbios_gates_GateMutex_query__F)
                  00830720    00000020                 : BIOS.obj (.text:ti_sysbios_gates_GateSwi_Instance_init__F)
                  00830740    00000020     bench_shm_pe66.oe66 (.text:ti_sysbios_gates_GateSwi_query__E)
                  00830760    00000020     sysbios.lib : BIOS.obj (.text:ti_sysbios_gates_GateSwi_query__F)
                  00830780    00000020     bench_shm_pe66.oe66 (.text:ti_sysbios_hal_Cache_CacheProxy_wait__E)
                  008307a0    00000020     bench_shm_pe66.oe66 (.text:ti_sysbios_hal_Hwi_HwiProxy_Module__startupDone__S)
                  008307c0    00000020     bench_shm_pe66.oe66 (.text:ti_sysbios_hal_Hwi_HwiProxy_clearInterrupt__E)
                  008307e0    00000020     bench_shm_pe66.oe66 (.text:ti_sysbios_hal_Hwi_HwiProxy_disableInterrupt__E)
                  00830800    00000020     bench_shm_pe66.oe66 (.text:ti_sysbios_hal_Hwi_HwiProxy_enableInterrupt__E)
                  00830820    00000020     bench_shm_pe66.oe66 (.text:ti_sysbios_hal_Hwi_HwiProxy_startup__E)
                  00830840    00000020     bench_shm_pe66.oe66 (.text:ti_sysbios_hal_Hwi_HwiProxy_switchFromBootStack__E)
                  00830860    00000020     bench_shm_pe66.oe66 (.text:ti_sysbios_hal_Hwi_Module_startup__E)
                  00830880    00000020     sysbios.lib : BIOS.obj (.text:ti_sysbios_hal_Hwi_Module_startup__F)
                  008308a0    00000020     bench_shm_pe66.oe66 (.text:ti_sysbios_hal_Timer_Module__startupDone__S)
                  008308c0    00000020     bench_shm_pe66.oe66 (.text:ti_sysbios_hal_Timer_Module_startup__E)
                  008308e0    00000020     sysbios.lib : BIOS.obj (.text:ti_sysbios_hal_Timer_Module_startup__F)
                  00830900    00000020     bench_shm_pe66.oe66 (.text:ti_sysbios_hal_Timer_TimerProxy_Module__startupDone__S)
                  00830920    00000020     bench_shm_pe66.oe66 (.text:ti_sysbios_hal_Timer_TimerProxy_getExpiredCounts__E)
                  00830940    00000020     bench_shm_pe66.oe66 (.text:ti_sysbios_hal_Timer_TimerProxy_getPeriod__E)
                  00830960    00000020     bench_shm_pe66.oe66 (.text:ti_sysbios_hal_Timer_TimerProxy_setNextTick__E)
                  00830980    00000020     bench_shm_pe66.oe66 (.text:ti_sysbios_hal_Timer_TimerProxy_startup__E)
                  008309a0    00000020     bench_shm_pe66.oe66 (.text:ti_sysbios_heaps_HeapMem_Module_GateProxy_enter__E)
                  008309c0    00000020     bench_shm_pe66.oe66 (.text:ti_sysbios_heaps_HeapMem_Module_GateProxy_leave__E)
                  008309e0    00000020     bench_shm_pe66.oe66 (.text:ti_sysbios_heaps_HeapMem_Module_GateProxy_query__E)
                  00830a00    00000020     sysbios.lib : BIOS.obj (.text:ti_sysbios_heaps_HeapMem_isBlocking__E)
                  00830a20    00000020     bench_shm_pe66.oe66 (.text:ti_sysbios_knl_Clock_Module_State_clockQ)
                  00830a40    00000020     bench_shm_pe66.oe66 (.text:ti_sysbios_knl_Clock_Module_startup__E)
                  00830a60    00000020     sysbios.lib : BIOS.obj (.text:ti_sysbios_knl_Queue_Instance_init__F)
                  00830a80    00000020                 : BIOS.obj (.text:ti_sysbios_knl_Queue_empty__E)
                  00830aa0    00000020     bench_shm_pe66.oe66 (.text:ti_sysbios_knl_Swi_Module_startup__E)
                  00830ac0    00000020     sysbios.lib : BIOS.obj (.text:ti_sysbios_knl_Swi_disable__E)
                  00830ae0    00000020     bench_shm_pe66.oe66 (.text:ti_sysbios_knl_Task_Module_startup__E)
                  00830b00    00000020     bench_shm_pe66.oe66 (.text:ti_sysbios_knl_Task_SupportProxy_Module__startupDone__S)
                  00830b20    00000020     bench_shm_pe66.oe66 (.text:ti_sysbios_knl_Task_SupportProxy_checkStack__E)
                  00830b40    00000020     bench_shm_pe66.oe66 (.text:ti_sysbios_knl_Task_SupportProxy_start__E)
                  00830b60    00000020     bench_shm_pe66.oe66 (.text:ti_sysbios_knl_Task_SupportProxy_swap__E)
                  00830b80    00000020     sysbios.lib : BIOS.obj (.text:ti_sysbios_knl_Task_disable__E)
                  00830ba0    00000020                 : BIOS.obj (.text:ti_sysbios_knl_Task_getPri__E)
                  00830bc0    00000020                 : BIOS.obj (.text:ti_sysbios_knl_Task_self__E)
                  00830be0    00000020     bench_shm_pe66.oe66 (.text:ti_sysbios_syncs_SyncSem_query__E)
                  00830c00    00000020     sysbios.lib : BIOS.obj (.text:ti_sysbios_syncs_SyncSem_query__F)
                  00830c20    00000020     bench_shm_pe66.oe66 (.text:ti_sysbios_syncs_SyncSem_signal__E)
                  00830c40    00000020     sysbios.lib : BIOS.obj (.text:ti_sysbios_syncs_SyncSem_signal__F)
                  00830c60    00000020     bench_shm_pe66.oe66 (.text:ti_sysbios_syncs_SyncSem_wait__E)
                  00830c80    00000020     bench_shm_pe66.oe66 (.text:ti_sysbios_timers_timer64_Timer_Module__startupDone__S)
                  00830ca0    00000020     bench_shm_pe66.oe66 (.text:ti_sysbios_timers_timer64_Timer_Module_startup__E)
                  00830cc0    00000020     bench_shm_pe66.oe66 (.text:ti_sysbios_timers_timer64_Timer_TimerSupportProxy_enable__E)
                  00830ce0    00000020     sysbios.lib : BIOS.obj (.text:ti_sysbios_timers_timer64_Timer_setNextTick__E)
                  00830d00    00000020     bench_shm_pe66.oe66 (.text:ti_sysbios_xdcruntime_GateThreadSupport_enter__E)
                  00830d20    00000020     bench_shm_pe66.oe66 (.text:ti_sysbios_xdcruntime_GateThreadSupport_leave__E)
                  00830d40    00000020     bench_shm_pe66.oe66 (.text:ti_sysbios_xdcruntime_GateThreadSupport_query__E)
                  00830d60    00000020     bench_shm_pe66.oe66 (.text:xdc_argToFloat)
                  00830d80    00000020     bench_shm_pe66.oe66 (.text:xdc_runtime_Error_check__E)
                  00830da0    00000020     bench_shm_pe66.oe66 (.text:xdc_runtime_Error_init__E)
                  00830dc0    00000020     bench_shm_pe66.oe66 (.text:xdc_runtime_Error_print__E)
                  00830de0    00000020     bench_shm_pe66.oe66 (.text:xdc_runtime_GateNull_enter__E)
                  00830e00    00000020     ti.targets.rts6000.ae66 : GateNull.oe66 (.text:xdc_runtime_GateNull_enter__F)
                  00830e20    00000020     bench_shm_pe66.oe66 (.text:xdc_runtime_GateNull_leave__E)
                  00830e40    00000020     ti.targets.rts6000.ae66 : GateNull.oe66 (.text:xdc_runtime_GateNull_leave__F)
                  00830e60    00000020     bench_shm_pe66.oe66 (.text:xdc_runtime_GateNull_query__E)
                  00830e80    00000020     ti.targets.rts6000.ae66 : GateNull.oe66 (.text:xdc_runtime_GateNull_query__F)
                  00830ea0    00000020     bench_shm_pe66.oe66 (.text:xdc_runtime_Gate_enterSystem__E)
                  00830ec0    00000020     ti.targets.rts6000.ae66 : Gate.oe66 (.text:xdc_runtime_Gate_enterSystem__F)
                  00830ee0    00000020     bench_shm_pe66.oe66 (.text:xdc_runtime_Gate_leaveSystem__E)
                  00830f00    00000020     bench_shm_pe66.oe66 (.text:xdc_runtime_Memory_HeapProxy_alloc__E)
                  00830f20    00000020     bench_shm_pe66.oe66 (.text:xdc_runtime_Memory_HeapProxy_free__E)
                  00830f40    00000020     bench_shm_pe66.oe66 (.text:xdc_runtime_Memory_alloc__E)
                  00830f60    00000020     bench_shm_pe66.oe66 (.text:xdc_runtime_Memory_calloc__E)
                  00830f80    00000020     bench_shm_pe66.oe66 (.text:xdc_runtime_Memory_free__E)
                  00830fa0    00000020     bench_shm_pe66.oe66 (.text:xdc_runtime_Memory_getMaxDefaultTypeAlign__E)
                  00830fc0    00000020     ti.targets.rts6000.ae66 : Memory.oe66 (.text:xdc_runtime_Memory_getMaxDefaultTypeAlign__F)
                  00830fe0    00000020     bench_shm_pe66.oe66 (.text:xdc_runtime_Registry_findById__E)
                  00831000    00000020     bench_shm_pe66.oe66 (.text:xdc_runtime_Startup_Module__startupDone__S)
                  00831020    00000020     bench_shm_pe66.oe66 (.text:xdc_runtime_Startup_exec__E)
                  00831040    00000020     bench_shm_pe66.oe66 (.text:xdc_runtime_Startup_reset__I)
                  00831060    00000020     bench_shm_pe66.oe66 (.text:xdc_runtime_Startup_rtsDone__E)
                  00831080    00000020     ti.targets.rts6000.ae66 : Startup.oe66 (.text:xdc_runtime_Startup_rtsDone__F)
                  008310a0    00000020     bench_shm_pe66.oe66 (.text:xdc_runtime_SysStd_abort__E)
                  008310c0    00000020     bench_shm_pe66.oe66 (.text:xdc_runtime_SysStd_exit__E)
                  008310e0    00000020     ti.targets.rts6000.ae66 : SysStd.oe66 (.text:xdc_runtime_SysStd_exit__F)
                  00831100    00000020     bench_shm_pe66.oe66 (.text:xdc_runtime_SysStd_putch__E)
                  00831120    00000020     ti.targets.rts6000.ae66 : SysStd.oe66 (.text:xdc_runtime_SysStd_putch__F)
                  00831140    00000020     bench_shm_pe66.oe66 (.text:xdc_runtime_SysStd_ready__E)
                  00831160    00000020     ti.targets.rts6000.ae66 : SysStd.oe66 (.text:xdc_runtime_SysStd_ready__F)
                  00831180    00000020     bench_shm_pe66.oe66 (.text:xdc_runtime_System_Module_GateProxy_enter__E)
                  008311a0    00000020     bench_shm_pe66.oe66 (.text:xdc_runtime_System_Module_GateProxy_leave__E)
                  008311c0    00000020     bench_shm_pe66.oe66 (.text:xdc_runtime_System_Module_startup__E)
                  008311e0    00000020     ti.targets.rts6000.ae66 : System.oe66 (.text:xdc_runtime_System_Module_startup__F)
                  00831200    00000020     bench_shm_pe66.oe66 (.text:xdc_runtime_System_SupportProxy_abort__E)
                  00831220    00000020     bench_shm_pe66.oe66 (.text:xdc_runtime_System_SupportProxy_exit__E)
                  00831240    00000020     bench_shm_pe66.oe66 (.text:xdc_runtime_System_SupportProxy_putch__E)
                  00831260    00000020     bench_shm_pe66.oe66 (.text:xdc_runtime_System_SupportProxy_ready__E)
                  00831280    00000020     bench_shm_pe66.oe66 (.text:xdc_runtime_System_abort__E)
                  008312a0    00000020     bench_shm_pe66.oe66 (.text:xdc_runtime_System_atexit__E)
                  008312c0    00000020     bench_shm_pe66.oe66 (.text:xdc_runtime_System_exit__E)
                  008312e0    00000020     ti.targets.rts6000.ae66 : System.oe66 (.text:xdc_runtime_System_exit__F)
                  00831300    00000020                             : System.oe66 (.text:xdc_runtime_System_lastFxn__I)
                  00831320    00000020     bench_shm_pe66.oe66 (.text:xdc_runtime_System_vsprintf__E)
                  00831340    00000020     ti.targets.rts6000.ae66 : System.oe66 (.text:xdc_runtime_System_vsprintf__F)
                  00831360    00000020     bench_shm_pe66.oe66 (.text:xdc_runtime_Text_cordText__E)
                  00831380    00000020     bench_shm_pe66.oe66 (.text:xdc_runtime_Text_putSite__E)
                  008313a0    00000020     bench_shm_pe66.oe66 (.text:xdc_runtime_Text_ropeText__E)
                  008313c0    00000020     bench_shm_pe66.oe66 (.text:xdc_runtime_Timestamp_SupportProxy_get32__E)
                  008313e0    00000020     bench_shm_pe66.oe66 (.text:xdc_runtime_Timestamp_SupportProxy_get64__E)
                  00831400    00000020     bench_shm_pe66.oe66 (.text:xdc_runtime_Timestamp_SupportProxy_getFreq__E)
                  00831420    00000020     bench_shm_pe66.oe66 (.text:xdc_runtime_Timestamp_get32__E)
                  00831440    00000020     bench_shm_pe66.oe66 (.text:xdc_runtime_Timestamp_get64__E)
                  00831460    00000020     bench_shm_pe66.oe66 (.text:xdc_runtime_Timestamp_getFreq__E)
                  00831480    00000020     bench_shm_pe66.oe66 (.text:xdc_runtime_knl_GateThread_Module__startupDone__S)
                  008314a0    00000020     bench_shm_pe66.oe66 (.text:xdc_runtime_knl_GateThread_Proxy_Object__delete__S)
                  008314c0    00000020     bench_shm_pe66.oe66 (.text:xdc_runtime_knl_GateThread_Proxy_enter__E)
                  008314e0    00000020     bench_shm_pe66.oe66 (.text:xdc_runtime_knl_GateThread_Proxy_leave__E)
                  00831500    00000020     bench_shm_pe66.oe66 (.text:xdc_runtime_knl_GateThread_Proxy_query__E)
                  00831520    00000020     bench_shm_pe66.oe66 (.text:xdc_runtime_knl_GateThread_enter__E)
                  00831540    00000020     ti.targets.rts6000.ae66 : GateThread.oe66 (.text:xdc_runtime_knl_GateThread_enter__F)
                  00831560    00000020     bench_shm_pe66.oe66 (.text:xdc_runtime_knl_GateThread_leave__E)
                  00831580    00000020     ti.targets.rts6000.ae66 : GateThread.oe66 (.text:xdc_runtime_knl_GateThread_leave__F)
                  008315a0    00000020     bench_shm_pe66.oe66 (.text:xdc_runtime_knl_GateThread_query__E)

.msgQ_ptrs 
*          0    008315c0    0000fa00     UNINITIALIZED
                  008315c0    0000fa00     bench_shm.obj (.msgQ_ptrs)

.far       0    00840fc0    00009608     UNINITIALIZED
                  00840fc0    00008014     bench_shm_pe66.oe66 (.far)
                  00848fd4    00000004     --HOLE--
                  00848fd8    00001000     bench_shm_pe66.oe66 (.far:taskStackSection)
                  00849fd8    00000370     bench_shm.obj (.far)
                  0084a348    00000140     rts6600_elf.lib : defs.obj (.far)
                  0084a488    000000f0     bench_osal.obj (.far)
                  0084a578    00000044     ti.platform.evm6657l.ae66 : evmc665x_i2c_eeprom.obj (.far)
                  0084a5bc    00000004     --HOLE--
                  0084a5c0    00000008     rts6600_elf.lib : trgdrv.obj (.far)

.fardata.1 
*          0    0084a5c8    00000008     
                  0084a5c8    00000008     rts6600_elf.lib : _lock.obj (.fardata)

.const     0    0084a5d0    0000497e     
                  0084a5d0    000025c6     bench_shm_pe66.oe66 (.const:xdc_runtime_Text_charTab__A)
                  0084cb96    00000002     --HOLE-- [fill = 0]
                  0084cb98    00000650     bench_shm.obj (.const:.string)
                  0084d1e8    0000042c     sysbios.lib : BIOS.obj (.const:.string)
                  0084d614    00000004     ti.targets.rts6000.ae66 : Assert.oe66 (.const:.string)
                  0084d618    00000400     bench_shm_pe66.oe66 (.const:ti_sysbios_family_c66_Cache_marvalues__C)
                  0084da18    00000174     bench_shm_pe66.oe66 (.const:xdc_runtime_Text_nodeTab__A)
                  0084db8c    00000004     bench_shm_pe66.oe66 (.const:ti_sdo_ipc_GateMP_A_invalidClose__C)
                  0084db90    00000101     rts6600_elf.lib : ctype.obj (.const:.string:_ctypes_)
                  0084dc91    00000003     --HOLE-- [fill = 0]
                  0084dc94    000000a8     bench_shm_pe66.oe66 (.const:.string)
                  0084dd3c    000000a4     bench_common.obj (.const:.string)
                  0084dde0    00000058     ti.platform.evm6657l.ae66 : platform.obj (.const:.string)
                  0084de38    00000058     ti.targets.rts6000.ae66 : Error.oe66 (.const:.string)
                  0084de90    00000040                             : Text.oe66 (.const:.string)
                  0084ded0    00000040     bench_shm_pe66.oe66 (.const:xdc_runtime_Startup_sfxnTab__A)
                  0084df10    00000038     bench_shm_pe66.oe66 (.const:ti_sdo_ipc_notifyDrivers_NotifyDriverCirc_Module__FXNS__C)
                  0084df48    00000034     bench_shm_pe66.oe66 (.const:ti_sdo_ipc_GateMP_Object__PARAMS__C)
                  0084df7c    00000034     bench_shm_pe66.oe66 (.const:ti_sdo_ipc_notifyDrivers_NotifyDriverCirc_Object__PARAMS__C)
                  0084dfb0    00000030     bench_shm_pe66.oe66 (.const:ti_sdo_ipc_heaps_HeapMemMP_Object__PARAMS__C)
                  0084dfe0    00000030     bench_shm_pe66.oe66 (.const:ti_sysbios_family_c64p_Hwi_Object__PARAMS__C)
                  0084e010    0000002c     ti.targets.rts6000.ae66 : Startup.oe66 (.const:.string)
                  0084e03c    0000002c     bench_shm_pe66.oe66 (.const:ti_sdo_ipc_gates_GateHWSem_Module__FXNS__C)
                  0084e068    0000002c     bench_shm_pe66.oe66 (.const:ti_sdo_ipc_gates_GateMPSupportNull_Module__FXNS__C)
                  0084e094    0000002c     bench_shm_pe66.oe66 (.const:ti_sdo_ipc_gates_GatePeterson_Module__FXNS__C)
                  0084e0c0    00000028     ti.platform.evm6657l.ae66 : evmc665x_nand.obj (.const:.string:$P$T0$1)
                  0084e0e8    00000028                               : evmc665x_nand.obj (.const:.string:$P$T1$2)
                  0084e110    00000028     bench_shm_pe66.oe66 (.const:ti_sdo_ipc_heaps_HeapMemMP_Module__FXNS__C)
                  0084e138    00000028     bench_shm_pe66.oe66 (.const:ti_sdo_ipc_nsremote_NameServerRemoteNotify_Module__FXNS__C)
                  0084e160    00000028     bench_shm_pe66.oe66 (.const:ti_sdo_ipc_transports_TransportShmNotify_Module__FXNS__C)
                  0084e188    00000028     bench_shm_pe66.oe66 (.const:ti_sysbios_heaps_HeapMem_Module__FXNS__C)
                  0084e1b0    00000028     bench_shm_pe66.oe66 (.const:ti_sysbios_knl_Swi_Object__PARAMS__C)
                  0084e1d8    00000024     bench_shm_pe66.oe66 (.const:ti_sdo_ipc_gates_GateHWSem_Object__PARAMS__C)
                  0084e1fc    00000024     bench_shm_pe66.oe66 (.const:ti_sdo_ipc_gates_GateMPSupportNull_Object__PARAMS__C)
                  0084e220    00000024     bench_shm_pe66.oe66 (.const:ti_sdo_ipc_gates_GatePeterson_Object__PARAMS__C)
                  0084e244    00000024     bench_shm_pe66.oe66 (.const:ti_sysbios_gates_GateAll_Module__FXNS__C)
                  0084e268    00000024     bench_shm_pe66.oe66 (.const:ti_sysbios_gates_GateHwi_Module__FXNS__C)
                  0084e28c    00000024     bench_shm_pe66.oe66 (.const:ti_sysbios_gates_GateMutexPri_Module__FXNS__C)
                  0084e2b0    00000024     bench_shm_pe66.oe66 (.const:ti_sysbios_gates_GateMutex_Module__FXNS__C)
                  0084e2d4    00000024     bench_shm_pe66.oe66 (.const:ti_sysbios_gates_GateSwi_Module__FXNS__C)
                  0084e2f8    00000024     bench_shm_pe66.oe66 (.const:ti_sysbios_knl_Clock_Object__PARAMS__C)
                  0084e31c    00000024     bench_shm_pe66.oe66 (.const:ti_sysbios_knl_Semaphore_Object__PARAMS__C)
                  0084e340    00000024     bench_shm_pe66.oe66 (.const:ti_sysbios_syncs_SyncSem_Module__FXNS__C)
                  0084e364    00000024     bench_shm_pe66.oe66 (.const:xdc_runtime_GateNull_Module__FXNS__C)
                  0084e388    00000024     bench_shm_pe66.oe66 (.const:xdc_runtime_knl_GateThread_Module__FXNS__C)
                  0084e3ac    00000023     rts6600_elf.lib : _printfi.obj (.const:.string)
                  0084e3cf    00000001     --HOLE-- [fill = 0]
                  0084e3d0    00000020     ti.targets.rts6000.ae66 : Core-mem.oe66 (.const:.string)
                  0084e3f0    00000020     bench_shm_pe66.oe66 (.const:ti_sdo_ipc_GateMP_Object__DESC__C)
                  0084e410    00000020     bench_shm_pe66.oe66 (.const:ti_sdo_ipc_MessageQ_Object__DESC__C)
                  0084e430    00000020     bench_shm_pe66.oe66 (.const:ti_sdo_ipc_Notify_Object__DESC__C)
                  0084e450    00000020     bench_shm_pe66.oe66 (.const:ti_sdo_ipc_gates_GateHWSem_Object__DESC__C)
                  0084e470    00000020     bench_shm_pe66.oe66 (.const:ti_sdo_ipc_gates_GateMPSupportNull_Object__DESC__C)
                  0084e490    00000020     bench_shm_pe66.oe66 (.const:ti_sdo_ipc_gates_GatePeterson_Object__DESC__C)
                  0084e4b0    00000020     bench_shm_pe66.oe66 (.const:ti_sdo_ipc_heaps_HeapMemMP_Object__DESC__C)
                  0084e4d0    00000020     bench_shm_pe66.oe66 (.const:ti_sdo_ipc_notifyDrivers_NotifyDriverCirc_Object__DESC__C)
                  0084e4f0    00000020     bench_shm_pe66.oe66 (.const:ti_sdo_ipc_nsremote_NameServerRemoteNotify_Object__DESC__C)
                  0084e510    00000020     bench_shm_pe66.oe66 (.const:ti_sdo_ipc_nsremote_NameServerRemoteNotify_Object__PARAMS__C)
                  0084e530    00000020     bench_shm_pe66.oe66 (.const:ti_sdo_ipc_transports_TransportShmNotify_Object__DESC__C)
                  0084e550    00000020     bench_shm_pe66.oe66 (.const:ti_sdo_utils_List_Object__DESC__C)
                  0084e570    00000020     bench_shm_pe66.oe66 (.const:ti_sysbios_family_c64p_Hwi_Object__DESC__C)
                  0084e590    00000020     bench_shm_pe66.oe66 (.const:ti_sysbios_gates_GateAll_Object__DESC__C)
                  0084e5b0    00000020     bench_shm_pe66.oe66 (.const:ti_sysbios_gates_GateHwi_Object__DESC__C)
                  0084e5d0    00000020     bench_shm_pe66.oe66 (.const:ti_sysbios_gates_GateMutexPri_Object__DESC__C)
                  0084e5f0    00000020     bench_shm_pe66.oe66 (.const:ti_sysbios_gates_GateMutex_Object__DESC__C)
                  0084e610    00000020     bench_shm_pe66.oe66 (.const:ti_sysbios_gates_GateSwi_Object__DESC__C)
                  0084e630    00000020     bench_shm_pe66.oe66 (.const:ti_sysbios_heaps_HeapMem_Object__DESC__C)
                  0084e650    00000020     bench_shm_pe66.oe66 (.const:ti_sysbios_heaps_HeapMem_Object__PARAMS__C)
                  0084e670    00000020     bench_shm_pe66.oe66 (.const:ti_sysbios_knl_Clock_Object__DESC__C)
                  0084e690    00000020     bench_shm_pe66.oe66 (.const:ti_sysbios_knl_Queue_Object__DESC__C)
                  0084e6b0    00000020     bench_shm_pe66.oe66 (.const:ti_sysbios_knl_Semaphore_Object__DESC__C)
                  0084e6d0    00000020     bench_shm_pe66.oe66 (.const:ti_sysbios_knl_Swi_Object__DESC__C)
                  0084e6f0    00000020     bench_shm_pe66.oe66 (.const:ti_sysbios_syncs_SyncSem_Object__DESC__C)
                  0084e710    00000020     bench_shm_pe66.oe66 (.const:ti_sysbios_xdcruntime_GateThreadSupport_Object__DESC__C)
                  0084e730    00000020     bench_shm_pe66.oe66 (.const:xdc_runtime_GateNull_Object__DESC__C)
                  0084e750    00000020     bench_shm_pe66.oe66 (.const:xdc_runtime_Startup_sfxnRts__A)
                  0084e770    00000020     bench_shm_pe66.oe66 (.const:xdc_runtime_knl_GateThread_Object__DESC__C)
                  0084e790    0000001c     bench_shm_pe66.oe66 (.const:ti_sdo_ipc_MessageQ_Object__PARAMS__C)
                  0084e7ac    0000001c     bench_shm_pe66.oe66 (.const:ti_sdo_ipc_transports_TransportShmNotify_Object__PARAMS__C)
                  0084e7c8    0000001c     bench_shm_pe66.oe66 (.const:ti_sysbios_syncs_SyncSem_Object__PARAMS__C)
                  0084e7e4    00000018     bench_shm_pe66.oe66 (.const:ti_sdo_ipc_Notify_Object__PARAMS__C)
                  0084e7fc    00000018     bench_shm_pe66.oe66 (.const:ti_sdo_utils_List_Object__PARAMS__C)
                  0084e814    00000018     bench_shm_pe66.oe66 (.const:ti_sysbios_gates_GateAll_Object__PARAMS__C)
                  0084e82c    00000018     bench_shm_pe66.oe66 (.const:ti_sysbios_gates_GateHwi_Object__PARAMS__C)
                  0084e844    00000018     bench_shm_pe66.oe66 (.const:ti_sysbios_gates_GateMutexPri_Object__PARAMS__C)
                  0084e85c    00000018     bench_shm_pe66.oe66 (.const:ti_sysbios_gates_GateMutex_Object__PARAMS__C)
                  0084e874    00000018     bench_shm_pe66.oe66 (.const:ti_sysbios_gates_GateSwi_Object__PARAMS__C)
                  0084e88c    00000018     bench_shm_pe66.oe66 (.const:ti_sysbios_knl_Queue_Object__PARAMS__C)
                  0084e8a4    00000004     bench_shm_pe66.oe66 (.const:ti_sdo_ipc_GateMP_A_invalidDelete__C)
                  0084e8a8    00000018     bench_shm_pe66.oe66 (.const:ti_sysbios_knl_Task_hooks__A)
                  0084e8c0    00000018     bench_shm_pe66.oe66 (.const:ti_sysbios_xdcruntime_GateThreadSupport_Object__PARAMS__C)
                  0084e8d8    00000018     bench_shm_pe66.oe66 (.const:xdc_runtime_GateNull_Object__PARAMS__C)
                  0084e8f0    00000018     bench_shm_pe66.oe66 (.const:xdc_runtime_knl_GateThread_Object__PARAMS__C)
                  0084e908    00000008     ti.targets.rts6000.ae66 : System.oe66 (.const:.string)
                  0084e910    00000011                             : System.oe66 (.const:digtohex)
                  0084e921    00000003     --HOLE-- [fill = 0]
                  0084e924    00000004     bench_shm_pe66.oe66 (.const:ti_sdo_ipc_GateMP_E_gateUnavailable__C)
                  0084e928    00000010     bench_shm_pe66.oe66 (.const:xdc_runtime_Startup_firstFxns__A)
                  0084e938    0000000c     bench_shm_pe66.oe66 (.const:ti_sysbios_family_c66_Cache_initSize__C)
                  0084e944    00000004     bench_shm_pe66.oe66 (.const:ti_sdo_ipc_GateMP_E_localGate__C)
                  0084e948    00000008     bench_shm_pe66.oe66 (.const:ti_sdo_utils_MultiProc_nameList__A)
                  0084e950    00000008     bench_shm_pe66.oe66 (.const:ti_sysbios_knl_Idle_funcList__C)
                  0084e958    00000008     bench_shm_pe66.oe66 (.const:ti_sysbios_knl_Task_hooks__C)
                  0084e960    00000008     bench_shm_pe66.oe66 (.const:xdc_runtime_Startup_firstFxns__C)
                  0084e968    00000008     bench_shm_pe66.oe66 (.const:xdc_runtime_Startup_lastFxns__C)
                  0084e970    00000004     bench_shm.obj (.const:$P$T0$1)
                  0084e974    00000004     bench_shm_pe66.oe66 (.const:ti_sdo_ipc_GateMP_LM_create__C)
                  0084e978    00000004     bench_shm.obj (.const:$P$T1$2)
                  0084e97c    00000004     bench_shm_pe66.oe66 (.const:ti_sdo_ipc_GateMP_LM_delete__C)
                  0084e980    00000004     bench_shm_pe66.oe66 (.const:ti_sdo_ipc_GateMP_LM_enter__C)
                  0084e984    00000004     bench_shm_pe66.oe66 (.const:ti_sdo_ipc_GateMP_LM_leave__C)
                  0084e988    00000004     bench_shm_pe66.oe66 (.const:ti_sdo_ipc_GateMP_LM_open__C)
                  0084e98c    00000004     bench_shm_pe66.oe66 (.const:ti_sdo_ipc_GateMP_Module__diagsEnabled__C)
                  0084e990    00000004     bench_shm_pe66.oe66 (.const:ti_sdo_ipc_GateMP_Module__diagsIncluded__C)
                  0084e994    00000004     bench_shm_pe66.oe66 (.const:ti_sdo_ipc_GateMP_Module__diagsMask__C)
                  0084e998    00000004     bench_shm_pe66.oe66 (.const:ti_sdo_ipc_GateMP_Module__loggerFxn2__C)
                  0084e99c    00000004     bench_shm_pe66.oe66 (.const:ti_sdo_ipc_GateMP_Module__loggerFxn4__C)
                  0084e9a0    00000004     bench_shm_pe66.oe66 (.const:ti_sdo_ipc_GateMP_Module__loggerObj__C)
                  0084e9a4    00000004     bench_shm_pe66.oe66 (.const:ti_sdo_ipc_Ipc_A_addrNotCacheAligned__C)
                  0084e9a8    00000004     bench_shm_pe66.oe66 (.const:ti_sdo_ipc_Ipc_A_addrNotInSharedRegion__C)
                  0084e9ac    00000004     bench_shm_pe66.oe66 (.const:ti_sdo_ipc_Ipc_A_internal__C)
                  0084e9b0    00000004     bench_shm_pe66.oe66 (.const:ti_sdo_ipc_Ipc_A_invArgument__C)
                  0084e9b4    00000004     bench_shm_pe66.oe66 (.const:ti_sdo_ipc_Ipc_A_invParam__C)
                  0084e9b8    00000004     bench_shm_pe66.oe66 (.const:ti_sdo_ipc_Ipc_A_nullArgument__C)
                  0084e9bc    00000004     bench_shm_pe66.oe66 (.const:ti_sdo_ipc_Ipc_E_internal__C)
                  0084e9c0    00000004     bench_shm_pe66.oe66 (.const:ti_sdo_ipc_Ipc_E_nameFailed__C)
                  0084e9c4    00000004     bench_shm_pe66.oe66 (.const:ti_sdo_ipc_Ipc_E_versionMismatch__C)
                  0084e9c8    00000004     bench_shm_pe66.oe66 (.const:ti_sdo_ipc_Ipc_Module__diagsEnabled__C)
                  0084e9cc    00000004     bench_shm_pe66.oe66 (.const:ti_sdo_ipc_Ipc_Module__diagsIncluded__C)
                  0084e9d0    00000004     bench_shm_pe66.oe66 (.const:ti_sdo_ipc_Ipc_Module__diagsMask__C)
                  0084e9d4    00000004     bench_shm_pe66.oe66 (.const:ti_sdo_ipc_Ipc_numUserFxns__C)
                  0084e9d8    00000004     bench_shm_pe66.oe66 (.const:ti_sdo_ipc_Ipc_procSync__C)
                  0084e9dc    00000004     bench_shm_pe66.oe66 (.const:ti_sdo_ipc_Ipc_userFxns__C)
                  0084e9e0    00000004     bench_shm_pe66.oe66 (.const:ti_sdo_ipc_MessageQ_A_cannotFreeStaticMsg__C)
                  0084e9e4    00000004     bench_shm_pe66.oe66 (.const:ti_sdo_ipc_MessageQ_A_heapIdInvalid__C)
                  0084e9e8    00000004     bench_shm_pe66.oe66 (.const:ti_sdo_ipc_MessageQ_A_invalidMsg__C)
                  0084e9ec    00000004     bench_shm_pe66.oe66 (.const:ti_sdo_ipc_MessageQ_A_invalidObj__C)
                  0084e9f0    00000004     bench_shm_pe66.oe66 (.const:ti_sdo_ipc_MessageQ_A_invalidParam__C)
                  0084e9f4    00000004     bench_shm_pe66.oe66 (.const:ti_sdo_ipc_MessageQ_A_invalidQueueId__C)
                  0084e9f8    00000004     bench_shm_pe66.oe66 (.const:ti_sdo_ipc_MessageQ_A_procIdInvalid__C)
                  0084e9fc    00000004     bench_shm_pe66.oe66 (.const:ti_sdo_ipc_MessageQ_A_unregisteredTransport__C)
                  0084ea00    00000004     bench_shm_pe66.oe66 (.const:ti_sdo_ipc_MessageQ_E_maxReached__C)
                  0084ea04    00000004     bench_shm_pe66.oe66 (.const:ti_sdo_ipc_MessageQ_E_nameFailed__C)
                  0084ea08    00000004     bench_shm_pe66.oe66 (.const:ti_sdo_ipc_MessageQ_Instance_State_highList__O)
                  0084ea0c    00000004     bench_shm_pe66.oe66 (.const:ti_sdo_ipc_MessageQ_Instance_State_normalList__O)
                  0084ea10    00000004     bench_shm_pe66.oe66 (.const:ti_sdo_ipc_MessageQ_LM_alloc__C)
                  0084ea14    00000004     bench_shm_pe66.oe66 (.const:ti_sdo_ipc_MessageQ_LM_free__C)
                  0084ea18    00000004     bench_shm_pe66.oe66 (.const:ti_sdo_ipc_MessageQ_LM_get__C)
                  0084ea1c    00000004     bench_shm_pe66.oe66 (.const:ti_sdo_ipc_MessageQ_LM_putLocal__C)
                  0084ea20    00000004     bench_shm_pe66.oe66 (.const:ti_sdo_ipc_MessageQ_Module__diagsEnabled__C)
                  0084ea24    00000004     bench_shm_pe66.oe66 (.const:ti_sdo_ipc_MessageQ_Module__diagsIncluded__C)
                  0084ea28    00000004     bench_shm_pe66.oe66 (.const:ti_sdo_ipc_MessageQ_Module__diagsMask__C)
                  0084ea2c    00000004     bench_shm_pe66.oe66 (.const:ti_sdo_ipc_MessageQ_Module__loggerFxn4__C)
                  0084ea30    00000004     bench_shm_pe66.oe66 (.const:ti_sdo_ipc_MessageQ_Module__loggerObj__C)
                  0084ea34    00000004     bench_shm_pe66.oe66 (.const:ti_sdo_ipc_MessageQ_Object__count__C)
                  0084ea38    00000004     bench_shm_pe66.oe66 (.const:ti_sdo_ipc_MessageQ_Object__heap__C)
                  0084ea3c    00000004     bench_shm_pe66.oe66 (.const:ti_sdo_ipc_MessageQ_Object__table__C)
                  0084ea40    00000004     bench_shm_pe66.oe66 (.const:ti_sdo_ipc_MessageQ_maxRuntimeEntries__C)
                  0084ea44    00000004     bench_shm_pe66.oe66 (.const:ti_sdo_ipc_Notify_A_alreadyRegistered__C)
                  0084ea48    00000004     bench_shm_pe66.oe66 (.const:ti_sdo_ipc_Notify_A_internal__C)
                  0084ea4c    00000004     bench_shm_pe66.oe66 (.const:ti_sdo_ipc_Notify_A_invArgument__C)
                  0084ea50    00000004     bench_shm_pe66.oe66 (.const:ti_sdo_ipc_Notify_A_notRegistered__C)
                  0084ea54    00000004     bench_shm_pe66.oe66 (.const:ti_sdo_ipc_Notify_A_reservedEvent__C)
                  0084ea58    00000004     bench_shm_pe66.oe66 (.const:ti_sdo_ipc_Notify_Module__diagsEnabled__C)
                  0084ea5c    00000004     bench_shm_pe66.oe66 (.const:ti_sdo_ipc_Notify_Module__diagsIncluded__C)
                  0084ea60    00000004     bench_shm_pe66.oe66 (.const:ti_sdo_ipc_Notify_Module__diagsMask__C)
                  0084ea64    00000004     bench_shm_pe66.oe66 (.const:ti_sdo_ipc_Notify_Module__gateObj__C)
                  0084ea68    00000004     bench_shm_pe66.oe66 (.const:ti_sdo_ipc_Notify_Object__heap__C)
                  0084ea6c    00000004     bench_shm_pe66.oe66 (.const:ti_sdo_ipc_Notify_numEvents__C)
                  0084ea70    00000004     bench_shm_pe66.oe66 (.const:ti_sdo_ipc_SharedRegion_A_addrOutOfRange__C)
                  0084ea74    00000004     bench_shm_pe66.oe66 (.const:ti_sdo_ipc_SharedRegion_A_idTooLarge__C)
                  0084ea78    00000004     bench_shm_pe66.oe66 (.const:ti_sdo_ipc_SharedRegion_A_noHeap__C)
                  0084ea7c    00000004     bench_shm_pe66.oe66 (.const:ti_sdo_ipc_SharedRegion_A_region0Invalid__C)
                  0084ea80    00000004     bench_shm_pe66.oe66 (.const:ti_sdo_ipc_SharedRegion_A_regionInvalid__C)
                  0084ea84    00000004     bench_shm_pe66.oe66 (.const:ti_sdo_ipc_SharedRegion_A_reserveTooMuch__C)
                  0084ea88    00000004     bench_shm_pe66.oe66 (.const:ti_sdo_ipc_SharedRegion_INVALIDSRPTR__C)
                  0084ea8c    00000004     bench_shm_pe66.oe66 (.const:ti_sdo_ipc_SharedRegion_Module__diagsEnabled__C)
                  0084ea90    00000004     bench_shm_pe66.oe66 (.const:ti_sdo_ipc_SharedRegion_Module__diagsIncluded__C)
                  0084ea94    00000004     bench_shm_pe66.oe66 (.const:ti_sdo_ipc_SharedRegion_Module__diagsMask__C)
                  0084ea98    00000004     bench_shm_pe66.oe66 (.const:ti_sdo_ipc_SharedRegion_cacheLineSize__C)
                  0084ea9c    00000004     bench_shm_pe66.oe66 (.const:ti_sdo_ipc_SharedRegion_numOffsetBits__C)
                  0084eaa0    00000004     bench_shm_pe66.oe66 (.const:ti_sdo_ipc_SharedRegion_offsetMask__C)
                  0084eaa4    00000004     bench_shm_pe66.oe66 (.const:ti_sdo_ipc_family_c647x_Interrupt_INTERDSPINT__C)
                  0084eaa8    00000004     bench_shm_pe66.oe66 (.const:ti_sdo_ipc_family_c647x_Interrupt_IPCAR0__C)
                  0084eaac    00000004     bench_shm_pe66.oe66 (.const:ti_sdo_ipc_family_c647x_Interrupt_IPCGR0__C)
                  0084eab0    00000004     bench_shm_pe66.oe66 (.const:ti_sdo_ipc_family_c647x_Interrupt_KICK0__C)
                  0084eab4    00000004     bench_shm_pe66.oe66 (.const:ti_sdo_ipc_family_c647x_Interrupt_KICK1__C)
                  0084eab8    00000004     bench_shm_pe66.oe66 (.const:ti_sdo_ipc_family_c647x_MultiProcSetup_A_invalidProcessor__C)
                  0084eabc    00000004     bench_shm_pe66.oe66 (.const:ti_sdo_ipc_family_c647x_MultiProcSetup_Module__diagsEnabled__C)
                  0084eac0    00000004     bench_shm_pe66.oe66 (.const:ti_sdo_ipc_family_c647x_MultiProcSetup_Module__diagsIncluded__C)
                  0084eac4    00000004     bench_shm_pe66.oe66 (.const:ti_sdo_ipc_family_c647x_MultiProcSetup_Module__diagsMask__C)
                  0084eac8    00000004     bench_shm_pe66.oe66 (.const:ti_sdo_ipc_family_c647x_MultiProcSetup_procMap__A)
                  0084eacc    00000004     bench_shm_pe66.oe66 (.const:ti_sdo_ipc_family_c647x_MultiProcSetup_procMap__C)
                  0084ead0    00000004     bench_shm_pe66.oe66 (.const:ti_sdo_ipc_family_c647x_NotifyCircSetup_dspIntVectId__C)
                  0084ead4    00000004     bench_shm_pe66.oe66 (.const:ti_sdo_ipc_gates_GateHWSem_A_invSemNum__C)
                  0084ead8    00000004     bench_shm_pe66.oe66 (.const:ti_sdo_ipc_gates_GateHWSem_Module__diagsEnabled__C)
                  0084eadc    00000004     bench_shm_pe66.oe66 (.const:ti_sdo_ipc_gates_GateHWSem_Module__diagsIncluded__C)
                  0084eae0    00000004     bench_shm_pe66.oe66 (.const:ti_sdo_ipc_gates_GateHWSem_Module__diagsMask__C)
                  0084eae4    00000004     bench_shm_pe66.oe66 (.const:ti_sdo_ipc_gates_GateHWSem_baseAddr__C)
                  0084eae8    00000004     bench_shm_pe66.oe66 (.const:ti_sdo_ipc_gates_GateHWSem_numSems__C)
                  0084eaec    00000004     bench_shm_pe66.oe66 (.const:ti_sdo_ipc_gates_GateHWSem_reservedMaskArr__C)
                  0084eaf0    00000004     bench_shm_pe66.oe66 (.const:ti_sdo_ipc_gates_GateHWSem_reservedMaskArr__A)
                  0084eaf4    00000004     bench_shm_pe66.oe66 (.const:ti_sdo_ipc_gates_GateMPSupportNull_A_invalidAction__C)
                  0084eaf8    00000004     bench_shm_pe66.oe66 (.const:ti_sdo_ipc_gates_GateMPSupportNull_Module__diagsEnabled__C)
                  0084eafc    00000004     bench_shm_pe66.oe66 (.const:ti_sdo_ipc_gates_GateMPSupportNull_Module__diagsIncluded__C)
                  0084eb00    00000004     bench_shm_pe66.oe66 (.const:ti_sdo_ipc_gates_GateMPSupportNull_Module__diagsMask__C)
                  0084eb04    00000004     bench_shm_pe66.oe66 (.const:ti_sdo_ipc_gates_GateMPSupportNull_action__C)
                  0084eb08    00000004     bench_shm_pe66.oe66 (.const:ti_sdo_ipc_gates_GatePeterson_E_gateRemotelyOpened__C)
                  0084eb0c    00000004     bench_shm_pe66.oe66 (.const:ti_sdo_ipc_gates_GatePeterson_Module__diagsEnabled__C)
                  0084eb10    00000004     bench_shm_pe66.oe66 (.const:ti_sdo_ipc_gates_GatePeterson_Module__diagsIncluded__C)
                  0084eb14    00000004     bench_shm_pe66.oe66 (.const:ti_sdo_ipc_gates_GatePeterson_Module__diagsMask__C)
                  0084eb18    00000004     bench_shm_pe66.oe66 (.const:ti_sdo_ipc_gates_GatePeterson_numInstances__C)
                  0084eb1c    00000004     bench_shm_pe66.oe66 (.const:ti_sdo_ipc_heaps_HeapMemMP_A_align__C)
                  0084eb20    00000004     bench_shm_pe66.oe66 (.const:ti_sdo_ipc_heaps_HeapMemMP_A_heapSize__C)
                  0084eb24    00000004     bench_shm_pe66.oe66 (.const:ti_sdo_ipc_heaps_HeapMemMP_A_invalidFree__C)
                  0084eb28    00000004     bench_shm_pe66.oe66 (.const:ti_sdo_ipc_heaps_HeapMemMP_A_zeroBlock__C)
                  0084eb2c    00000004     bench_shm_pe66.oe66 (.const:ti_sdo_ipc_heaps_HeapMemMP_E_memory__C)
                  0084eb30    00000004     bench_shm_pe66.oe66 (.const:ti_sdo_ipc_heaps_HeapMemMP_Module__diagsEnabled__C)
                  0084eb34    00000004     bench_shm_pe66.oe66 (.const:ti_sdo_ipc_heaps_HeapMemMP_Module__diagsIncluded__C)
                  0084eb38    00000004     bench_shm_pe66.oe66 (.const:ti_sdo_ipc_heaps_HeapMemMP_Module__diagsMask__C)
                  0084eb3c    00000004     bench_shm_pe66.oe66 (.const:ti_sdo_ipc_interfaces_IGateMPSupport_Interface__BASE__C)
                  0084eb40    00000004     bench_shm_pe66.oe66 (.const:ti_sdo_ipc_interfaces_IMessageQTransport_Interface__BASE__C)
                  0084eb44    00000004     bench_shm_pe66.oe66 (.const:ti_sdo_ipc_interfaces_INotifyDriver_Interface__BASE__C)
                  0084eb48    00000004     bench_shm_pe66.oe66 (.const:ti_sdo_ipc_notifyDrivers_NotifyDriverCirc_A_notSupported__C)
                  0084eb4c    00000004     bench_shm_pe66.oe66 (.const:ti_sdo_ipc_notifyDrivers_NotifyDriverCirc_Module__diagsEnabled__C)
                  0084eb50    00000004     bench_shm_pe66.oe66 (.const:ti_sdo_ipc_notifyDrivers_NotifyDriverCirc_Module__diagsIncluded__C)
                  0084eb54    00000004     bench_shm_pe66.oe66 (.const:ti_sdo_ipc_notifyDrivers_NotifyDriverCirc_Module__diagsMask__C)
                  0084eb58    00000004     bench_shm_pe66.oe66 (.const:ti_sdo_ipc_notifyDrivers_NotifyDriverCirc_maxIndex__C)
                  0084eb5c    00000004     bench_shm_pe66.oe66 (.const:ti_sdo_ipc_notifyDrivers_NotifyDriverCirc_modIndex__C)
                  0084eb60    00000004     bench_shm_pe66.oe66 (.const:ti_sdo_ipc_notifyDrivers_NotifyDriverCirc_numMsgs__C)
                  0084eb64    00000004     bench_shm_pe66.oe66 (.const:ti_sdo_ipc_nsremote_NameServerRemoteNotify_A_invalidValueLen__C)
                  0084eb68    00000004     bench_shm_pe66.oe66 (.const:ti_sdo_ipc_nsremote_NameServerRemoteNotify_Instance_State_semMultiBlock__O)
                  0084eb6c    00000004     bench_shm_pe66.oe66 (.const:ti_sdo_ipc_nsremote_NameServerRemoteNotify_Instance_State_semRemoteWait__O)
                  0084eb70    00000004     bench_shm_pe66.oe66 (.const:ti_sdo_ipc_nsremote_NameServerRemoteNotify_Instance_State_swiObj__O)
                  0084eb74    00000004     bench_shm_pe66.oe66 (.const:ti_sdo_ipc_nsremote_NameServerRemoteNotify_Module__diagsEnabled__C)
                  0084eb78    00000004     bench_shm_pe66.oe66 (.const:ti_sdo_ipc_nsremote_NameServerRemoteNotify_Module__diagsIncluded__C)
                  0084eb7c    00000004     bench_shm_pe66.oe66 (.const:ti_sdo_ipc_nsremote_NameServerRemoteNotify_Module__diagsMask__C)
                  0084eb80    00000004     bench_shm_pe66.oe66 (.const:ti_sdo_ipc_nsremote_NameServerRemoteNotify_notifyEventId__C)
                  0084eb84    00000004     bench_shm_pe66.oe66 (.const:ti_sdo_ipc_nsremote_NameServerRemoteNotify_timeout__C)
                  0084eb88    00000004     bench_shm_pe66.oe66 (.const:ti_sdo_ipc_transports_TransportShmNotifySetup_priority__C)
                  0084eb8c    00000004     bench_shm_pe66.oe66 (.const:ti_sdo_utils_INameServerRemote_Interface__BASE__C)
                  0084eb90    00000004     bench_shm_pe66.oe66 (.const:ti_sdo_utils_List_Object__count__C)
                  0084eb94    00000004     bench_shm_pe66.oe66 (.const:ti_sdo_utils_List_Object__table__C)
                  0084eb98    00000004     bench_shm_pe66.oe66 (.const:ti_sdo_utils_MultiProc_A_invalidMultiProcId__C)
                  0084eb9c    00000004     bench_shm_pe66.oe66 (.const:ti_sdo_utils_MultiProc_Module__diagsEnabled__C)
                  0084eba0    00000004     bench_shm_pe66.oe66 (.const:ti_sdo_utils_MultiProc_Module__diagsIncluded__C)
                  0084eba4    00000004     bench_shm_pe66.oe66 (.const:ti_sdo_utils_MultiProc_Module__diagsMask__C)
                  0084eba8    00000004     bench_shm_pe66.oe66 (.const:ti_sdo_utils_MultiProc_nameList__C)
                  0084ebac    00000004     bench_shm_pe66.oe66 (.const:ti_sdo_utils_NameServer_A_invArgument__C)
                  0084ebb0    00000004     bench_shm_pe66.oe66 (.const:ti_sdo_utils_NameServer_A_invalidLen__C)
                  0084ebb4    00000004     bench_shm_pe66.oe66 (.const:ti_sdo_utils_NameServer_E_entryExists__C)
                  0084ebb8    00000004     bench_shm_pe66.oe66 (.const:ti_sdo_utils_NameServer_E_maxReached__C)
                  0084ebbc    00000004     bench_shm_pe66.oe66 (.const:ti_sdo_utils_NameServer_Instance_State_freeList__O)
                  0084ebc0    00000004     bench_shm_pe66.oe66 (.const:ti_sdo_utils_NameServer_Instance_State_nameList__O)
                  0084ebc4    00000004     bench_shm_pe66.oe66 (.const:ti_sdo_utils_NameServer_Module__diagsEnabled__C)
                  0084ebc8    00000004     bench_shm_pe66.oe66 (.const:ti_sdo_utils_NameServer_Module__diagsIncluded__C)
                  0084ebcc    00000004     bench_shm_pe66.oe66 (.const:ti_sdo_utils_NameServer_Module__diagsMask__C)
                  0084ebd0    00000004     bench_shm_pe66.oe66 (.const:ti_sdo_utils_NameServer_Object__count__C)
                  0084ebd4    00000004     bench_shm_pe66.oe66 (.const:ti_sdo_utils_NameServer_Object__table__C)
                  0084ebd8    00000004     bench_shm_pe66.oe66 (.const:ti_sysbios_BIOS_Module__diagsEnabled__C)
                  0084ebdc    00000004     bench_shm_pe66.oe66 (.const:ti_sysbios_BIOS_Module__diagsIncluded__C)
                  0084ebe0    00000004     bench_shm_pe66.oe66 (.const:ti_sysbios_BIOS_Module__diagsMask__C)
                  0084ebe4    00000004     bench_shm_pe66.oe66 (.const:ti_sysbios_BIOS_installedErrorHook__C)
                  0084ebe8    00000004     bench_shm_pe66.oe66 (.const:ti_sysbios_family_c64p_Exception_E_exceptionMin__C)
                  0084ebec    00000004     bench_shm_pe66.oe66 (.const:ti_sysbios_family_c64p_Exception_exceptionHook__C)
                  0084ebf0    00000004     bench_shm_pe66.oe66 (.const:ti_sysbios_family_c64p_Exception_externalHook__C)
                  0084ebf4    00000004     bench_shm_pe66.oe66 (.const:ti_sysbios_family_c64p_Exception_internalHook__C)
                  0084ebf8    00000004     bench_shm_pe66.oe66 (.const:ti_sysbios_family_c64p_Exception_nmiHook__C)
                  0084ebfc    00000004     bench_shm_pe66.oe66 (.const:ti_sysbios_family_c64p_Hwi_E_alreadyDefined__C)
                  0084ec00    00000004     bench_shm_pe66.oe66 (.const:ti_sysbios_family_c64p_Hwi_E_handleNotFound__C)
                  0084ec04    00000004     bench_shm_pe66.oe66 (.const:ti_sysbios_family_c64p_Hwi_LD_end__C)
                  0084ec08    00000004     bench_shm_pe66.oe66 (.const:ti_sysbios_family_c64p_Hwi_LM_begin__C)
                  0084ec0c    00000004     bench_shm_pe66.oe66 (.const:ti_sysbios_family_c64p_Hwi_Module__diagsEnabled__C)
                  0084ec10    00000004     bench_shm_pe66.oe66 (.const:ti_sysbios_family_c64p_Hwi_Module__diagsIncluded__C)
                  0084ec14    00000004     bench_shm_pe66.oe66 (.const:ti_sysbios_family_c64p_Hwi_Module__diagsMask__C)
                  0084ec18    00000004     bench_shm_pe66.oe66 (.const:ti_sysbios_family_c64p_Hwi_Module__loggerFxn1__C)
                  0084ec1c    00000004     bench_shm_pe66.oe66 (.const:ti_sysbios_family_c64p_Hwi_Module__loggerFxn8__C)
                  0084ec20    00000004     bench_shm_pe66.oe66 (.const:ti_sysbios_family_c64p_Hwi_Module__loggerObj__C)
                  0084ec24    00000004     bench_shm_pe66.oe66 (.const:ti_sysbios_family_c66_Cache_atomicBlockSize__C)
                  0084ec28    00000004     bench_shm_pe66.oe66 (.const:ti_sysbios_gates_GateMutexPri_A_badContext__C)
                  0084ec2c    00000004     bench_shm_pe66.oe66 (.const:ti_sysbios_gates_GateMutexPri_Instance_State_pendQ__O)
                  0084ec30    00000004     bench_shm_pe66.oe66 (.const:ti_sysbios_gates_GateMutexPri_Module__diagsEnabled__C)
                  0084ec34    00000004     bench_shm_pe66.oe66 (.const:ti_sysbios_gates_GateMutexPri_Module__diagsIncluded__C)
                  0084ec38    00000004     bench_shm_pe66.oe66 (.const:ti_sysbios_gates_GateMutexPri_Module__diagsMask__C)
                  0084ec3c    00000004     bench_shm_pe66.oe66 (.const:ti_sysbios_gates_GateMutex_A_badContext__C)
                  0084ec40    00000004     bench_shm_pe66.oe66 (.const:ti_sysbios_gates_GateMutex_Instance_State_sem__O)
                  0084ec44    00000004     bench_shm_pe66.oe66 (.const:ti_sysbios_gates_GateMutex_Module__diagsEnabled__C)
                  0084ec48    00000004     bench_shm_pe66.oe66 (.const:ti_sysbios_gates_GateMutex_Module__diagsIncluded__C)
                  0084ec4c    00000004     bench_shm_pe66.oe66 (.const:ti_sysbios_gates_GateMutex_Module__diagsMask__C)
                  0084ec50    00000004     bench_shm_pe66.oe66 (.const:ti_sysbios_gates_GateSwi_A_badContext__C)
                  0084ec54    00000004     bench_shm_pe66.oe66 (.const:ti_sysbios_gates_GateSwi_Module__diagsEnabled__C)
                  0084ec58    00000004     bench_shm_pe66.oe66 (.const:ti_sysbios_gates_GateSwi_Module__diagsIncluded__C)
                  0084ec5c    00000004     bench_shm_pe66.oe66 (.const:ti_sysbios_gates_GateSwi_Module__diagsMask__C)
                  0084ec60    00000004     bench_shm_pe66.oe66 (.const:ti_sysbios_hal_Hwi_E_stackOverflow__C)
                  0084ec64    00000004     bench_shm_pe66.oe66 (.const:ti_sysbios_heaps_HeapMem_A_align__C)
                  0084ec68    00000004     bench_shm_pe66.oe66 (.const:ti_sysbios_heaps_HeapMem_A_heapSize__C)
                  0084ec6c    00000004     bench_shm_pe66.oe66 (.const:ti_sysbios_heaps_HeapMem_A_invalidFree__C)
                  0084ec70    00000004     bench_shm_pe66.oe66 (.const:ti_sysbios_heaps_HeapMem_A_zeroBlock__C)
                  0084ec74    00000004     bench_shm_pe66.oe66 (.const:ti_sysbios_heaps_HeapMem_E_memory__C)
                  0084ec78    00000004     bench_shm_pe66.oe66 (.const:ti_sysbios_heaps_HeapMem_Module__diagsEnabled__C)
                  0084ec7c    00000004     bench_shm_pe66.oe66 (.const:ti_sysbios_heaps_HeapMem_Module__diagsIncluded__C)
                  0084ec80    00000004     bench_shm_pe66.oe66 (.const:ti_sysbios_heaps_HeapMem_Module__diagsMask__C)
                  0084ec84    00000004     bench_shm_pe66.oe66 (.const:ti_sysbios_heaps_HeapMem_Module__gateObj__C)
                  0084ec88    00000004     bench_shm_pe66.oe66 (.const:ti_sysbios_heaps_HeapMem_Object__count__C)
                  0084ec8c    00000004     bench_shm_pe66.oe66 (.const:ti_sysbios_heaps_HeapMem_Object__table__C)
                  0084ec90    00000004     bench_shm_pe66.oe66 (.const:ti_sysbios_heaps_HeapMem_reqAlignMask__C)
                  0084ec94    00000004     bench_shm_pe66.oe66 (.const:ti_sysbios_heaps_HeapMem_reqAlign__C)
                  0084ec98    00000004     bench_shm_pe66.oe66 (.const:ti_sysbios_knl_Clock_A_badThreadType__C)
                  0084ec9c    00000004     bench_shm_pe66.oe66 (.const:ti_sysbios_knl_Clock_LM_begin__C)
                  0084eca0    00000004     bench_shm_pe66.oe66 (.const:ti_sysbios_knl_Clock_LM_tick__C)
                  0084eca4    00000004     bench_shm_pe66.oe66 (.const:ti_sysbios_knl_Clock_LW_delayed__C)
                  0084eca8    00000004     bench_shm_pe66.oe66 (.const:ti_sysbios_knl_Clock_Module_State_clockQ__O)
                  0084ecac    00000004     bench_shm_pe66.oe66 (.const:ti_sysbios_knl_Clock_Module__diagsEnabled__C)
                  0084ecb0    00000004     bench_shm_pe66.oe66 (.const:ti_sysbios_knl_Clock_Module__diagsIncluded__C)
                  0084ecb4    00000004     bench_shm_pe66.oe66 (.const:ti_sysbios_knl_Clock_Module__diagsMask__C)
                  0084ecb8    00000004     bench_shm_pe66.oe66 (.const:ti_sysbios_knl_Clock_Module__loggerFxn1__C)
                  0084ecbc    00000004     bench_shm_pe66.oe66 (.const:ti_sysbios_knl_Clock_Module__loggerFxn2__C)
                  0084ecc0    00000004     bench_shm_pe66.oe66 (.const:ti_sysbios_knl_Clock_Module__loggerObj__C)
                  0084ecc4    00000004     bench_shm_pe66.oe66 (.const:ti_sysbios_knl_Clock_tickMode__C)
                  0084ecc8    00000004     bench_shm_pe66.oe66 (.const:ti_sysbios_knl_Clock_tickPeriod__C)
                  0084eccc    00000004     bench_shm_pe66.oe66 (.const:ti_sysbios_knl_Clock_tickSource__C)
                  0084ecd0    00000004     bench_shm_pe66.oe66 (.const:ti_sysbios_knl_Idle_funcList__A)
                  0084ecd4    00000004     bench_shm_pe66.oe66 (.const:ti_sysbios_knl_Queue_Object__count__C)
                  0084ecd8    00000004     bench_shm_pe66.oe66 (.const:ti_sysbios_knl_Queue_Object__table__C)
                  0084ecdc    00000004     bench_shm_pe66.oe66 (.const:ti_sysbios_knl_Semaphore_A_badContext__C)
                  0084ece0    00000004     bench_shm_pe66.oe66 (.const:ti_sysbios_knl_Semaphore_A_noEvents__C)
                  0084ece4    00000004     bench_shm_pe66.oe66 (.const:ti_sysbios_knl_Semaphore_A_overflow__C)
                  0084ece8    00000004     bench_shm_pe66.oe66 (.const:ti_sysbios_knl_Semaphore_Instance_State_pendQ__O)
                  0084ecec    00000004     bench_shm_pe66.oe66 (.const:ti_sysbios_knl_Semaphore_LM_pend__C)
                  0084ecf0    00000004     bench_shm_pe66.oe66 (.const:ti_sysbios_knl_Semaphore_LM_post__C)
                  0084ecf4    00000004     bench_shm_pe66.oe66 (.const:ti_sysbios_knl_Semaphore_Module__diagsEnabled__C)
                  0084ecf8    00000004     bench_shm_pe66.oe66 (.const:ti_sysbios_knl_Semaphore_Module__diagsIncluded__C)
                  0084ecfc    00000004     bench_shm_pe66.oe66 (.const:ti_sysbios_knl_Semaphore_Module__diagsMask__C)
                  0084ed00    00000004     bench_shm_pe66.oe66 (.const:ti_sysbios_knl_Semaphore_Module__loggerFxn2__C)
                  0084ed04    00000004     bench_shm_pe66.oe66 (.const:ti_sysbios_knl_Semaphore_Module__loggerFxn4__C)
                  0084ed08    00000004     bench_shm_pe66.oe66 (.const:ti_sysbios_knl_Semaphore_Module__loggerObj__C)
                  0084ed0c    00000004     bench_shm_pe66.oe66 (.const:ti_sysbios_knl_Swi_A_badPriority__C)
                  0084ed10    00000004     bench_shm_pe66.oe66 (.const:ti_sysbios_knl_Swi_LD_end__C)
                  0084ed14    00000004     bench_shm_pe66.oe66 (.const:ti_sysbios_knl_Swi_LM_begin__C)
                  0084ed18    00000004     bench_shm_pe66.oe66 (.const:ti_sysbios_knl_Swi_LM_post__C)
                  0084ed1c    00000004     bench_shm_pe66.oe66 (.const:ti_sysbios_knl_Swi_Module__diagsEnabled__C)
                  0084ed20    00000004     bench_shm_pe66.oe66 (.const:ti_sysbios_knl_Swi_Module__diagsIncluded__C)
                  0084ed24    00000004     bench_shm_pe66.oe66 (.const:ti_sysbios_knl_Swi_Module__diagsMask__C)
                  0084ed28    00000004     bench_shm_pe66.oe66 (.const:ti_sysbios_knl_Swi_Module__loggerFxn1__C)
                  0084ed2c    00000004     bench_shm_pe66.oe66 (.const:ti_sysbios_knl_Swi_Module__loggerFxn4__C)
                  0084ed30    00000004     bench_shm_pe66.oe66 (.const:ti_sysbios_knl_Swi_Module__loggerObj__C)
                  0084ed34    00000004     bench_shm_pe66.oe66 (.const:ti_sysbios_knl_Swi_Object__count__C)
                  0084ed38    00000004     bench_shm_pe66.oe66 (.const:ti_sysbios_knl_Swi_Object__table__C)
                  0084ed3c    00000004     bench_shm_pe66.oe66 (.const:ti_sysbios_knl_Task_A_badPriority__C)
                  0084ed40    00000004     bench_shm_pe66.oe66 (.const:ti_sysbios_knl_Task_E_spOutOfBounds__C)
                  0084ed44    00000004     bench_shm_pe66.oe66 (.const:ti_sysbios_knl_Task_E_stackOverflow__C)
                  0084ed48    00000004     bench_shm_pe66.oe66 (.const:ti_sysbios_knl_Task_LD_block__C)
                  0084ed4c    00000004     bench_shm_pe66.oe66 (.const:ti_sysbios_knl_Task_LD_exit__C)
                  0084ed50    00000004     bench_shm_pe66.oe66 (.const:ti_sysbios_knl_Task_LD_ready__C)
                  0084ed54    00000004     bench_shm_pe66.oe66 (.const:ti_sysbios_knl_Task_LM_setPri__C)
                  0084ed58    00000004     bench_shm_pe66.oe66 (.const:ti_sysbios_knl_Task_LM_switch__C)
                  0084ed5c    00000004     bench_shm_pe66.oe66 (.const:ti_sysbios_knl_Task_LM_yield__C)
                  0084ed60    00000004     bench_shm_pe66.oe66 (.const:ti_sysbios_knl_Task_Module_State_inactiveQ__O)
                  0084ed64    00000004     bench_shm_pe66.oe66 (.const:ti_sysbios_knl_Task_Module_State_terminatedQ__O)
                  0084ed68    00000004     bench_shm_pe66.oe66 (.const:ti_sysbios_knl_Task_Module__diagsEnabled__C)
                  0084ed6c    00000004     bench_shm_pe66.oe66 (.const:ti_sysbios_knl_Task_Module__diagsIncluded__C)
                  0084ed70    00000004     bench_shm_pe66.oe66 (.const:ti_sysbios_knl_Task_Module__diagsMask__C)
                  0084ed74    00000004     bench_shm_pe66.oe66 (.const:ti_sysbios_knl_Task_Module__loggerFxn2__C)
                  0084ed78    00000004     bench_shm_pe66.oe66 (.const:ti_sysbios_knl_Task_Module__loggerFxn4__C)
                  0084ed7c    00000004     bench_shm_pe66.oe66 (.const:ti_sysbios_knl_Task_Module__loggerObj__C)
                  0084ed80    00000004     bench_shm_pe66.oe66 (.const:ti_sysbios_knl_Task_Object__count__C)
                  0084ed84    00000004     bench_shm_pe66.oe66 (.const:ti_sysbios_knl_Task_Object__table__C)
                  0084ed88    00000004     bench_shm_pe66.oe66 (.const:ti_sysbios_knl_Task_allBlockedFunc__C)
                  0084ed8c    00000004     bench_shm_pe66.oe66 (.const:ti_sysbios_knl_Task_numConstructedTasks__C)
                  0084ed90    00000004     bench_shm_pe66.oe66 (.const:ti_sysbios_knl_Task_numPriorities__C)
                  0084ed94    00000004     bench_shm_pe66.oe66 (.const:ti_sysbios_syncs_SyncSem_Module__diagsEnabled__C)
                  0084ed98    00000004     bench_shm_pe66.oe66 (.const:ti_sysbios_syncs_SyncSem_Module__diagsIncluded__C)
                  0084ed9c    00000004     bench_shm_pe66.oe66 (.const:ti_sysbios_syncs_SyncSem_Module__diagsMask__C)
                  0084eda0    00000004     bench_shm_pe66.oe66 (.const:ti_sysbios_timers_timer64_Timer_A_notAvailable__C)
                  0084eda4    00000004     bench_shm_pe66.oe66 (.const:ti_sysbios_timers_timer64_Timer_E_cannotSupport__C)
                  0084eda8    00000004     bench_shm_pe66.oe66 (.const:ti_sysbios_timers_timer64_Timer_Module__diagsEnabled__C)
                  0084edac    00000004     bench_shm_pe66.oe66 (.const:ti_sysbios_timers_timer64_Timer_Module__diagsIncluded__C)
                  0084edb0    00000004     bench_shm_pe66.oe66 (.const:ti_sysbios_timers_timer64_Timer_Module__diagsMask__C)
                  0084edb4    00000004     bench_shm_pe66.oe66 (.const:ti_sysbios_timers_timer64_Timer_anyMask__C)
                  0084edb8    00000004     bench_shm_pe66.oe66 (.const:ti_sysbios_timers_timer64_Timer_freqDivisor__C)
                  0084edbc    00000004     bench_shm_pe66.oe66 (.const:ti_sysbios_timers_timer64_Timer_numLocalTimers__C)
                  0084edc0    00000004     bench_shm_pe66.oe66 (.const:ti_sysbios_timers_timer64_Timer_numTimerDevices__C)
                  0084edc4    00000004     bench_shm_pe66.oe66 (.const:ti_sysbios_xdcruntime_GateThreadSupport_Instance_State_gate__O)
                  0084edc8    00000004     bench_shm_pe66.oe66 (.const:xdc_runtime_Assert_E_assertFailed__C)
                  0084edcc    00000004     bench_shm_pe66.oe66 (.const:xdc_runtime_Core_A_initializedParams__C)
                  0084edd0    00000004     bench_shm_pe66.oe66 (.const:xdc_runtime_Core_Module__diagsEnabled__C)
                  0084edd4    00000004     bench_shm_pe66.oe66 (.const:xdc_runtime_Core_Module__diagsIncluded__C)
                  0084edd8    00000004     bench_shm_pe66.oe66 (.const:xdc_runtime_Core_Module__diagsMask__C)
                  0084eddc    00000004     bench_shm_pe66.oe66 (.const:xdc_runtime_Error_E_generic__C)
                  0084ede0    00000004     bench_shm_pe66.oe66 (.const:xdc_runtime_Error_E_memory__C)
                  0084ede4    00000004     bench_shm_pe66.oe66 (.const:xdc_runtime_Error_Module__diagsEnabled__C)
                  0084ede8    00000004     bench_shm_pe66.oe66 (.const:xdc_runtime_Error_Module__diagsIncluded__C)
                  0084edec    00000004     bench_shm_pe66.oe66 (.const:xdc_runtime_Error_Module__diagsMask__C)
                  0084edf0    00000004     bench_shm_pe66.oe66 (.const:xdc_runtime_Error_Module__loggerFxn8__C)
                  0084edf4    00000004     bench_shm_pe66.oe66 (.const:xdc_runtime_Error_Module__loggerObj__C)
                  0084edf8    00000004     bench_shm_pe66.oe66 (.const:xdc_runtime_Error_policy__C)
                  0084edfc    00000004     bench_shm_pe66.oe66 (.const:xdc_runtime_Error_raiseHook__C)
                  0084ee00    00000004     bench_shm_pe66.oe66 (.const:xdc_runtime_IGateProvider_Interface__BASE__C)
                  0084ee04    00000004     bench_shm_pe66.oe66 (.const:xdc_runtime_IHeap_Interface__BASE__C)
                  0084ee08    00000004     bench_shm_pe66.oe66 (.const:xdc_runtime_IModule_Interface__BASE__C)
                  0084ee0c    00000004     bench_shm_pe66.oe66 (.const:xdc_runtime_Log_L_error__C)
                  0084ee10    00000004     bench_shm_pe66.oe66 (.const:xdc_runtime_Main_Module__diagsEnabled__C)
                  0084ee14    00000004     bench_shm_pe66.oe66 (.const:xdc_runtime_Main_Module__diagsIncluded__C)
                  0084ee18    00000004     bench_shm_pe66.oe66 (.const:xdc_runtime_Main_Module__diagsMask__C)
                  0084ee1c    00000004     bench_shm_pe66.oe66 (.const:xdc_runtime_Memory_defaultHeapInstance__C)
                  0084ee20    00000004     bench_shm_pe66.oe66 (.const:xdc_runtime_Startup_execImpl__C)
                  0084ee24    00000004     bench_shm_pe66.oe66 (.const:xdc_runtime_Startup_maxPasses__C)
                  0084ee28    00000004     bench_shm_pe66.oe66 (.const:xdc_runtime_Startup_lastFxns__A)
                  0084ee2c    00000004     bench_shm_pe66.oe66 (.const:xdc_runtime_Startup_sfxnRts__C)
                  0084ee30    00000004     bench_shm_pe66.oe66 (.const:xdc_runtime_Startup_sfxnTab__C)
                  0084ee34    00000004     bench_shm_pe66.oe66 (.const:xdc_runtime_Startup_startModsFxn__C)
                  0084ee38    00000004     bench_shm_pe66.oe66 (.const:xdc_runtime_System_A_cannotFitIntoArg__C)
                  0084ee3c    00000004     bench_shm_pe66.oe66 (.const:xdc_runtime_System_Module__gateObj__C)
                  0084ee40    00000004     bench_shm_pe66.oe66 (.const:xdc_runtime_System_extendFxn__C)
                  0084ee44    00000004     bench_shm_pe66.oe66 (.const:xdc_runtime_System_maxAtexitHandlers__C)
                  0084ee48    00000004     bench_shm_pe66.oe66 (.const:xdc_runtime_Text_charTab__C)
                  0084ee4c    00000004     bench_shm_pe66.oe66 (.const:xdc_runtime_Text_nameEmpty__C)
                  0084ee50    00000004     bench_shm_pe66.oe66 (.const:xdc_runtime_Text_nameStatic__C)
                  0084ee54    00000004     bench_shm_pe66.oe66 (.const:xdc_runtime_Text_nameUnknown__C)
                  0084ee58    00000004     bench_shm_pe66.oe66 (.const:xdc_runtime_Text_nodeTab__C)
                  0084ee5c    00000004     bench_shm_pe66.oe66 (.const:xdc_runtime_Text_visitRopeFxn__C)
                  0084ee60    00000004     bench_shm_pe66.oe66 (.const:xdc_runtime_knl_ISync_Interface__BASE__C)
                  0084ee64    00000002     bench_shm_pe66.oe66 (.const:ti_sdo_ipc_GateMP_Module__id__C)
                  0084ee66    00000002     --HOLE-- [fill = 0]
                  0084ee68    00000002     bench_shm_pe66.oe66 (.const:ti_sdo_ipc_GateMP_Module__loggerDefined__C)
                  0084ee6a    00000002     --HOLE-- [fill = 0]
                  0084ee6c    00000002     bench_shm_pe66.oe66 (.const:ti_sdo_ipc_Ipc_Module__id__C)
                  0084ee6e    00000002     --HOLE-- [fill = 0]
                  0084ee70    00000002     bench_shm_pe66.oe66 (.const:ti_sdo_ipc_Ipc_generateSlaveDataForHost__C)
                  0084ee72    00000002     --HOLE-- [fill = 0]
                  0084ee74    00000002     bench_shm_pe66.oe66 (.const:ti_sdo_ipc_MessageQ_Module__id__C)
                  0084ee76    00000002     --HOLE-- [fill = 0]
                  0084ee78    00000002     bench_shm_pe66.oe66 (.const:ti_sdo_ipc_MessageQ_Module__loggerDefined__C)
                  0084ee7a    00000002     --HOLE-- [fill = 0]
                  0084ee7c    00000002     bench_shm_pe66.oe66 (.const:ti_sdo_ipc_Notify_Module__id__C)
                  0084ee7e    00000002     --HOLE-- [fill = 0]
                  0084ee80    00000002     bench_shm_pe66.oe66 (.const:ti_sdo_ipc_Notify_numLines__C)
                  0084ee82    00000002     --HOLE-- [fill = 0]
                  0084ee84    00000002     bench_shm_pe66.oe66 (.const:ti_sdo_ipc_Notify_reservedEvents__C)
                  0084ee86    00000002     --HOLE-- [fill = 0]
                  0084ee88    00000002     bench_shm_pe66.oe66 (.const:ti_sdo_ipc_SharedRegion_Module__id__C)
                  0084ee8a    00000002     --HOLE-- [fill = 0]
                  0084ee8c    00000002     bench_shm_pe66.oe66 (.const:ti_sdo_ipc_SharedRegion_numEntries__C)
                  0084ee8e    00000002     --HOLE-- [fill = 0]
                  0084ee90    00000002     bench_shm_pe66.oe66 (.const:ti_sdo_ipc_SharedRegion_translate__C)
                  0084ee92    00000002     --HOLE-- [fill = 0]
                  0084ee94    00000002     bench_shm_pe66.oe66 (.const:ti_sdo_ipc_family_c647x_Interrupt_enableKick__C)
                  0084ee96    00000002     --HOLE-- [fill = 0]
                  0084ee98    00000002     bench_shm_pe66.oe66 (.const:ti_sdo_ipc_family_c647x_MultiProcSetup_Module__id__C)
                  0084ee9a    00000002     --HOLE-- [fill = 0]
                  0084ee9c    00000002     bench_shm_pe66.oe66 (.const:ti_sdo_ipc_gates_GateHWSem_Module__id__C)
                  0084ee9e    00000002     --HOLE-- [fill = 0]
                  0084eea0    00000002     bench_shm_pe66.oe66 (.const:ti_sdo_ipc_gates_GateMPSupportNull_Module__id__C)
                  0084eea2    00000002     --HOLE-- [fill = 0]
                  0084eea4    00000002     bench_shm_pe66.oe66 (.const:ti_sdo_ipc_gates_GatePeterson_Module__id__C)
                  0084eea6    00000002     --HOLE-- [fill = 0]
                  0084eea8    00000002     bench_shm_pe66.oe66 (.const:ti_sdo_ipc_heaps_HeapMemMP_Module__id__C)
                  0084eeaa    00000002     --HOLE-- [fill = 0]
                  0084eeac    00000002     bench_shm_pe66.oe66 (.const:ti_sdo_ipc_notifyDrivers_NotifyDriverCirc_Module__id__C)
                  0084eeae    00000002     --HOLE-- [fill = 0]
                  0084eeb0    00000002     bench_shm_pe66.oe66 (.const:ti_sdo_ipc_notifyDrivers_NotifyDriverCirc_enableStats__C)
                  0084eeb2    00000002     --HOLE-- [fill = 0]
                  0084eeb4    00000002     bench_shm_pe66.oe66 (.const:ti_sdo_ipc_nsremote_NameServerRemoteNotify_Module__id__C)
                  0084eeb6    00000002     --HOLE-- [fill = 0]
                  0084eeb8    00000002     bench_shm_pe66.oe66 (.const:ti_sdo_ipc_transports_TransportShmNotify_alwaysWriteBackMsg__C)
                  0084eeba    00000002     --HOLE-- [fill = 0]
                  0084eebc    00000002     bench_shm_pe66.oe66 (.const:ti_sdo_ipc_transports_TransportShmNotify_notifyEventId__C)
                  0084eebe    00000002     --HOLE-- [fill = 0]
                  0084eec0    00000002     bench_shm_pe66.oe66 (.const:ti_sdo_utils_MultiProc_Module__id__C)
                  0084eec2    00000002     --HOLE-- [fill = 0]
                  0084eec4    00000002     bench_shm_pe66.oe66 (.const:ti_sdo_utils_MultiProc_numProcessors__C)
                  0084eec6    00000002     --HOLE-- [fill = 0]
                  0084eec8    00000002     bench_shm_pe66.oe66 (.const:ti_sdo_utils_MultiProc_numProcsInCluster__C)
                  0084eeca    00000002     --HOLE-- [fill = 0]
                  0084eecc    00000002     bench_shm_pe66.oe66 (.const:ti_sdo_utils_NameServer_Module__id__C)
                  0084eece    00000002     --HOLE-- [fill = 0]
                  0084eed0    00000002     bench_shm_pe66.oe66 (.const:ti_sdo_utils_NameServer_singleProcessor__C)
                  0084eed2    00000002     --HOLE-- [fill = 0]
                  0084eed4    00000002     bench_shm_pe66.oe66 (.const:ti_sysbios_BIOS_Module__id__C)
                  0084eed6    00000002     --HOLE-- [fill = 0]
                  0084eed8    00000002     bench_shm_pe66.oe66 (.const:ti_sysbios_family_c64p_Exception_Module__id__C)
                  0084eeda    00000002     --HOLE-- [fill = 0]
                  0084eedc    00000002     bench_shm_pe66.oe66 (.const:ti_sysbios_family_c64p_Hwi_Module__id__C)
                  0084eede    00000002     --HOLE-- [fill = 0]
                  0084eee0    00000002     bench_shm_pe66.oe66 (.const:ti_sysbios_family_c64p_Hwi_Module__loggerDefined__C)
                  0084eee2    00000002     --HOLE-- [fill = 0]
                  0084eee4    00000002     bench_shm_pe66.oe66 (.const:ti_sysbios_gates_GateMutexPri_Module__id__C)
                  0084eee6    00000002     --HOLE-- [fill = 0]
                  0084eee8    00000002     bench_shm_pe66.oe66 (.const:ti_sysbios_gates_GateMutex_Module__id__C)
                  0084eeea    00000002     --HOLE-- [fill = 0]
                  0084eeec    00000002     bench_shm_pe66.oe66 (.const:ti_sysbios_gates_GateSwi_Module__id__C)
                  0084eeee    00000002     --HOLE-- [fill = 0]
                  0084eef0    00000002     bench_shm_pe66.oe66 (.const:ti_sysbios_hal_Hwi_Module__id__C)
                  0084eef2    00000002     --HOLE-- [fill = 0]
                  0084eef4    00000002     bench_shm_pe66.oe66 (.const:ti_sysbios_heaps_HeapMem_Module__id__C)
                  0084eef6    00000002     --HOLE-- [fill = 0]
                  0084eef8    00000002     bench_shm_pe66.oe66 (.const:ti_sysbios_knl_Clock_Module__id__C)
                  0084eefa    00000002     --HOLE-- [fill = 0]
                  0084eefc    00000002     bench_shm_pe66.oe66 (.const:ti_sysbios_knl_Clock_Module__loggerDefined__C)
                  0084eefe    00000002     --HOLE-- [fill = 0]
                  0084ef00    00000002     bench_shm_pe66.oe66 (.const:ti_sysbios_knl_Semaphore_Module__id__C)
                  0084ef02    00000002     --HOLE-- [fill = 0]
                  0084ef04    00000002     bench_shm_pe66.oe66 (.const:ti_sysbios_knl_Semaphore_Module__loggerDefined__C)
                  0084ef06    00000002     --HOLE-- [fill = 0]
                  0084ef08    00000002     bench_shm_pe66.oe66 (.const:ti_sysbios_knl_Swi_Module__id__C)
                  0084ef0a    00000002     --HOLE-- [fill = 0]
                  0084ef0c    00000002     bench_shm_pe66.oe66 (.const:ti_sysbios_knl_Swi_Module__loggerDefined__C)
                  0084ef0e    00000002     --HOLE-- [fill = 0]
                  0084ef10    00000002     bench_shm_pe66.oe66 (.const:ti_sysbios_knl_Task_Module__id__C)
                  0084ef12    00000002     --HOLE-- [fill = 0]
                  0084ef14    00000002     bench_shm_pe66.oe66 (.const:ti_sysbios_knl_Task_Module__loggerDefined__C)
                  0084ef16    00000002     --HOLE-- [fill = 0]
                  0084ef18    00000002     bench_shm_pe66.oe66 (.const:ti_sysbios_knl_Task_deleteTerminatedTasks__C)
                  0084ef1a    00000002     --HOLE-- [fill = 0]
                  0084ef1c    00000002     bench_shm_pe66.oe66 (.const:ti_sysbios_knl_Task_initStackFlag__C)
                  0084ef1e    00000002     --HOLE-- [fill = 0]
                  0084ef20    00000002     bench_shm_pe66.oe66 (.const:ti_sysbios_syncs_SyncSem_Module__id__C)
                  0084ef22    00000002     --HOLE-- [fill = 0]
                  0084ef24    00000002     bench_shm_pe66.oe66 (.const:ti_sysbios_timers_timer64_Timer_Module__id__C)
                  0084ef26    00000002     --HOLE-- [fill = 0]
                  0084ef28    00000002     bench_shm_pe66.oe66 (.const:ti_sysbios_timers_timer64_Timer_startupNeeded__C)
                  0084ef2a    00000002     --HOLE-- [fill = 0]
                  0084ef2c    00000002     bench_shm_pe66.oe66 (.const:xdc_runtime_Core_Module__id__C)
                  0084ef2e    00000002     --HOLE-- [fill = 0]
                  0084ef30    00000002     bench_shm_pe66.oe66 (.const:xdc_runtime_Error_Module__loggerDefined__C)
                  0084ef32    00000002     --HOLE-- [fill = 0]
                  0084ef34    00000002     bench_shm_pe66.oe66 (.const:xdc_runtime_Error_maxDepth__C)
                  0084ef36    00000002     --HOLE-- [fill = 0]
                  0084ef38    00000002     bench_shm_pe66.oe66 (.const:xdc_runtime_Main_Module__id__C)
                  0084ef3a    00000002     --HOLE-- [fill = 0]
                  0084ef3c    00000002     bench_shm_pe66.oe66 (.const:xdc_runtime_Memory_Module__id__C)
                  0084ef3e    00000002     --HOLE-- [fill = 0]
                  0084ef40    00000002     bench_shm_pe66.oe66 (.const:xdc_runtime_Text_charCnt__C)
                  0084ef42    00000002     --HOLE-- [fill = 0]
                  0084ef44    00000002     bench_shm_pe66.oe66 (.const:xdc_runtime_Text_isLoaded__C)
                  0084ef46    00000002     --HOLE-- [fill = 0]
                  0084ef48    00000002     bench_shm_pe66.oe66 (.const:xdc_runtime_Text_registryModsLastId__C)
                  0084ef4a    00000002     --HOLE-- [fill = 0]
                  0084ef4c    00000002     bench_shm_pe66.oe66 (.const:xdc_runtime_Text_unnamedModsLastId__C)

.fardata.2 
*          0    0084ef50    0000153c     
                  0084ef50    00000800     bench_shm_pe66.oe66 (.fardata:ti_sdo_ipc_GateMP_Module_State_0_remoteCustom1Gates__A)
                  0084f750    00000308     bench_shm_pe66.oe66 (.fardata)
                  0084fa58    000001e0     rts6600_elf.lib : defs.obj (.fardata:_ftable)
                  0084fc38    000000c0     bench_shm_pe66.oe66 (.fardata:ti_sysbios_timers_timer64_Timer_Module_State_0_device__A)
                  0084fcf8    000000a8     bench_shm_pe66.oe66 (.fardata:ti_sdo_utils_NameServer_Object__table__V)
                  0084fda0    000000a0     rts6600_elf.lib : lowlev.obj (.fardata:_stream)
                  0084fe40    00000090     bench_shm_pe66.oe66 (.fardata:ti_sdo_ipc_SharedRegion_Module_State_0_regions__A)
                  0084fed0    00000088     rts6600_elf.lib : pow.obj (.fardata:A1$1)
                  0084ff58    00000088     bench_shm_pe66.oe66 (.fardata:ti_sysbios_knl_Task_Object__table__V)
                  0084ffe0    00000080     bench_shm_pe66.oe66 (.fardata:ti_sdo_ipc_GateMP_Module_State_0_remoteSystemGates__A)
                  00850060    00000080     bench_shm_pe66.oe66 (.fardata:ti_sysbios_knl_Swi_Module_State_0_readyQ__A)
                  008500e0    00000080     bench_shm_pe66.oe66 (.fardata:ti_sysbios_knl_Task_Module_State_0_readyQ__A)
                  00850160    00000078     rts6600_elf.lib : lowlev.obj (.fardata:_device)
                  008501d8    00000040                     : pow.obj (.fardata:A2$2)
                  00850218    00000040     bench_shm_pe66.oe66 (.fardata:ti_sysbios_gates_GateMutex_Object__table__V)
                  00850258    00000040     bench_shm_pe66.oe66 (.fardata:ti_sysbios_timers_timer64_Timer_Module_State_0_gctrl__A)
                  00850298    00000040     bench_shm_pe66.oe66 (.fardata:ti_sysbios_timers_timer64_Timer_Module_State_0_handles__A)
                  008502d8    00000040     bench_shm_pe66.oe66 (.fardata:ti_sysbios_timers_timer64_Timer_Module_State_0_intFreqs__A)
                  00850318    00000038     rts6600_elf.lib : pow.obj (.fardata:Q$4)
                  00850350    00000028     bench_shm_pe66.oe66 (.fardata:ti_sdo_ipc_Ipc_Module_State_0_procEntry__A)
                  00850378    00000020     rts6600_elf.lib : pow.obj (.fardata:P$3)
                  00850398    00000020     bench_shm_pe66.oe66 (.fardata:ti_sdo_ipc_MessageQ_Module_State_0_heaps__A)
                  008503b8    00000020     bench_shm_pe66.oe66 (.fardata:xdc_runtime_System_Module_State_0_atexitHandlers__A)
                  008503d8    00000018     bench_shm_pe66.oe66 (.fardata:ti_sysbios_gates_GateMutexPri_Object__table__V)
                  008503f0    00000014     bench_shm_pe66.oe66 (.fardata:ti_sysbios_heaps_HeapMem_Object__table__V)
                  00850404    00000004     rts6600_elf.lib : defs.obj (.fardata)
                  00850408    00000010     bench_shm_pe66.oe66 (.fardata:ti_sdo_ipc_MessageQ_Module_State_0_transports__A)
                  00850418    00000010     bench_shm_pe66.oe66 (.fardata:ti_sdo_ipc_family_c647x_Interrupt_Module_State_0_fxnTable__A)
                  00850428    00000010     bench_shm_pe66.oe66 (.fardata:ti_sysbios_gates_GateAll_Object__table__V)
                  00850438    0000000c     rts6600_elf.lib : exit.obj (.fardata)
                  00850444    00000004                     : dtor_list.obj (.fardata)
                  00850448    0000000c     bench_shm_pe66.oe66 (.fardata:ti_sysbios_gates_GateSwi_Object__table__V)
                  00850454    00000004     rts6600_elf.lib : errno.obj (.fardata)
                  00850458    00000008     bench_shm_pe66.oe66 (.fardata:ti_sdo_ipc_Notify_Module_State_0_notifyHandles__A)
                  00850460    00000008     bench_shm_pe66.oe66 (.fardata:ti_sdo_ipc_transports_TransportShmNotifySetup_Module_State_0_handles__A)
                  00850468    00000004     bench_shm_pe66.oe66 (.fardata:ti_sdo_ipc_GateMP_Module_State_0_remoteCustom2Gates__A)
                  0085046c    00000004     --HOLE--
                  00850470    00000004     bench_shm_pe66.oe66 (.fardata:ti_sdo_ipc_Notify_Module_State_0_notifyHandles_0__A)
                  00850474    00000004     --HOLE--
                  00850478    00000004     bench_shm_pe66.oe66 (.fardata:ti_sdo_ipc_Notify_Module_State_0_notifyHandles_1__A)
                  0085047c    00000004     --HOLE--
                  00850480    00000004     bench_shm_pe66.oe66 (.fardata:ti_sysbios_gates_GateHwi_Object__table__V)
                  00850484    00000004     --HOLE--
                  00850488    00000004     bench_shm_pe66.oe66 (.fardata:xdc_runtime_GateNull_Object__table__V)

.stack     0    00850490    00001000     UNINITIALIZED
                  00850490    00000008     boot.ae66 : boot.oe66 (.stack)
                  00850498    00000ff8     --HOLE--

platform_lib 
*          0    00851490    00000da0     
                  00851490    00000840     ti.platform.evm6657l.ae66 : evmc665x_nand.obj (platform_lib) [fill = 0]
                  00851cd0    00000458                               : platform.obj (platform_lib:uninit) [fill = 0]
                  00852128    00000108                               : platform.obj (platform_lib:init)

.cio       0    00852230    00000120     UNINITIALIZED
                  00852230    00000120     rts6600_elf.lib : trgmsg.obj (.cio)

.switch    0    00852350    00000080     
                  00852350    00000070     ti.csl.ae66 : csl_chip.oe66 (.switch:CSL_chipReadReg)
                  008523c0    00000010     ipc.lib : Ipc.obj (.switch:ti_sdo_ipc_GateMP_Instance_finalize__F)

.vecs      0    00852400    00000200     
                  00852400    00000200     bench_shm_pe66.oe66 (.vecs)

.bss       0    00852600    00000018     UNINITIALIZED
                  00852600    00000010     bench_shm.obj (.bss)
                  00852610    00000004     bench_shm_pe66.oe66 (.bss)
                  00852614    00000004     ti.platform.evm6657l.ae66 : evmc665x_spi.obj (.bss)

.neardata 
*          0    00852618    00000050     
                  00852618    00000024     bench_osal.obj (.neardata)
                  0085263c    00000004     --HOLE-- [fill = 0]
                  00852640    00000020     bench_shm.obj (.neardata)
                  00852660    00000008     ti.platform.evm6657l.ae66 : platform.obj (.neardata)

.rodata    0    00852668    00000000     UNINITIALIZED

.cinit     0    00852668    00000840     
                  00852668    0000072c     (.cinit..fardata.2.load) [load image, compression = rle]
                  00852d94    0000009b     (.cinit.platform_lib.load) [load image, compression = rle]
                  00852e2f    00000001     --HOLE-- [fill = 0]
                  00852e30    0000000e     (.cinit..fardata.1.load) [load image, compression = rle]
                  00852e3e    00000002     --HOLE-- [fill = 0]
                  00852e40    0000000c     (__TI_handler_table)
                  00852e4c    00000009     (.cinit..neardata.load) [load image, compression = rle]
                  00852e55    00000003     --HOLE-- [fill = 0]
                  00852e58    00000008     (.cinit..bss.load) [load image, compression = zero_init]
                  00852e60    00000008     (.cinit..far.load) [load image, compression = zero_init]
                  00852e68    00000008     (.cinit..msgQ_ptrs.load) [load image, compression = zero_init]
                  00852e70    00000038     (__TI_cinit_table)

ti.sdo.ipc.SharedRegion_0 
*          0    0c000000    00100000     NOLOAD SECTION
                  0c000000    00100000     --HOLE--


LINKER GENERATED COPY TABLES

__TI_cinit_table @ 00852e70 records: 7, size/record: 8, table size: 56
	.fardata.2: load addr=00852668, load size=0000072c bytes, run addr=0084ef50, run size=0000153c bytes, compression=rle
	platform_lib: load addr=00852d94, load size=0000009b bytes, run addr=00851490, run size=00000da0 bytes, compression=rle
	.fardata.1: load addr=00852e30, load size=0000000e bytes, run addr=0084a5c8, run size=00000008 bytes, compression=rle
	.neardata: load addr=00852e4c, load size=00000009 bytes, run addr=00852618, run size=00000050 bytes, compression=rle
	.bss: load addr=00852e58, load size=00000008 bytes, run addr=00852600, run size=00000018 bytes, compression=zero_init
	.far: load addr=00852e60, load size=00000008 bytes, run addr=00840fc0, run size=00009608 bytes, compression=zero_init
	.msgQ_ptrs: load addr=00852e68, load size=00000008 bytes, run addr=008315c0, run size=0000fa00 bytes, compression=zero_init


LINKER GENERATED HANDLER TABLE

__TI_handler_table @ 00852e40 records: 3, size/record: 4, table size: 12
	index: 0, handler: __TI_zero_init
	index: 1, handler: __TI_decompress_rle24
	index: 2, handler: __TI_decompress_none


GLOBAL SYMBOLS: SORTED ALPHABETICALLY BY Name 

address    name
--------   ----
0082f780   C$$EXIT
0082d3b8   C$$IO$$
00824cc0   CSL_chipReadReg
00801e30   Convert_CoreLocal2GlobalAddr
008030d4   CorePllcGetHwSetup
00802e88   CorePllcHwSetup
008033a0   DDR3Init
0082c820   GateMP_Params_init
00824e00   GateMP_close
0081fa00   GateMP_enter
0082f540   GateMP_getDefaultRemote
0081fc00   GateMP_leave
00819ba0   GateMP_openByAddr
00818ec0   GateMP_sharedMemReq
0082a3e0   HOSTclose
008268a0   HOSTlseek
00827ba0   HOSTopen
00828ee0   HOSTread
00821840   HOSTrename
00828fa0   HOSTunlink
00829060   HOSTwrite
0082c880   HeapMemMP_Params_init
00829120   HeapMemMP_create
00820f80   HeapMemMP_openByAddr
008187c0   HeapMemMP_sharedMemReq
00809220   Ipc_attach
0080a560   Ipc_detach
00852610   Ipc_sr0MemorySetup
0081b5a0   Ipc_start
00818b40   MessageQ_alloc
0082a480   MessageQ_create
008132e0   MessageQ_free
0081eb20   MessageQ_get
0081b2e0   MessageQ_open
0080c000   MessageQ_put
00824f40   MessageQ_registerHeap
0082f560   MultiProc_getBaseIdOfCluster
00822880   MultiProc_getName
0082f580   MultiProc_getNumProcessors
0082f5a0   MultiProc_self
00822a00   MultiProc_setLocalId
0080ebc0   NameServer_add
00813840   NameServer_get
00822b80   NameServer_getHandle
0081b840   NameServer_getLocal
008058f8   NandGetDetails
00804f70   NandReadSpareArea
00805330   NandWriteDataBytes
00805620   NandWriteSpareArea
00825080   Notify_attach
00822d00   Notify_intLineRegistered
0082c8e0   Notify_numIntLines
00810500   Notify_registerEventSingle
0080f8c0   Notify_sendEvent
00810ae0   Notify_unregisterEventSingle
0080b22c   Osal_cppiBeginMemAccess
0080b1e0   Osal_cppiCsEnter
0080b204   Osal_cppiCsExit
0080b26c   Osal_cppiEndMemAccess
0080b2e8   Osal_cppiFree
0080b2a8   Osal_cppiMalloc
0080b394   Osal_dataBufferInitMemory
0080b058   Osal_platformFree
0080b028   Osal_platformMalloc
0080b084   Osal_platformSpiCsEnter
0080b0a0   Osal_platformSpiCsExit
0080b0ac   Osal_qmssBeginMemAccess
0080b128   Osal_qmssCsEnter
0080b14c   Osal_qmssCsExit
0080b0ec   Osal_qmssEndMemAccess
0080b1a8   Osal_qmssFree
0080b16c   Osal_qmssMalloc
0080b714   Osal_srioBeginDescriptorAccess
0080b69c   Osal_srioBeginMemAccess
0080b5d0   Osal_srioCreateSem
0080b524   Osal_srioDataBufferFree
0080b460   Osal_srioDataBufferMalloc
0080b5e4   Osal_srioDeleteSem
0080b758   Osal_srioEndDescriptorAccess
0080b6d8   Osal_srioEndMemAccess
0080b610   Osal_srioEnterMultipleCoreCriticalSection
0080b654   Osal_srioEnterSingleCoreCriticalSection
0080b634   Osal_srioExitMultipleCoreCriticalSection
0080b678   Osal_srioExitSingleCoreCriticalSection
0080b360   Osal_srioFree
0080b5b8   Osal_srioLog
0080b324   Osal_srioMalloc
0080b5f0   Osal_srioPendSem
0080b604   Osal_srioPostSem
008031c0   PowerUpDomains
008031f0   SetDDR3PllConfig
008219e0   SharedRegion_getCacheLineSize
0081a1a0   SharedRegion_getEntry
00821b80   SharedRegion_getHeap
0081a480   SharedRegion_getPtr
0081c020   SharedRegion_getSRPtr
00821d20   SharedRegion_isCacheEnabled
0084ff9c   TSK_idle
0080de40   UartInit
0080e478   UartIsDataReady
0080e4b4   UartIsDataReady_B
0080e280   UartReadBaudRate
0080e2f0   UartReadBaudRate_B
0080e368   UartReadData
0080e394   UartReadData_B
0080e198   UartSetBaudRate
0080e210   UartSetBaudRate_B
0080e3c4   UartWriteData
0080e420   UartWriteData_B
00800000   __ASM__
00852230   __CIOBUF_
00800090   __ISA__
008000a8   __PLAT__
008000d0   __TARG__
00852e70   __TI_CINIT_Base
00852ea8   __TI_CINIT_Limit
00852e40   __TI_Handler_Table_Base
00852e4c   __TI_Handler_Table_Limit
UNDEFED    __TI_INITARRAY_Base
UNDEFED    __TI_INITARRAY_Limit
00851490   __TI_STACK_END
00001000   __TI_STACK_SIZE
00852600   __TI_STATIC_BASE
00000001   __TI_args_main
0082f7c0   __TI_decompress_none
0082f7e0   __TI_decompress_rle24
00850440   __TI_enable_exit_profile_output
ffffffff   __TI_pprof_out_hndl
ffffffff   __TI_prof_data_size
ffffffff   __TI_prof_data_start
00827f20   __TI_zero_init
008000f8   __TRDR__
ffffffff   __binit__
008110a0   __c6xabi_divd
0081c2a0   __c6xabi_divf
00829360   __c6xabi_divu
00821ec0   __c6xabi_divul
0081db60   __c6xabi_divull
0082f5c0   __c6xabi_errno_addr
0082b1a0   __c6xabi_fixdu
0082b220   __c6xabi_fixfu
0082a520   __c6xabi_fltulld
0082c940   __c6xabi_frcmpyd_div
0082d600   __c6xabi_isinf
0082b2a0   __c6xabi_llshl
0082c9a0   __c6xabi_llshru
0082f5e0   __c6xabi_negll
0082a5c0   __c6xabi_nround
0082a660   __c6xabi_remu
0082f600   __c6xabi_trunc
ffffffff   __c_args__
0082f620   __cxa_atexit
008292a0   __cxa_finalize
0082f640   __cxa_ia64_exit
00829360   __divu
00850454   __errno
0082a660   __remu
0082f660   __xdc__init
0084fa54   __xdc__init__addr
0082d680   _args_main
00000000   _argsize
008251c0   _auto_init_elf
0082a700   _c_int00
0082a7a0   _cleanup
00850438   _cleanup_ptr
008260c0   _closefile
0084db90   _ctypes_
00829420   _doflush
0085043c   _dtors_ptr
00850404   _ft_end
0084fa58   _ftable
0084a5c8   _lock
0082f680   _nop
00815640   _printfi
0082f700   _register_lock
0082f720   _register_unlock
00850490   _stack
0082ca00   _subcull
0084a348   _tmpnams
0084a5cc   _unlock
008269a0   _wrt_ok
0082f780   abort
00806b54   allocateMessages
0082f7a0   atexit
00827d60   atoi
0080696c   attachAll
ffffffff   binit
00807244   calculateThroughput
00827e40   close
00824294   configSerdes
00852628   cppiFreeCounter
00852624   cppiMallocCounter
00849ff8   cpuFreq
0085260c   cpuTimerFreqRatio
00806a6c   detachAll
00852228   emac_port_mode
00850454   errno
0082b520   evmI2CInit
008294e0   exit
00828000   fflush
00814d78   fpgaControlUserLEDs
00814f4c   fpgaDisableEepromWriteProtect
00814e38   fpgaDisableNandWriteProtect
00814ec4   fpgaDisableNorWriteProtect
00814f90   fpgaEnableEepromWriteProtect
00814e80   fpgaEnableNandWriteProtect
00814f08   fpgaEnableNorWriteProtect
00815020   fpgaGetAMCDetect
00814fd4   fpgaGetUserSwitch
00815110   fpgaReadConfigurationRegister
00815064   fpgaWriteConfigurationRegister
0081ef60   fputc
00818420   fputs
0082d780   free
00806bd0   freeMessages
00823000   frexp
00826300   fseek
0084a488   gDataBufferMemMgr
00852618   gDataBufferMemMgrMaxSize
008521b4   gDeviceEeprom0
008521ec   gDeviceEeprom1
00852144   gDeviceNand
00851d28   gDeviceNandBBlist
0085217c   gDeviceNor
0084a578   gI2cBlock
00814ce0   getBoardVersion
008071ec   getExecutionTime64
00814d2c   getFpgaDevID
008071c4   getStartTime64
008067a0   getStats
00806440   i2cEepromMacRead
008061a8   i2cEepromMacWrite
00805d2c   i2cEepromRead
00805f30   i2cEepromWrite
00805a64   i2cEepromWriteBlock
00806050   i2cEepromWriteByteAddr
00807764   initPlatform
0082d7c0   l2_global_address
0084a190   latencies
0084a320   latencyStats
00823f00   ldexp
00849fd8   localQueueName
0082ab60   lseek
008280e0   ltoa
00807b48   main
0082b3a0   malloc
0082ca60   memccpy
0082ac00   memcpy
008281c0   memset
00852650   messageQ
0082aca0   modf
00805738   nandFlashBlockErase
00805a00   nandInit
00852604   nextQueueId
00849fe0   nextQueueName
008146d4   nor_erase
00814360   nor_get_details
008143ec   nor_init
00814470   nor_read
00814500   nor_write
00852640   numCores
00801748   platform_blocknpage_to_offset
00800ca0   platform_delay
00800d00   platform_delaycycles
008011d0   platform_device_close
00801d6c   platform_device_erase_block
0080130c   platform_device_mark_block_bad
0080104c   platform_device_open
008014c0   platform_device_read
0080126c   platform_device_read_spare_data
00801840   platform_device_write
00801420   platform_device_write_spare_data
00852660   platform_errno
00800d40   platform_external_memory_test
00800c34   platform_fpgaReadConfigReg
00800c10   platform_fpgaWriteConfigReg
008009c4   platform_get_coreid
008009d0   platform_get_emac_info
00800af4   platform_get_emac_start_evt_id
008004a8   platform_get_info
00800a64   platform_get_macaddr
00800af8   platform_get_phy_addr
00800b18   platform_get_switch_state
008007b4   platform_init
00852664   platform_init_return_code
00800dc0   platform_internal_memory_test
00800c54   platform_led
00801620   platform_offset_to_blocknpage
00800b28   platform_phy_link_status
00800bf4   platform_uart_init
00800b38   platform_uart_read
00800bc0   platform_uart_set_baudrate
00800ba4   platform_uart_write
00800f28   platform_write
00800ef0   platform_write_configure
0080d740   pow
00852600   prevCoreId
00852608   prevQueueId
00849fe8   prevQueueName
00807360   printStatistics
008282a0   printf
00802d24   prog_pll1_values
0082f820   putc
0082f840   putchar
00852620   qmssFreeCounter
0085261c   qmssMallocCounter
0084a000   rawtimestamps
00805068   readNandPage
0082b420   readmsg
00807094   receiveMessages
0082c4a0   remove
008392c0   rxMsgPtrs
00852602   selfId
00806f28   sendMessages
00800390   serial_num_isvalid
00820400   setvbuf
00811c50   spi_claim
00811f48   spi_cmd
00811fc0   spi_cmd_read
00812020   spi_cmd_write
00812080   spi_read_word
00811df8   spi_release
0081212c   spi_write_word
00811e10   spi_xfer
00824060   sqrt
00852638   srioDataBufferFreeCounter
00852634   srioDataBufferMallocCounter
00852630   srioFreeCounter
0085262c   srioMallocCounter
0082d840   strlen
0082b4a0   strncpy
00806d88   syncReceiveCore
00806c34   syncSendCore
0084db8c   ti_sdo_ipc_GateMP_A_invalidClose__C
0084e8a4   ti_sdo_ipc_GateMP_A_invalidDelete__C
0084e924   ti_sdo_ipc_GateMP_E_gateUnavailable__C
0084e944   ti_sdo_ipc_GateMP_E_localGate__C
0080b7a0   ti_sdo_ipc_GateMP_Instance_finalize__F
008037a0   ti_sdo_ipc_GateMP_Instance_init__F
0084e974   ti_sdo_ipc_GateMP_LM_create__C
0084e97c   ti_sdo_ipc_GateMP_LM_delete__C
0084e980   ti_sdo_ipc_GateMP_LM_enter__C
0084e984   ti_sdo_ipc_GateMP_LM_leave__C
0084e988   ti_sdo_ipc_GateMP_LM_open__C
0084ef50   ti_sdo_ipc_GateMP_Module_State_0_remoteCustom1Gates__A
00850468   ti_sdo_ipc_GateMP_Module_State_0_remoteCustom2Gates__A
0084ffe0   ti_sdo_ipc_GateMP_Module_State_0_remoteSystemGates__A
0084e98c   ti_sdo_ipc_GateMP_Module__diagsEnabled__C
0084e990   ti_sdo_ipc_GateMP_Module__diagsIncluded__C
0084e994   ti_sdo_ipc_GateMP_Module__diagsMask__C
0084ee64   ti_sdo_ipc_GateMP_Module__id__C
0084ee68   ti_sdo_ipc_GateMP_Module__loggerDefined__C
0084e998   ti_sdo_ipc_GateMP_Module__loggerFxn2__C
0084e99c   ti_sdo_ipc_GateMP_Module__loggerFxn4__C
0084e9a0   ti_sdo_ipc_GateMP_Module__loggerObj__C
0084f750   ti_sdo_ipc_GateMP_Module__root__V
0084f758   ti_sdo_ipc_GateMP_Module__state__V
0084e3f0   ti_sdo_ipc_GateMP_Object__DESC__C
0084df48   ti_sdo_ipc_GateMP_Object__PARAMS__C
008295a0   ti_sdo_ipc_GateMP_Object__create__S
0082d880   ti_sdo_ipc_GateMP_Object__delete__S
0082d8c0   ti_sdo_ipc_GateMP_Params__init__S
0082d900   ti_sdo_ipc_GateMP_RemoteCustom1Proxy_Object__create__S
0082f860   ti_sdo_ipc_GateMP_RemoteCustom1Proxy_Object__delete__S
0082f880   ti_sdo_ipc_GateMP_RemoteCustom1Proxy_Params__init__S
0082f8a0   ti_sdo_ipc_GateMP_RemoteCustom1Proxy_Proxy__abstract__S
0082f8c0   ti_sdo_ipc_GateMP_RemoteCustom1Proxy_Proxy__delegate__S
0082f8e0   ti_sdo_ipc_GateMP_RemoteCustom1Proxy_getReservedMask__E
0082f900   ti_sdo_ipc_GateMP_RemoteCustom1Proxy_sharedMemReq__E
0082d940   ti_sdo_ipc_GateMP_RemoteCustom2Proxy_Object__create__S
0082f920   ti_sdo_ipc_GateMP_RemoteCustom2Proxy_Object__delete__S
0082f940   ti_sdo_ipc_GateMP_RemoteCustom2Proxy_Params__init__S
0082f960   ti_sdo_ipc_GateMP_RemoteCustom2Proxy_Proxy__abstract__S
0082f980   ti_sdo_ipc_GateMP_RemoteCustom2Proxy_Proxy__delegate__S
0082f9a0   ti_sdo_ipc_GateMP_RemoteCustom2Proxy_getReservedMask__E
0082f9c0   ti_sdo_ipc_GateMP_RemoteCustom2Proxy_sharedMemReq__E
0082d980   ti_sdo_ipc_GateMP_RemoteSystemProxy_Object__create__S
0082f9e0   ti_sdo_ipc_GateMP_RemoteSystemProxy_Object__delete__S
0082fa00   ti_sdo_ipc_GateMP_RemoteSystemProxy_Params__init__S
0082fa20   ti_sdo_ipc_GateMP_RemoteSystemProxy_Proxy__abstract__S
0082fa40   ti_sdo_ipc_GateMP_RemoteSystemProxy_Proxy__delegate__S
0082fa60   ti_sdo_ipc_GateMP_RemoteSystemProxy_getReservedMask__E
0082fa80   ti_sdo_ipc_GateMP_RemoteSystemProxy_sharedMemReq__E
0082faa0   ti_sdo_ipc_GateMP_attach__E
00820800   ti_sdo_ipc_GateMP_attach__F
00824320   ti_sdo_ipc_GateMP_createLocal__F
008209e0   ti_sdo_ipc_GateMP_getFreeResource__I
0082fac0   ti_sdo_ipc_GateMP_getRegion0ReservedSize__E
00829660   ti_sdo_ipc_GateMP_getRegion0ReservedSize__F
0082fae0   ti_sdo_ipc_GateMP_getSharedAddr__E
0082fb00   ti_sdo_ipc_GateMP_getSharedAddr__F
00822060   ti_sdo_ipc_GateMP_openRegion0Reserved__F
00815f00   ti_sdo_ipc_GateMP_setRegion0Reserved__F
0082fb20   ti_sdo_ipc_GateMP_start__E
00826ba0   ti_sdo_ipc_GateMP_start__F
0084e9a4   ti_sdo_ipc_Ipc_A_addrNotCacheAligned__C
0084e9a8   ti_sdo_ipc_Ipc_A_addrNotInSharedRegion__C
0084e9ac   ti_sdo_ipc_Ipc_A_internal__C
0084e9b0   ti_sdo_ipc_Ipc_A_invArgument__C
0084e9b4   ti_sdo_ipc_Ipc_A_invParam__C
0084e9b8   ti_sdo_ipc_Ipc_A_nullArgument__C
0084e9bc   ti_sdo_ipc_Ipc_E_internal__C
0084e9c0   ti_sdo_ipc_Ipc_E_nameFailed__C
0084e9c4   ti_sdo_ipc_Ipc_E_versionMismatch__C
00850350   ti_sdo_ipc_Ipc_Module_State_0_procEntry__A
0084e9c8   ti_sdo_ipc_Ipc_Module__diagsEnabled__C
0084e9cc   ti_sdo_ipc_Ipc_Module__diagsIncluded__C
0084e9d0   ti_sdo_ipc_Ipc_Module__diagsMask__C
0084ee6c   ti_sdo_ipc_Ipc_Module__id__C
0084f7a0   ti_sdo_ipc_Ipc_Module__state__V
0084ee70   ti_sdo_ipc_Ipc_generateSlaveDataForHost__C
0084e9d4   ti_sdo_ipc_Ipc_numUserFxns__C
00816360   ti_sdo_ipc_Ipc_procSyncFinish__I
00813da0   ti_sdo_ipc_Ipc_procSyncStart__I
0084e9d8   ti_sdo_ipc_Ipc_procSync__C
0084e9dc   ti_sdo_ipc_Ipc_userFxns__C
0084e9e0   ti_sdo_ipc_MessageQ_A_cannotFreeStaticMsg__C
0084e9e4   ti_sdo_ipc_MessageQ_A_heapIdInvalid__C
0084e9e8   ti_sdo_ipc_MessageQ_A_invalidMsg__C
0084e9ec   ti_sdo_ipc_MessageQ_A_invalidObj__C
0084e9f0   ti_sdo_ipc_MessageQ_A_invalidParam__C
0084e9f4   ti_sdo_ipc_MessageQ_A_invalidQueueId__C
0084e9f8   ti_sdo_ipc_MessageQ_A_procIdInvalid__C
0084e9fc   ti_sdo_ipc_MessageQ_A_unregisteredTransport__C
0084ea00   ti_sdo_ipc_MessageQ_E_maxReached__C
0084ea04   ti_sdo_ipc_MessageQ_E_nameFailed__C
0084ea08   ti_sdo_ipc_MessageQ_Instance_State_highList__O
0084ea0c   ti_sdo_ipc_MessageQ_Instance_State_normalList__O
0081e220   ti_sdo_ipc_MessageQ_Instance_finalize__F
008167c0   ti_sdo_ipc_MessageQ_Instance_init__F
0084ea10   ti_sdo_ipc_MessageQ_LM_alloc__C
0084ea14   ti_sdo_ipc_MessageQ_LM_free__C
0084ea18   ti_sdo_ipc_MessageQ_LM_get__C
0084ea1c   ti_sdo_ipc_MessageQ_LM_putLocal__C
00850398   ti_sdo_ipc_MessageQ_Module_State_0_heaps__A
00850408   ti_sdo_ipc_MessageQ_Module_State_0_transports__A
0084ea20   ti_sdo_ipc_MessageQ_Module__diagsEnabled__C
0084ea24   ti_sdo_ipc_MessageQ_Module__diagsIncluded__C
0084ea28   ti_sdo_ipc_MessageQ_Module__diagsMask__C
0084ee74   ti_sdo_ipc_MessageQ_Module__id__C
0084ee78   ti_sdo_ipc_MessageQ_Module__loggerDefined__C
0084ea2c   ti_sdo_ipc_MessageQ_Module__loggerFxn4__C
0084ea30   ti_sdo_ipc_MessageQ_Module__loggerObj__C
0084f7ac   ti_sdo_ipc_MessageQ_Module__root__V
0084f7b4   ti_sdo_ipc_MessageQ_Module__state__V
0082fb40   ti_sdo_ipc_MessageQ_Module_startup__E
00826540   ti_sdo_ipc_MessageQ_Module_startup__F
0084e410   ti_sdo_ipc_MessageQ_Object__DESC__C
0084e790   ti_sdo_ipc_MessageQ_Object__PARAMS__C
0084ea34   ti_sdo_ipc_MessageQ_Object__count__C
00829720   ti_sdo_ipc_MessageQ_Object__create__S
0082cac0   ti_sdo_ipc_MessageQ_Object__get__S
0084ea38   ti_sdo_ipc_MessageQ_Object__heap__C
0084ea3c   ti_sdo_ipc_MessageQ_Object__table__C
0082d9c0   ti_sdo_ipc_MessageQ_Params__init__S
0082fb60   ti_sdo_ipc_MessageQ_SetupTransportProxy_attach__E
0082fb80   ti_sdo_ipc_MessageQ_SetupTransportProxy_detach__E
0082fba0   ti_sdo_ipc_MessageQ_SetupTransportProxy_isRegistered__E
0082fbc0   ti_sdo_ipc_MessageQ_SetupTransportProxy_sharedMemReq__E
0084ea40   ti_sdo_ipc_MessageQ_maxRuntimeEntries__C
0082da00   ti_sdo_ipc_MessageQ_registerTransport__E
00823300   ti_sdo_ipc_MessageQ_registerTransport__F
0082fbe0   ti_sdo_ipc_MessageQ_unregisterTransport__E
00824480   ti_sdo_ipc_MessageQ_unregisterTransport__F
0084ea44   ti_sdo_ipc_Notify_A_alreadyRegistered__C
0084ea48   ti_sdo_ipc_Notify_A_internal__C
0084ea4c   ti_sdo_ipc_Notify_A_invArgument__C
0084ea50   ti_sdo_ipc_Notify_A_notRegistered__C
0084ea54   ti_sdo_ipc_Notify_A_reservedEvent__C
00826ca0   ti_sdo_ipc_Notify_Instance_finalize__F
008174a0   ti_sdo_ipc_Notify_Instance_init__F
0082fc00   ti_sdo_ipc_Notify_Module_GateProxy_enter__E
0082fc20   ti_sdo_ipc_Notify_Module_GateProxy_leave__E
00850470   ti_sdo_ipc_Notify_Module_State_0_notifyHandles_0__A
00850478   ti_sdo_ipc_Notify_Module_State_0_notifyHandles_1__A
00850458   ti_sdo_ipc_Notify_Module_State_0_notifyHandles__A
0084ea58   ti_sdo_ipc_Notify_Module__diagsEnabled__C
0084ea5c   ti_sdo_ipc_Notify_Module__diagsIncluded__C
0084ea60   ti_sdo_ipc_Notify_Module__diagsMask__C
0084ea64   ti_sdo_ipc_Notify_Module__gateObj__C
0084ee7c   ti_sdo_ipc_Notify_Module__id__C
0084f7d0   ti_sdo_ipc_Notify_Module__root__V
0084f7d8   ti_sdo_ipc_Notify_Module__state__V
0082fc40   ti_sdo_ipc_Notify_Module_startup__E
00823480   ti_sdo_ipc_Notify_Module_startup__F
0084e430   ti_sdo_ipc_Notify_Object__DESC__C
0084e7e4   ti_sdo_ipc_Notify_Object__PARAMS__C
00828380   ti_sdo_ipc_Notify_Object__create__S
0082da40   ti_sdo_ipc_Notify_Object__delete__S
0084ea68   ti_sdo_ipc_Notify_Object__heap__C
0082fc60   ti_sdo_ipc_Notify_SetupProxy_attach__E
0082fc80   ti_sdo_ipc_Notify_SetupProxy_numIntLines__E
0082fca0   ti_sdo_ipc_Notify_SetupProxy_sharedMemReq__E
0082fcc0   ti_sdo_ipc_Notify_detach__E
00828460   ti_sdo_ipc_Notify_detach__F
0082fce0   ti_sdo_ipc_Notify_exec__E
00825580   ti_sdo_ipc_Notify_exec__F
0084ea6c   ti_sdo_ipc_Notify_numEvents__C
0084ee80   ti_sdo_ipc_Notify_numLines__C
0084ee84   ti_sdo_ipc_Notify_reservedEvents__C
0084ea70   ti_sdo_ipc_SharedRegion_A_addrOutOfRange__C
0084ea74   ti_sdo_ipc_SharedRegion_A_idTooLarge__C
0084ea78   ti_sdo_ipc_SharedRegion_A_noHeap__C
0084ea7c   ti_sdo_ipc_SharedRegion_A_region0Invalid__C
0084ea80   ti_sdo_ipc_SharedRegion_A_regionInvalid__C
0084ea84   ti_sdo_ipc_SharedRegion_A_reserveTooMuch__C
0084ea88   ti_sdo_ipc_SharedRegion_INVALIDSRPTR__C
0084fe40   ti_sdo_ipc_SharedRegion_Module_State_0_regions__A
0084ea8c   ti_sdo_ipc_SharedRegion_Module__diagsEnabled__C
0084ea90   ti_sdo_ipc_SharedRegion_Module__diagsIncluded__C
0084ea94   ti_sdo_ipc_SharedRegion_Module__diagsMask__C
0084ee88   ti_sdo_ipc_SharedRegion_Module__id__C
0084f7e0   ti_sdo_ipc_SharedRegion_Module__state__V
0082fd00   ti_sdo_ipc_SharedRegion_attach__E
00826da0   ti_sdo_ipc_SharedRegion_attach__F
0084ea98   ti_sdo_ipc_SharedRegion_cacheLineSize__C
0082fd20   ti_sdo_ipc_SharedRegion_clearReservedMemory__E
00826ea0   ti_sdo_ipc_SharedRegion_clearReservedMemory__F
0084ee8c   ti_sdo_ipc_SharedRegion_numEntries__C
0084ea9c   ti_sdo_ipc_SharedRegion_numOffsetBits__C
0084eaa0   ti_sdo_ipc_SharedRegion_offsetMask__C
0082fd40   ti_sdo_ipc_SharedRegion_reserveMemory__E
00817ca0   ti_sdo_ipc_SharedRegion_reserveMemory__F
0082fd60   ti_sdo_ipc_SharedRegion_start__E
008121e0   ti_sdo_ipc_SharedRegion_start__F
0084ee90   ti_sdo_ipc_SharedRegion_translate__C
0084eaa4   ti_sdo_ipc_family_c647x_Interrupt_INTERDSPINT__C
0084eaa8   ti_sdo_ipc_family_c647x_Interrupt_IPCAR0__C
0084eaac   ti_sdo_ipc_family_c647x_Interrupt_IPCGR0__C
0084eab0   ti_sdo_ipc_family_c647x_Interrupt_KICK0__C
0084eab4   ti_sdo_ipc_family_c647x_Interrupt_KICK1__C
00850418   ti_sdo_ipc_family_c647x_Interrupt_Module_State_0_fxnTable__A
0084f7e4   ti_sdo_ipc_family_c647x_Interrupt_Module__state__V
0082fd80   ti_sdo_ipc_family_c647x_Interrupt_Module_startup__E
00826fa0   ti_sdo_ipc_family_c647x_Interrupt_Module_startup__F
0084ee94   ti_sdo_ipc_family_c647x_Interrupt_enableKick__C
0082da80   ti_sdo_ipc_family_c647x_Interrupt_intClear__E
0082fda0   ti_sdo_ipc_family_c647x_Interrupt_intDisable__E
0082fdc0   ti_sdo_ipc_family_c647x_Interrupt_intEnable__E
00826660   ti_sdo_ipc_family_c647x_Interrupt_intRegister__E
0082dac0   ti_sdo_ipc_family_c647x_Interrupt_intSend__E
008297e0   ti_sdo_ipc_family_c647x_Interrupt_intShmStub__I
0082ad40   ti_sdo_ipc_family_c647x_Interrupt_intUnregister__E
0084eab8   ti_sdo_ipc_family_c647x_MultiProcSetup_A_invalidProcessor__C
0084eabc   ti_sdo_ipc_family_c647x_MultiProcSetup_Module__diagsEnabled__C
0084eac0   ti_sdo_ipc_family_c647x_MultiProcSetup_Module__diagsIncluded__C
0084eac4   ti_sdo_ipc_family_c647x_MultiProcSetup_Module__diagsMask__C
0084ee98   ti_sdo_ipc_family_c647x_MultiProcSetup_Module__id__C
00820600   ti_sdo_ipc_family_c647x_MultiProcSetup_init__I
0084eac8   ti_sdo_ipc_family_c647x_MultiProcSetup_procMap__A
0084eacc   ti_sdo_ipc_family_c647x_MultiProcSetup_procMap__C
00828540   ti_sdo_ipc_family_c647x_NotifyCircSetup_attach__E
0084ead0   ti_sdo_ipc_family_c647x_NotifyCircSetup_dspIntVectId__C
0082fde0   ti_sdo_ipc_family_c647x_NotifyCircSetup_numIntLines__E
0082cb20   ti_sdo_ipc_family_c647x_NotifyCircSetup_sharedMemReq__E
0084ead4   ti_sdo_ipc_gates_GateHWSem_A_invSemNum__C
0082db00   ti_sdo_ipc_gates_GateHWSem_Handle__label__S
008245e0   ti_sdo_ipc_gates_GateHWSem_Instance_init__F
0084e03c   ti_sdo_ipc_gates_GateHWSem_Module__FXNS__C
0084ead8   ti_sdo_ipc_gates_GateHWSem_Module__diagsEnabled__C
0084eadc   ti_sdo_ipc_gates_GateHWSem_Module__diagsIncluded__C
0084eae0   ti_sdo_ipc_gates_GateHWSem_Module__diagsMask__C
0084ee9c   ti_sdo_ipc_gates_GateHWSem_Module__id__C
0084f7ec   ti_sdo_ipc_gates_GateHWSem_Module__root__V
0082fe00   ti_sdo_ipc_gates_GateHWSem_Module_startup__E
008270a0   ti_sdo_ipc_gates_GateHWSem_Module_startup__F
0084e450   ti_sdo_ipc_gates_GateHWSem_Object__DESC__C
0084e1d8   ti_sdo_ipc_gates_GateHWSem_Object__PARAMS__C
0082b5a0   ti_sdo_ipc_gates_GateHWSem_Object__create__S
0082db40   ti_sdo_ipc_gates_GateHWSem_Object__delete__S
0082db80   ti_sdo_ipc_gates_GateHWSem_Params__init__S
0084eae4   ti_sdo_ipc_gates_GateHWSem_baseAddr__C
00828620   ti_sdo_ipc_gates_GateHWSem_enter__E
0082fe20   ti_sdo_ipc_gates_GateHWSem_getReservedMask__E
0082cb80   ti_sdo_ipc_gates_GateHWSem_leave__E
0084eae8   ti_sdo_ipc_gates_GateHWSem_numSems__C
0082fe40   ti_sdo_ipc_gates_GateHWSem_query__E
0082fe60   ti_sdo_ipc_gates_GateHWSem_query__F
0084eaf0   ti_sdo_ipc_gates_GateHWSem_reservedMaskArr__A
0084eaec   ti_sdo_ipc_gates_GateHWSem_reservedMaskArr__C
0082fe80   ti_sdo_ipc_gates_GateHWSem_sharedMemReq__E
0084eaf4   ti_sdo_ipc_gates_GateMPSupportNull_A_invalidAction__C
0082dbc0   ti_sdo_ipc_gates_GateMPSupportNull_Handle__label__S
0082fea0   ti_sdo_ipc_gates_GateMPSupportNull_Instance_init__F
0084e068   ti_sdo_ipc_gates_GateMPSupportNull_Module__FXNS__C
0084eaf8   ti_sdo_ipc_gates_GateMPSupportNull_Module__diagsEnabled__C
0084eafc   ti_sdo_ipc_gates_GateMPSupportNull_Module__diagsIncluded__C
0084eb00   ti_sdo_ipc_gates_GateMPSupportNull_Module__diagsMask__C
0084eea0   ti_sdo_ipc_gates_GateMPSupportNull_Module__id__C
0084f7f4   ti_sdo_ipc_gates_GateMPSupportNull_Module__root__V
0084e470   ti_sdo_ipc_gates_GateMPSupportNull_Object__DESC__C
0084e1fc   ti_sdo_ipc_gates_GateMPSupportNull_Object__PARAMS__C
0082b620   ti_sdo_ipc_gates_GateMPSupportNull_Object__create__S
0082dc00   ti_sdo_ipc_gates_GateMPSupportNull_Object__delete__S
0082dc40   ti_sdo_ipc_gates_GateMPSupportNull_Params__init__S
0084eb04   ti_sdo_ipc_gates_GateMPSupportNull_action__C
008271a0   ti_sdo_ipc_gates_GateMPSupportNull_enter__E
0082fec0   ti_sdo_ipc_gates_GateMPSupportNull_getReservedMask__E
008272a0   ti_sdo_ipc_gates_GateMPSupportNull_leave__E
0082fee0   ti_sdo_ipc_gates_GateMPSupportNull_query__E
0082ff00   ti_sdo_ipc_gates_GateMPSupportNull_query__F
0082ff20   ti_sdo_ipc_gates_GateMPSupportNull_sharedMemReq__E
0084eb08   ti_sdo_ipc_gates_GatePeterson_E_gateRemotelyOpened__C
0082dc80   ti_sdo_ipc_gates_GatePeterson_Handle__label__S
0082cbe0   ti_sdo_ipc_gates_GatePeterson_Instance_finalize__F
008151a0   ti_sdo_ipc_gates_GatePeterson_Instance_init__F
0084e094   ti_sdo_ipc_gates_GatePeterson_Module__FXNS__C
0084eb0c   ti_sdo_ipc_gates_GatePeterson_Module__diagsEnabled__C
0084eb10   ti_sdo_ipc_gates_GatePeterson_Module__diagsIncluded__C
0084eb14   ti_sdo_ipc_gates_GatePeterson_Module__diagsMask__C
0084eea4   ti_sdo_ipc_gates_GatePeterson_Module__id__C
0084f7fc   ti_sdo_ipc_gates_GatePeterson_Module__root__V
0084e490   ti_sdo_ipc_gates_GatePeterson_Object__DESC__C
0084e220   ti_sdo_ipc_gates_GatePeterson_Object__PARAMS__C
008298a0   ti_sdo_ipc_gates_GatePeterson_Object__create__S
0082dcc0   ti_sdo_ipc_gates_GatePeterson_Object__delete__S
0082dd00   ti_sdo_ipc_gates_GatePeterson_Params__init__S
00823600   ti_sdo_ipc_gates_GatePeterson_enter__E
0082ff40   ti_sdo_ipc_gates_GatePeterson_getReservedMask__E
0082ade0   ti_sdo_ipc_gates_GatePeterson_leave__E
0084eb18   ti_sdo_ipc_gates_GatePeterson_numInstances__C
0082ff60   ti_sdo_ipc_gates_GatePeterson_query__E
0082ff80   ti_sdo_ipc_gates_GatePeterson_query__F
0082cc40   ti_sdo_ipc_gates_GatePeterson_sharedMemReq__E
0084eb1c   ti_sdo_ipc_heaps_HeapMemMP_A_align__C
0084eb20   ti_sdo_ipc_heaps_HeapMemMP_A_heapSize__C
0084eb24   ti_sdo_ipc_heaps_HeapMemMP_A_invalidFree__C
0084eb28   ti_sdo_ipc_heaps_HeapMemMP_A_zeroBlock__C
0084eb2c   ti_sdo_ipc_heaps_HeapMemMP_E_memory__C
0082dd40   ti_sdo_ipc_heaps_HeapMemMP_Handle__label__S
0081d6a0   ti_sdo_ipc_heaps_HeapMemMP_Instance_finalize__F
0080c840   ti_sdo_ipc_heaps_HeapMemMP_Instance_init__F
0084e110   ti_sdo_ipc_heaps_HeapMemMP_Module__FXNS__C
0084eb30   ti_sdo_ipc_heaps_HeapMemMP_Module__diagsEnabled__C
0084eb34   ti_sdo_ipc_heaps_HeapMemMP_Module__diagsIncluded__C
0084eb38   ti_sdo_ipc_heaps_HeapMemMP_Module__diagsMask__C
0084eea8   ti_sdo_ipc_heaps_HeapMemMP_Module__id__C
0084f804   ti_sdo_ipc_heaps_HeapMemMP_Module__root__V
0084f80c   ti_sdo_ipc_heaps_HeapMemMP_Module__state__V
0084e4b0   ti_sdo_ipc_heaps_HeapMemMP_Object__DESC__C
0084dfb0   ti_sdo_ipc_heaps_HeapMemMP_Object__PARAMS__C
00829960   ti_sdo_ipc_heaps_HeapMemMP_Object__create__S
0082dd80   ti_sdo_ipc_heaps_HeapMemMP_Object__delete__S
0082ddc0   ti_sdo_ipc_heaps_HeapMemMP_Params__init__S
00807de0   ti_sdo_ipc_heaps_HeapMemMP_alloc__E
00808840   ti_sdo_ipc_heaps_HeapMemMP_free__E
00816c20   ti_sdo_ipc_heaps_HeapMemMP_getStats__E
0082ffa0   ti_sdo_ipc_heaps_HeapMemMP_isBlocking__E
0082ffc0   ti_sdo_ipc_heaps_HeapMemMP_isBlocking__F
00817060   ti_sdo_ipc_heaps_HeapMemMP_postInit__I
0084eb3c   ti_sdo_ipc_interfaces_IGateMPSupport_Interface__BASE__C
0084eb40   ti_sdo_ipc_interfaces_IMessageQTransport_Interface__BASE__C
0084eb44   ti_sdo_ipc_interfaces_INotifyDriver_Interface__BASE__C
0084eb48   ti_sdo_ipc_notifyDrivers_NotifyDriverCirc_A_notSupported__C
0082de00   ti_sdo_ipc_notifyDrivers_NotifyDriverCirc_Handle__label__S
0082ae80   ti_sdo_ipc_notifyDrivers_NotifyDriverCirc_Instance_finalize__F
00814800   ti_sdo_ipc_notifyDrivers_NotifyDriverCirc_Instance_init__F
0082ffe0   ti_sdo_ipc_notifyDrivers_NotifyDriverCirc_InterruptProxy_intClear__E
00830000   ti_sdo_ipc_notifyDrivers_NotifyDriverCirc_InterruptProxy_intDisable__E
00830020   ti_sdo_ipc_notifyDrivers_NotifyDriverCirc_InterruptProxy_intEnable__E
0082de40   ti_sdo_ipc_notifyDrivers_NotifyDriverCirc_InterruptProxy_intRegister__E
00830040   ti_sdo_ipc_notifyDrivers_NotifyDriverCirc_InterruptProxy_intSend__E
00830060   ti_sdo_ipc_notifyDrivers_NotifyDriverCirc_InterruptProxy_intUnregister__E
0084df10   ti_sdo_ipc_notifyDrivers_NotifyDriverCirc_Module__FXNS__C
0084eb4c   ti_sdo_ipc_notifyDrivers_NotifyDriverCirc_Module__diagsEnabled__C
0084eb50   ti_sdo_ipc_notifyDrivers_NotifyDriverCirc_Module__diagsIncluded__C
0084eb54   ti_sdo_ipc_notifyDrivers_NotifyDriverCirc_Module__diagsMask__C
0084eeac   ti_sdo_ipc_notifyDrivers_NotifyDriverCirc_Module__id__C
0084f810   ti_sdo_ipc_notifyDrivers_NotifyDriverCirc_Module__root__V
0084e4d0   ti_sdo_ipc_notifyDrivers_NotifyDriverCirc_Object__DESC__C
0084df7c   ti_sdo_ipc_notifyDrivers_NotifyDriverCirc_Object__PARAMS__C
0082b6a0   ti_sdo_ipc_notifyDrivers_NotifyDriverCirc_Object__create__S
0082de80   ti_sdo_ipc_notifyDrivers_NotifyDriverCirc_Object__delete__S
0082dec0   ti_sdo_ipc_notifyDrivers_NotifyDriverCirc_Params__init__S
00828700   ti_sdo_ipc_notifyDrivers_NotifyDriverCirc_disableEvent__E
0082df00   ti_sdo_ipc_notifyDrivers_NotifyDriverCirc_disable__E
0082df40   ti_sdo_ipc_notifyDrivers_NotifyDriverCirc_enableEvent__E
0084eeb0   ti_sdo_ipc_notifyDrivers_NotifyDriverCirc_enableStats__C
008287e0   ti_sdo_ipc_notifyDrivers_NotifyDriverCirc_enable__E
0081aa40   ti_sdo_ipc_notifyDrivers_NotifyDriverCirc_isr__I
0084eb58   ti_sdo_ipc_notifyDrivers_NotifyDriverCirc_maxIndex__C
0084eb5c   ti_sdo_ipc_notifyDrivers_NotifyDriverCirc_modIndex__C
0084eb60   ti_sdo_ipc_notifyDrivers_NotifyDriverCirc_numMsgs__C
0082df80   ti_sdo_ipc_notifyDrivers_NotifyDriverCirc_registerEvent__E
0081e460   ti_sdo_ipc_notifyDrivers_NotifyDriverCirc_sendEvent__E
00830080   ti_sdo_ipc_notifyDrivers_NotifyDriverCirc_setNotifyHandle__E
008300a0   ti_sdo_ipc_notifyDrivers_NotifyDriverCirc_sharedMemReq__E
0081ca20   ti_sdo_ipc_notifyDrivers_NotifyDriverCirc_sharedMemReq__F
0082dfc0   ti_sdo_ipc_notifyDrivers_NotifyDriverCirc_unregisterEvent__E
0084eb64   ti_sdo_ipc_nsremote_NameServerRemoteNotify_A_invalidValueLen__C
0082e000   ti_sdo_ipc_nsremote_NameServerRemoteNotify_Handle__label__S
0084eb68   ti_sdo_ipc_nsremote_NameServerRemoteNotify_Instance_State_semMultiBlock__O
0084eb6c   ti_sdo_ipc_nsremote_NameServerRemoteNotify_Instance_State_semRemoteWait__O
0084eb70   ti_sdo_ipc_nsremote_NameServerRemoteNotify_Instance_State_swiObj__O
00826780   ti_sdo_ipc_nsremote_NameServerRemoteNotify_Instance_finalize__F
0080e500   ti_sdo_ipc_nsremote_NameServerRemoteNotify_Instance_init__F
0084e138   ti_sdo_ipc_nsremote_NameServerRemoteNotify_Module__FXNS__C
0084eb74   ti_sdo_ipc_nsremote_NameServerRemoteNotify_Module__diagsEnabled__C
0084eb78   ti_sdo_ipc_nsremote_NameServerRemoteNotify_Module__diagsIncluded__C
0084eb7c   ti_sdo_ipc_nsremote_NameServerRemoteNotify_Module__diagsMask__C
0084eeb4   ti_sdo_ipc_nsremote_NameServerRemoteNotify_Module__id__C
0084f818   ti_sdo_ipc_nsremote_NameServerRemoteNotify_Module__root__V
0084e4f0   ti_sdo_ipc_nsremote_NameServerRemoteNotify_Object__DESC__C
0084e510   ti_sdo_ipc_nsremote_NameServerRemoteNotify_Object__PARAMS__C
00829a20   ti_sdo_ipc_nsremote_NameServerRemoteNotify_Object__create__S
0082e040   ti_sdo_ipc_nsremote_NameServerRemoteNotify_Object__delete__S
0082e080   ti_sdo_ipc_nsremote_NameServerRemoteNotify_Object__first__S
0082e0c0   ti_sdo_ipc_nsremote_NameServerRemoteNotify_Object__next__S
0082e100   ti_sdo_ipc_nsremote_NameServerRemoteNotify_Params__init__S
00822200   ti_sdo_ipc_nsremote_NameServerRemoteNotify_attach__E
008300c0   ti_sdo_ipc_nsremote_NameServerRemoteNotify_cbFxn__I
0082b720   ti_sdo_ipc_nsremote_NameServerRemoteNotify_detach__E
0082e140   ti_sdo_ipc_nsremote_NameServerRemoteNotify_get__E
00812d60   ti_sdo_ipc_nsremote_NameServerRemoteNotify_get__F
0084eb80   ti_sdo_ipc_nsremote_NameServerRemoteNotify_notifyEventId__C
0082e180   ti_sdo_ipc_nsremote_NameServerRemoteNotify_sharedMemReq__E
00819200   ti_sdo_ipc_nsremote_NameServerRemoteNotify_swiFxn__I
0084eb84   ti_sdo_ipc_nsremote_NameServerRemoteNotify_timeout__C
00850460   ti_sdo_ipc_transports_TransportShmNotifySetup_Module_State_0_handles__A
0084f828   ti_sdo_ipc_transports_TransportShmNotifySetup_Module__state__V
00829ae0   ti_sdo_ipc_transports_TransportShmNotifySetup_attach__E
0082cca0   ti_sdo_ipc_transports_TransportShmNotifySetup_detach__E
008300e0   ti_sdo_ipc_transports_TransportShmNotifySetup_isRegistered__E
0084eb88   ti_sdo_ipc_transports_TransportShmNotifySetup_priority__C
00830100   ti_sdo_ipc_transports_TransportShmNotifySetup_sharedMemReq__E
0082e1c0   ti_sdo_ipc_transports_TransportShmNotify_Handle__label__S
0082b7a0   ti_sdo_ipc_transports_TransportShmNotify_Instance_finalize__F
008273a0   ti_sdo_ipc_transports_TransportShmNotify_Instance_init__F
0084e160   ti_sdo_ipc_transports_TransportShmNotify_Module__FXNS__C
0084f820   ti_sdo_ipc_transports_TransportShmNotify_Module__root__V
0084e530   ti_sdo_ipc_transports_TransportShmNotify_Object__DESC__C
0084e7ac   ti_sdo_ipc_transports_TransportShmNotify_Object__PARAMS__C
00829ba0   ti_sdo_ipc_transports_TransportShmNotify_Object__create__S
0082e200   ti_sdo_ipc_transports_TransportShmNotify_Object__delete__S
0082e240   ti_sdo_ipc_transports_TransportShmNotify_Params__init__S
0084eeb8   ti_sdo_ipc_transports_TransportShmNotify_alwaysWriteBackMsg__C
00830120   ti_sdo_ipc_transports_TransportShmNotify_control__E
00830140   ti_sdo_ipc_transports_TransportShmNotify_getStatus__E
0084eebc   ti_sdo_ipc_transports_TransportShmNotify_notifyEventId__C
0082cd00   ti_sdo_ipc_transports_TransportShmNotify_notifyFxn__I
008223a0   ti_sdo_ipc_transports_TransportShmNotify_put__E
00830160   ti_sdo_ipc_transports_TransportShmNotify_setErrFxn__E
00830180   ti_sdo_ipc_transports_TransportShmNotify_setErrFxn__F
0084eb8c   ti_sdo_utils_INameServerRemote_Interface__BASE__C
008301a0   ti_sdo_utils_List_Instance_init__F
0084f82c   ti_sdo_utils_List_Module__root__V
0084e550   ti_sdo_utils_List_Object__DESC__C
0084e7fc   ti_sdo_utils_List_Object__PARAMS__C
0084eb90   ti_sdo_utils_List_Object__count__C
0082b820   ti_sdo_utils_List_Object__create__S
0082e280   ti_sdo_utils_List_Object__destruct__S
0082cd60   ti_sdo_utils_List_Object__get__S
0084eb94   ti_sdo_utils_List_Object__table__C
0084eb98   ti_sdo_utils_MultiProc_A_invalidMultiProcId__C
0084eb9c   ti_sdo_utils_MultiProc_Module__diagsEnabled__C
0084eba0   ti_sdo_utils_MultiProc_Module__diagsIncluded__C
0084eba4   ti_sdo_utils_MultiProc_Module__diagsMask__C
0084eec0   ti_sdo_utils_MultiProc_Module__id__C
0084f834   ti_sdo_utils_MultiProc_Module__state__V
008301c0   ti_sdo_utils_MultiProc_getClusterId__E
008301e0   ti_sdo_utils_MultiProc_getClusterId__F
0084e948   ti_sdo_utils_MultiProc_nameList__A
0084eba8   ti_sdo_utils_MultiProc_nameList__C
0084eec4   ti_sdo_utils_MultiProc_numProcessors__C
0084eec8   ti_sdo_utils_MultiProc_numProcsInCluster__C
0084f848   ti_sdo_utils_NameServerRemoteNull_Module__root__V
0084ebac   ti_sdo_utils_NameServer_A_invArgument__C
0084ebb0   ti_sdo_utils_NameServer_A_invalidLen__C
0084ebb4   ti_sdo_utils_NameServer_E_entryExists__C
0084ebb8   ti_sdo_utils_NameServer_E_maxReached__C
0084ebbc   ti_sdo_utils_NameServer_Instance_State_freeList__O
0084ebc0   ti_sdo_utils_NameServer_Instance_State_nameList__O
00840fc0   ti_sdo_utils_NameServer_Module_State_0_nsRemoteHandle__A
0084ebc4   ti_sdo_utils_NameServer_Module__diagsEnabled__C
0084ebc8   ti_sdo_utils_NameServer_Module__diagsIncluded__C
0084ebcc   ti_sdo_utils_NameServer_Module__diagsMask__C
0084eecc   ti_sdo_utils_NameServer_Module__id__C
0084f838   ti_sdo_utils_NameServer_Module__root__V
0082e2c0   ti_sdo_utils_NameServer_Module__startupDone__F
00830200   ti_sdo_utils_NameServer_Module__startupDone__S
0084f840   ti_sdo_utils_NameServer_Module__state__V
00830220   ti_sdo_utils_NameServer_Module_startup__E
00823780   ti_sdo_utils_NameServer_Module_startup__F
0084ebd0   ti_sdo_utils_NameServer_Object__count__C
0082e300   ti_sdo_utils_NameServer_Object__first__S
0082cdc0   ti_sdo_utils_NameServer_Object__get__S
0082e340   ti_sdo_utils_NameServer_Object__next__S
0084ebd4   ti_sdo_utils_NameServer_Object__table__C
0084fcf8   ti_sdo_utils_NameServer_Object__table__V
00830240   ti_sdo_utils_NameServer_SetupProxy_attach__E
00830260   ti_sdo_utils_NameServer_SetupProxy_detach__E
00830280   ti_sdo_utils_NameServer_SetupProxy_sharedMemReq__E
00824740   ti_sdo_utils_NameServer_isRegistered__E
008248a0   ti_sdo_utils_NameServer_registerRemoteDriver__E
0084eed0   ti_sdo_utils_NameServer_singleProcessor__C
00824a00   ti_sdo_utils_NameServer_unregisterRemoteDriver__E
0084ebd8   ti_sysbios_BIOS_Module__diagsEnabled__C
0084ebdc   ti_sysbios_BIOS_Module__diagsIncluded__C
0084ebe0   ti_sysbios_BIOS_Module__diagsMask__C
0084eed4   ti_sysbios_BIOS_Module__id__C
0084f850   ti_sysbios_BIOS_Module__state__V
008302a0   ti_sysbios_BIOS_RtsGateProxy_enter__E
008302c0   ti_sysbios_BIOS_RtsGateProxy_leave__E
00829c60   ti_sysbios_BIOS_errorRaiseHook__I
0082ce20   ti_sysbios_BIOS_exitFunc__I
008302e0   ti_sysbios_BIOS_getCpuFreq__E
00830300   ti_sysbios_BIOS_getThreadType__E
0084ebe4   ti_sysbios_BIOS_installedErrorHook__C
0082ce80   ti_sysbios_BIOS_registerRTSLock__I
00830320   ti_sysbios_BIOS_setThreadType__E
0082e380   ti_sysbios_BIOS_startFunc__I
0082e3c0   ti_sysbios_BIOS_start__E
00830340   ti_sysbios_family_c62_TaskSupport_Module__startupDone__S
0082d700   ti_sysbios_family_c62_TaskSupport_buildTaskStack
00830360   ti_sysbios_family_c62_TaskSupport_checkStack__E
0082f740   ti_sysbios_family_c62_TaskSupport_glue
0082b8a0   ti_sysbios_family_c62_TaskSupport_start__E
0082b320   ti_sysbios_family_c62_TaskSupport_swap__E
0084ebe8   ti_sysbios_family_c64p_Exception_E_exceptionMin__C
0084eed8   ti_sysbios_family_c64p_Exception_Module__id__C
0084f86c   ti_sysbios_family_c64p_Exception_Module__state__V
00830380   ti_sysbios_family_c64p_Exception_Module_startup__E
0082b920   ti_sysbios_family_c64p_Exception_Module_startup__F
00823180   ti_sysbios_family_c64p_Exception_dispatch__E
0084ebec   ti_sysbios_family_c64p_Exception_exceptionHook__C
0084ebf0   ti_sysbios_family_c64p_Exception_externalHook__C
0080cfc0   ti_sysbios_family_c64p_Exception_handler__I
0081e6a0   ti_sysbios_family_c64p_Exception_internalHandler__I
0084ebf4   ti_sysbios_family_c64p_Exception_internalHook__C
0084ebf8   ti_sysbios_family_c64p_Exception_nmiHook__C
00852400   ti_sysbios_family_c64p_Hwi0
00852420   ti_sysbios_family_c64p_Hwi1
00852540   ti_sysbios_family_c64p_Hwi10
00852560   ti_sysbios_family_c64p_Hwi11
00852580   ti_sysbios_family_c64p_Hwi12
008525a0   ti_sysbios_family_c64p_Hwi13
008525c0   ti_sysbios_family_c64p_Hwi14
008525e0   ti_sysbios_family_c64p_Hwi15
00852440   ti_sysbios_family_c64p_Hwi2
00852460   ti_sysbios_family_c64p_Hwi3
00852480   ti_sysbios_family_c64p_Hwi4
008524a0   ti_sysbios_family_c64p_Hwi5
008524c0   ti_sysbios_family_c64p_Hwi6
008524e0   ti_sysbios_family_c64p_Hwi7
00852500   ti_sysbios_family_c64p_Hwi8
00852520   ti_sysbios_family_c64p_Hwi9
0084ebfc   ti_sysbios_family_c64p_Hwi_E_alreadyDefined__C
0084ec00   ti_sysbios_family_c64p_Hwi_E_handleNotFound__C
008288c0   ti_sysbios_family_c64p_Hwi_Instance_finalize__F
008289a0   ti_sysbios_family_c64p_Hwi_Instance_init__F
0084ec04   ti_sysbios_family_c64p_Hwi_LD_end__C
0084ec08   ti_sysbios_family_c64p_Hwi_LM_begin__C
0084ec0c   ti_sysbios_family_c64p_Hwi_Module__diagsEnabled__C
0084ec10   ti_sysbios_family_c64p_Hwi_Module__diagsIncluded__C
0084ec14   ti_sysbios_family_c64p_Hwi_Module__diagsMask__C
0084eedc   ti_sysbios_family_c64p_Hwi_Module__id__C
0084eee0   ti_sysbios_family_c64p_Hwi_Module__loggerDefined__C
0084ec18   ti_sysbios_family_c64p_Hwi_Module__loggerFxn1__C
0084ec1c   ti_sysbios_family_c64p_Hwi_Module__loggerFxn8__C
0084ec20   ti_sysbios_family_c64p_Hwi_Module__loggerObj__C
0084f898   ti_sysbios_family_c64p_Hwi_Module__root__V
0082e400   ti_sysbios_family_c64p_Hwi_Module__startupDone__F
008303a0   ti_sysbios_family_c64p_Hwi_Module__startupDone__S
0084f8a0   ti_sysbios_family_c64p_Hwi_Module__state__V
008303c0   ti_sysbios_family_c64p_Hwi_Module_startup__E
008256c0   ti_sysbios_family_c64p_Hwi_Module_startup__F
0084e570   ti_sysbios_family_c64p_Hwi_Object__DESC__C
0084dfe0   ti_sysbios_family_c64p_Hwi_Object__PARAMS__C
00828a80   ti_sysbios_family_c64p_Hwi_Object__create__S
0082e440   ti_sysbios_family_c64p_Hwi_Object__delete__S
0082e480   ti_sysbios_family_c64p_Hwi_Params__init__S
008303e0   ti_sysbios_family_c64p_Hwi_clearInterrupt__E
0082e4c0   ti_sysbios_family_c64p_Hwi_disableInterrupt__E
00820000   ti_sysbios_family_c64p_Hwi_dispatchAlways
00819ea0   ti_sysbios_family_c64p_Hwi_dispatchC__I
0082e500   ti_sysbios_family_c64p_Hwi_enableInterrupt__E
0082b9a0   ti_sysbios_family_c64p_Hwi_eventMap__E
00830400   ti_sysbios_family_c64p_Hwi_getHandle__E
0082aa20   ti_sysbios_family_c64p_Hwi_plug__E
0081f180   ti_sysbios_family_c64p_Hwi_reconfig__E
00830420   ti_sysbios_family_c64p_Hwi_startup__E
00830440   ti_sysbios_family_c64p_Hwi_switchFromBootStack__E
00830460   ti_sysbios_family_c64p_Hwi_unPluggedInterrupt__I
00830480   ti_sysbios_family_c64p_TimestampProvider_Module_startup__E
008304a0   ti_sysbios_family_c64p_TimestampProvider_Module_startup__F
008304c0   ti_sysbios_family_c64p_TimestampProvider_get32__E
008304e0   ti_sysbios_family_c64p_TimestampProvider_get64__E
008302e0   ti_sysbios_family_c64p_TimestampProvider_getFreq__E
00830500   ti_sysbios_family_c64p_tci6488_TimerSupport_enable__E
00830520   ti_sysbios_family_c66_Cache_Module_startup__E
00825800   ti_sysbios_family_c66_Cache_Module_startup__F
0084ec24   ti_sysbios_family_c66_Cache_atomicBlockSize__C
0084e938   ti_sysbios_family_c66_Cache_initSize__C
0082ba20   ti_sysbios_family_c66_Cache_invL1pAll__E
00830540   ti_sysbios_family_c66_Cache_inv__E
0084d618   ti_sysbios_family_c66_Cache_marvalues__C
0082e540   ti_sysbios_family_c66_Cache_wait__E
00830560   ti_sysbios_family_c66_Cache_wbInv__E
00830580   ti_sysbios_family_c66_Cache_wb__E
0082d740   ti_sysbios_family_xxx_Hwi_switchToIsrStack
0082f760   ti_sysbios_family_xxx_Hwi_switchToTaskStack
0082e580   ti_sysbios_gates_GateAll_Handle__label__S
008305a0   ti_sysbios_gates_GateAll_Instance_init__F
0084e244   ti_sysbios_gates_GateAll_Module__FXNS__C
0084f908   ti_sysbios_gates_GateAll_Module__root__V
0084e590   ti_sysbios_gates_GateAll_Object__DESC__C
0084e814   ti_sysbios_gates_GateAll_Object__PARAMS__C
0082baa0   ti_sysbios_gates_GateAll_Object__create__S
0082e5c0   ti_sysbios_gates_GateAll_Object__delete__S
00850428   ti_sysbios_gates_GateAll_Object__table__V
0082cee0   ti_sysbios_gates_GateAll_enter__E
00829d20   ti_sysbios_gates_GateAll_leave__E
008305c0   ti_sysbios_gates_GateAll_query__E
008305e0   ti_sysbios_gates_GateAll_query__F
0082e600   ti_sysbios_gates_GateHwi_Handle__label__S
00830600   ti_sysbios_gates_GateHwi_Instance_init__F
0084e268   ti_sysbios_gates_GateHwi_Module__FXNS__C
0084f910   ti_sysbios_gates_GateHwi_Module__root__V
0084e5b0   ti_sysbios_gates_GateHwi_Object__DESC__C
0084e82c   ti_sysbios_gates_GateHwi_Object__PARAMS__C
0082bb20   ti_sysbios_gates_GateHwi_Object__create__S
0082e640   ti_sysbios_gates_GateHwi_Object__delete__S
00850480   ti_sysbios_gates_GateHwi_Object__table__V
00830620   ti_sysbios_gates_GateHwi_enter__E
00830640   ti_sysbios_gates_GateHwi_leave__E
00830660   ti_sysbios_gates_GateHwi_query__E
00830680   ti_sysbios_gates_GateHwi_query__F
0084ec28   ti_sysbios_gates_GateMutexPri_A_badContext__C
0082e680   ti_sysbios_gates_GateMutexPri_Handle__label__S
0084ec2c   ti_sysbios_gates_GateMutexPri_Instance_State_pendQ__O
0082e6c0   ti_sysbios_gates_GateMutexPri_Instance_finalize__F
0082e700   ti_sysbios_gates_GateMutexPri_Instance_init__F
0084e28c   ti_sysbios_gates_GateMutexPri_Module__FXNS__C
0084ec30   ti_sysbios_gates_GateMutexPri_Module__diagsEnabled__C
0084ec34   ti_sysbios_gates_GateMutexPri_Module__diagsIncluded__C
0084ec38   ti_sysbios_gates_GateMutexPri_Module__diagsMask__C
0084eee4   ti_sysbios_gates_GateMutexPri_Module__id__C
0084f920   ti_sysbios_gates_GateMutexPri_Module__root__V
0084e5d0   ti_sysbios_gates_GateMutexPri_Object__DESC__C
0084e844   ti_sysbios_gates_GateMutexPri_Object__PARAMS__C
0082bba0   ti_sysbios_gates_GateMutexPri_Object__create__S
0082e740   ti_sysbios_gates_GateMutexPri_Object__delete__S
0082e780   ti_sysbios_gates_GateMutexPri_Object__destruct__S
008503d8   ti_sysbios_gates_GateMutexPri_Object__table__V
0081ad20   ti_sysbios_gates_GateMutexPri_enter__E
008274a0   ti_sysbios_gates_GateMutexPri_leave__E
008306a0   ti_sysbios_gates_GateMutexPri_query__E
008306c0   ti_sysbios_gates_GateMutexPri_query__F
0084ec3c   ti_sysbios_gates_GateMutex_A_badContext__C
0082e7c0   ti_sysbios_gates_GateMutex_Handle__label__S
0084ec40   ti_sysbios_gates_GateMutex_Instance_State_sem__O
0082e800   ti_sysbios_gates_GateMutex_Instance_finalize__F
0082cf40   ti_sysbios_gates_GateMutex_Instance_init__F
0084e2b0   ti_sysbios_gates_GateMutex_Module__FXNS__C
0084ec44   ti_sysbios_gates_GateMutex_Module__diagsEnabled__C
0084ec48   ti_sysbios_gates_GateMutex_Module__diagsIncluded__C
0084ec4c   ti_sysbios_gates_GateMutex_Module__diagsMask__C
0084eee8   ti_sysbios_gates_GateMutex_Module__id__C
0084f918   ti_sysbios_gates_GateMutex_Module__root__V
0084e5f0   ti_sysbios_gates_GateMutex_Object__DESC__C
0084e85c   ti_sysbios_gates_GateMutex_Object__PARAMS__C
0082bc20   ti_sysbios_gates_GateMutex_Object__create__S
0082e840   ti_sysbios_gates_GateMutex_Object__delete__S
00850218   ti_sysbios_gates_GateMutex_Object__table__V
00822540   ti_sysbios_gates_GateMutex_enter__E
0082e880   ti_sysbios_gates_GateMutex_leave__E
008306e0   ti_sysbios_gates_GateMutex_query__E
00830700   ti_sysbios_gates_GateMutex_query__F
0084ec50   ti_sysbios_gates_GateSwi_A_badContext__C
0082e8c0   ti_sysbios_gates_GateSwi_Handle__label__S
00830720   ti_sysbios_gates_GateSwi_Instance_init__F
0084e2d4   ti_sysbios_gates_GateSwi_Module__FXNS__C
0084ec54   ti_sysbios_gates_GateSwi_Module__diagsEnabled__C
0084ec58   ti_sysbios_gates_GateSwi_Module__diagsIncluded__C
0084ec5c   ti_sysbios_gates_GateSwi_Module__diagsMask__C
0084eeec   ti_sysbios_gates_GateSwi_Module__id__C
0084f928   ti_sysbios_gates_GateSwi_Module__root__V
0084e610   ti_sysbios_gates_GateSwi_Object__DESC__C
0084e874   ti_sysbios_gates_GateSwi_Object__PARAMS__C
0082bca0   ti_sysbios_gates_GateSwi_Object__create__S
0082e900   ti_sysbios_gates_GateSwi_Object__delete__S
00850448   ti_sysbios_gates_GateSwi_Object__table__V
00825940   ti_sysbios_gates_GateSwi_enter__E
0082bd20   ti_sysbios_gates_GateSwi_leave__E
00830740   ti_sysbios_gates_GateSwi_query__E
00830760   ti_sysbios_gates_GateSwi_query__F
0082e940   ti_sysbios_hal_Cache_CacheProxy_inv__E
00830780   ti_sysbios_hal_Cache_CacheProxy_wait__E
0082e980   ti_sysbios_hal_Cache_CacheProxy_wbInv__E
0082e9c0   ti_sysbios_hal_Cache_CacheProxy_wb__E
0082e940   ti_sysbios_hal_Cache_inv__E
00830780   ti_sysbios_hal_Cache_wait__E
0082e980   ti_sysbios_hal_Cache_wbInv__E
0082e9c0   ti_sysbios_hal_Cache_wb__E
0084ec60   ti_sysbios_hal_Hwi_E_stackOverflow__C
008307a0   ti_sysbios_hal_Hwi_HwiProxy_Module__startupDone__S
008307c0   ti_sysbios_hal_Hwi_HwiProxy_clearInterrupt__E
008307e0   ti_sysbios_hal_Hwi_HwiProxy_disableInterrupt__E
00830800   ti_sysbios_hal_Hwi_HwiProxy_enableInterrupt__E
00830820   ti_sysbios_hal_Hwi_HwiProxy_startup__E
00830840   ti_sysbios_hal_Hwi_HwiProxy_switchFromBootStack__E
0084eef0   ti_sysbios_hal_Hwi_Module__id__C
0084f930   ti_sysbios_hal_Hwi_Module__root__V
00830860   ti_sysbios_hal_Hwi_Module_startup__E
00830880   ti_sysbios_hal_Hwi_Module_startup__F
0082bda0   ti_sysbios_hal_Hwi_checkStack
008307c0   ti_sysbios_hal_Hwi_clearInterrupt__E
008307e0   ti_sysbios_hal_Hwi_disableInterrupt__E
00830800   ti_sysbios_hal_Hwi_enableInterrupt__E
0082cfa0   ti_sysbios_hal_Hwi_initStack
00830820   ti_sysbios_hal_Hwi_startup__E
00830840   ti_sysbios_hal_Hwi_switchFromBootStack__E
0084f938   ti_sysbios_hal_Timer_Module__root__V
0082ea00   ti_sysbios_hal_Timer_Module__startupDone__F
008308a0   ti_sysbios_hal_Timer_Module__startupDone__S
008308c0   ti_sysbios_hal_Timer_Module_startup__E
008308e0   ti_sysbios_hal_Timer_Module_startup__F
00830900   ti_sysbios_hal_Timer_TimerProxy_Module__startupDone__S
00830920   ti_sysbios_hal_Timer_TimerProxy_getExpiredCounts__E
00830940   ti_sysbios_hal_Timer_TimerProxy_getPeriod__E
00830960   ti_sysbios_hal_Timer_TimerProxy_setNextTick__E
00830980   ti_sysbios_hal_Timer_TimerProxy_startup__E
00830980   ti_sysbios_hal_Timer_startup__E
0084ec64   ti_sysbios_heaps_HeapMem_A_align__C
0084ec68   ti_sysbios_heaps_HeapMem_A_heapSize__C
0084ec6c   ti_sysbios_heaps_HeapMem_A_invalidFree__C
0084ec70   ti_sysbios_heaps_HeapMem_A_zeroBlock__C
0084ec74   ti_sysbios_heaps_HeapMem_E_memory__C
0082ea40   ti_sysbios_heaps_HeapMem_Handle__label__S
00840fc8   ti_sysbios_heaps_HeapMem_Instance_State_0_buf__A
00823900   ti_sysbios_heaps_HeapMem_Instance_init__F
008309a0   ti_sysbios_heaps_HeapMem_Module_GateProxy_enter__E
008309c0   ti_sysbios_heaps_HeapMem_Module_GateProxy_leave__E
008309e0   ti_sysbios_heaps_HeapMem_Module_GateProxy_query__E
0084e188   ti_sysbios_heaps_HeapMem_Module__FXNS__C
0084ec78   ti_sysbios_heaps_HeapMem_Module__diagsEnabled__C
0084ec7c   ti_sysbios_heaps_HeapMem_Module__diagsIncluded__C
0084ec80   ti_sysbios_heaps_HeapMem_Module__diagsMask__C
0084ec84   ti_sysbios_heaps_HeapMem_Module__gateObj__C
0084eef4   ti_sysbios_heaps_HeapMem_Module__id__C
0084f940   ti_sysbios_heaps_HeapMem_Module__root__V
0084e630   ti_sysbios_heaps_HeapMem_Object__DESC__C
0084e650   ti_sysbios_heaps_HeapMem_Object__PARAMS__C
0084ec88   ti_sysbios_heaps_HeapMem_Object__count__C
0082be20   ti_sysbios_heaps_HeapMem_Object__create__S
0082ea80   ti_sysbios_heaps_HeapMem_Object__delete__S
0082d000   ti_sysbios_heaps_HeapMem_Object__get__S
0084ec8c   ti_sysbios_heaps_HeapMem_Object__table__C
008503f0   ti_sysbios_heaps_HeapMem_Object__table__V
0080fee0   ti_sysbios_heaps_HeapMem_alloc__E
0080f260   ti_sysbios_heaps_HeapMem_free__E
00829de0   ti_sysbios_heaps_HeapMem_getStats__E
0082af20   ti_sysbios_heaps_HeapMem_init__I
00830a00   ti_sysbios_heaps_HeapMem_isBlocking__E
0084ec90   ti_sysbios_heaps_HeapMem_reqAlignMask__C
0084ec94   ti_sysbios_heaps_HeapMem_reqAlign__C
0084ec98   ti_sysbios_knl_Clock_A_badThreadType__C
00825a80   ti_sysbios_knl_Clock_Instance_finalize__F
0081cca0   ti_sysbios_knl_Clock_Instance_init__F
0084ec9c   ti_sysbios_knl_Clock_LM_begin__C
0084eca0   ti_sysbios_knl_Clock_LM_tick__C
0084eca4   ti_sysbios_knl_Clock_LW_delayed__C
0084eca8   ti_sysbios_knl_Clock_Module_State_clockQ__O
0084ecac   ti_sysbios_knl_Clock_Module__diagsEnabled__C
0084ecb0   ti_sysbios_knl_Clock_Module__diagsIncluded__C
0084ecb4   ti_sysbios_knl_Clock_Module__diagsMask__C
0084eef8   ti_sysbios_knl_Clock_Module__id__C
0084eefc   ti_sysbios_knl_Clock_Module__loggerDefined__C
0084ecb8   ti_sysbios_knl_Clock_Module__loggerFxn1__C
0084ecbc   ti_sysbios_knl_Clock_Module__loggerFxn2__C
0084ecc0   ti_sysbios_knl_Clock_Module__loggerObj__C
0084f948   ti_sysbios_knl_Clock_Module__root__V
0084f950   ti_sysbios_knl_Clock_Module__state__V
00830a40   ti_sysbios_knl_Clock_Module_startup__E
0082bea0   ti_sysbios_knl_Clock_Module_startup__F
0084e670   ti_sysbios_knl_Clock_Object__DESC__C
0084e2f8   ti_sysbios_knl_Clock_Object__PARAMS__C
0082bf20   ti_sysbios_knl_Clock_Object__create__S
0082eac0   ti_sysbios_knl_Clock_Object__destruct__S
0082eb00   ti_sysbios_knl_Clock_Params__init__S
0082d060   ti_sysbios_knl_Clock_doTick__I
0082bfa0   ti_sysbios_knl_Clock_getTicks__E
00829ea0   ti_sysbios_knl_Clock_logTick__E
008275a0   ti_sysbios_knl_Clock_startI__E
00828b60   ti_sysbios_knl_Clock_start__E
0084ecc4   ti_sysbios_knl_Clock_tickMode__C
0084ecc8   ti_sysbios_knl_Clock_tickPeriod__C
0084eccc   ti_sysbios_knl_Clock_tickSource__C
0081bd80   ti_sysbios_knl_Clock_workFunc__E
0084ecd0   ti_sysbios_knl_Idle_funcList__A
0084e950   ti_sysbios_knl_Idle_funcList__C
0082c020   ti_sysbios_knl_Idle_loop__E
00830a60   ti_sysbios_knl_Queue_Instance_init__F
0084f97c   ti_sysbios_knl_Queue_Module__root__V
0084e690   ti_sysbios_knl_Queue_Object__DESC__C
0084e88c   ti_sysbios_knl_Queue_Object__PARAMS__C
0084ecd4   ti_sysbios_knl_Queue_Object__count__C
0082c0a0   ti_sysbios_knl_Queue_Object__create__S
0082eb40   ti_sysbios_knl_Queue_Object__destruct__S
0082d0c0   ti_sysbios_knl_Queue_Object__get__S
0084ecd8   ti_sysbios_knl_Queue_Object__table__C
00830a80   ti_sysbios_knl_Queue_empty__E
0084ecdc   ti_sysbios_knl_Semaphore_A_badContext__C
0084ece0   ti_sysbios_knl_Semaphore_A_noEvents__C
0084ece4   ti_sysbios_knl_Semaphore_A_overflow__C
0084ece8   ti_sysbios_knl_Semaphore_Instance_State_pendQ__O
0082eb80   ti_sysbios_knl_Semaphore_Instance_finalize__F
00825bc0   ti_sysbios_knl_Semaphore_Instance_init__F
0084ecec   ti_sysbios_knl_Semaphore_LM_pend__C
0084ecf0   ti_sysbios_knl_Semaphore_LM_post__C
0084ecf4   ti_sysbios_knl_Semaphore_Module__diagsEnabled__C
0084ecf8   ti_sysbios_knl_Semaphore_Module__diagsIncluded__C
0084ecfc   ti_sysbios_knl_Semaphore_Module__diagsMask__C
0084ef00   ti_sysbios_knl_Semaphore_Module__id__C
0084ef04   ti_sysbios_knl_Semaphore_Module__loggerDefined__C
0084ed00   ti_sysbios_knl_Semaphore_Module__loggerFxn2__C
0084ed04   ti_sysbios_knl_Semaphore_Module__loggerFxn4__C
0084ed08   ti_sysbios_knl_Semaphore_Module__loggerObj__C
0084f984   ti_sysbios_knl_Semaphore_Module__root__V
0084e6b0   ti_sysbios_knl_Semaphore_Object__DESC__C
0084e31c   ti_sysbios_knl_Semaphore_Object__PARAMS__C
0082c120   ti_sysbios_knl_Semaphore_Object__create__S
0082ebc0   ti_sysbios_knl_Semaphore_Object__delete__S
0082ec00   ti_sysbios_knl_Semaphore_Object__destruct__S
0082ec40   ti_sysbios_knl_Semaphore_Params__init__S
0082c1a0   ti_sysbios_knl_Semaphore_pendTimeout__I
008178a0   ti_sysbios_knl_Semaphore_pend__E
0081e8e0   ti_sysbios_knl_Semaphore_post__E
0084ed0c   ti_sysbios_knl_Swi_A_badPriority__C
00829f60   ti_sysbios_knl_Swi_Instance_finalize__F
00821300   ti_sysbios_knl_Swi_Instance_init__F
0084ed10   ti_sysbios_knl_Swi_LD_end__C
0084ed14   ti_sysbios_knl_Swi_LM_begin__C
0084ed18   ti_sysbios_knl_Swi_LM_post__C
00850060   ti_sysbios_knl_Swi_Module_State_0_readyQ__A
0084ed1c   ti_sysbios_knl_Swi_Module__diagsEnabled__C
0084ed20   ti_sysbios_knl_Swi_Module__diagsIncluded__C
0084ed24   ti_sysbios_knl_Swi_Module__diagsMask__C
0084ef08   ti_sysbios_knl_Swi_Module__id__C
0084ef0c   ti_sysbios_knl_Swi_Module__loggerDefined__C
0084ed28   ti_sysbios_knl_Swi_Module__loggerFxn1__C
0084ed2c   ti_sysbios_knl_Swi_Module__loggerFxn4__C
0084ed30   ti_sysbios_knl_Swi_Module__loggerObj__C
0084f98c   ti_sysbios_knl_Swi_Module__root__V
0084f994   ti_sysbios_knl_Swi_Module__state__V
00830aa0   ti_sysbios_knl_Swi_Module_startup__E
0082d120   ti_sysbios_knl_Swi_Module_startup__F
0084e6d0   ti_sysbios_knl_Swi_Object__DESC__C
0084e1b0   ti_sysbios_knl_Swi_Object__PARAMS__C
0084ed34   ti_sysbios_knl_Swi_Object__count__C
0082a020   ti_sysbios_knl_Swi_Object__create__S
0082ec80   ti_sysbios_knl_Swi_Object__destruct__S
0082d180   ti_sysbios_knl_Swi_Object__get__S
0084ed38   ti_sysbios_knl_Swi_Object__table__C
0082ecc0   ti_sysbios_knl_Swi_Params__init__S
00830ac0   ti_sysbios_knl_Swi_disable__E
00825d00   ti_sysbios_knl_Swi_post__E
008276a0   ti_sysbios_knl_Swi_restoreHwi__E
0081f3a0   ti_sysbios_knl_Swi_run__I
00823a80   ti_sysbios_knl_Swi_schedule__I
0082c220   ti_sysbios_knl_Swi_startup__E
0084ed3c   ti_sysbios_knl_Task_A_badPriority__C
0084ed40   ti_sysbios_knl_Task_E_spOutOfBounds__C
0084ed44   ti_sysbios_knl_Task_E_stackOverflow__C
00848fc8   ti_sysbios_knl_Task_Instance_State_0_hookEnv__A
00848fd8   ti_sysbios_knl_Task_Instance_State_0_stack__A
00848fd0   ti_sysbios_knl_Task_Instance_State_1_hookEnv__A
008497d8   ti_sysbios_knl_Task_Instance_State_1_stack__A
0084ed48   ti_sysbios_knl_Task_LD_block__C
0084ed4c   ti_sysbios_knl_Task_LD_exit__C
0084ed50   ti_sysbios_knl_Task_LD_ready__C
0084ed54   ti_sysbios_knl_Task_LM_setPri__C
0084ed58   ti_sysbios_knl_Task_LM_switch__C
0084ed5c   ti_sysbios_knl_Task_LM_yield__C
008500e0   ti_sysbios_knl_Task_Module_State_0_readyQ__A
0084ed60   ti_sysbios_knl_Task_Module_State_inactiveQ__O
0084ed64   ti_sysbios_knl_Task_Module_State_terminatedQ__O
0084ed68   ti_sysbios_knl_Task_Module__diagsEnabled__C
0084ed6c   ti_sysbios_knl_Task_Module__diagsIncluded__C
0084ed70   ti_sysbios_knl_Task_Module__diagsMask__C
0084ef10   ti_sysbios_knl_Task_Module__id__C
0084ef14   ti_sysbios_knl_Task_Module__loggerDefined__C
0084ed74   ti_sysbios_knl_Task_Module__loggerFxn2__C
0084ed78   ti_sysbios_knl_Task_Module__loggerFxn4__C
0084ed7c   ti_sysbios_knl_Task_Module__loggerObj__C
0084f9b0   ti_sysbios_knl_Task_Module__root__V
0084f9b8   ti_sysbios_knl_Task_Module__state__V
00830ae0   ti_sysbios_knl_Task_Module_startup__E
0081b000   ti_sysbios_knl_Task_Module_startup__F
0084ed80   ti_sysbios_knl_Task_Object__count__C
0082ed00   ti_sysbios_knl_Task_Object__first__S
0082d1e0   ti_sysbios_knl_Task_Object__get__S
0082ed40   ti_sysbios_knl_Task_Object__next__S
0084ed84   ti_sysbios_knl_Task_Object__table__C
0084ff58   ti_sysbios_knl_Task_Object__table__V
00830b00   ti_sysbios_knl_Task_SupportProxy_Module__startupDone__S
00830b20   ti_sysbios_knl_Task_SupportProxy_checkStack__E
00830b40   ti_sysbios_knl_Task_SupportProxy_start__E
00830b60   ti_sysbios_knl_Task_SupportProxy_swap__E
0084ed88   ti_sysbios_knl_Task_allBlockedFunc__C
0082d240   ti_sysbios_knl_Task_allBlockedFunction__I
00825e40   ti_sysbios_knl_Task_blockI__E
008214c0   ti_sysbios_knl_Task_checkStacks__E
0084ef18   ti_sysbios_knl_Task_deleteTerminatedTasks__C
00830b80   ti_sysbios_knl_Task_disable__E
0082d2a0   ti_sysbios_knl_Task_enter__I
0081cf20   ti_sysbios_knl_Task_exit__E
00830ba0   ti_sysbios_knl_Task_getPri__E
0084e8a8   ti_sysbios_knl_Task_hooks__A
0084e958   ti_sysbios_knl_Task_hooks__C
0084ef1c   ti_sysbios_knl_Task_initStackFlag__C
0084ed8c   ti_sysbios_knl_Task_numConstructedTasks__C
0084ed90   ti_sysbios_knl_Task_numPriorities__C
00820bc0   ti_sysbios_knl_Task_postInit__I
0082c2a0   ti_sysbios_knl_Task_restore__E
0081f5c0   ti_sysbios_knl_Task_schedule__I
00830bc0   ti_sysbios_knl_Task_self__E
00818060   ti_sysbios_knl_Task_setPri__E
0081f7e0   ti_sysbios_knl_Task_startup__E
00823c00   ti_sysbios_knl_Task_unblockI__E
00825f80   ti_sysbios_knl_Task_yield__E
0082ed80   ti_sysbios_syncs_SyncSem_Handle__label__S
0082edc0   ti_sysbios_syncs_SyncSem_Instance_finalize__F
00824b60   ti_sysbios_syncs_SyncSem_Instance_init__F
0084e340   ti_sysbios_syncs_SyncSem_Module__FXNS__C
0084ed94   ti_sysbios_syncs_SyncSem_Module__diagsEnabled__C
0084ed98   ti_sysbios_syncs_SyncSem_Module__diagsIncluded__C
0084ed9c   ti_sysbios_syncs_SyncSem_Module__diagsMask__C
0084ef20   ti_sysbios_syncs_SyncSem_Module__id__C
0084f9ec   ti_sysbios_syncs_SyncSem_Module__root__V
0084e6f0   ti_sysbios_syncs_SyncSem_Object__DESC__C
0084e7c8   ti_sysbios_syncs_SyncSem_Object__PARAMS__C
0082a0e0   ti_sysbios_syncs_SyncSem_Object__create__S
0082ee00   ti_sysbios_syncs_SyncSem_Object__delete__S
00830be0   ti_sysbios_syncs_SyncSem_query__E
00830c00   ti_sysbios_syncs_SyncSem_query__F
00830c20   ti_sysbios_syncs_SyncSem_signal__E
00830c40   ti_sysbios_syncs_SyncSem_signal__F
00830c60   ti_sysbios_syncs_SyncSem_wait__E
0082afc0   ti_sysbios_syncs_SyncSem_wait__F
0084eda0   ti_sysbios_timers_timer64_Timer_A_notAvailable__C
0084eda4   ti_sysbios_timers_timer64_Timer_E_cannotSupport__C
0084fc38   ti_sysbios_timers_timer64_Timer_Module_State_0_device__A
00850258   ti_sysbios_timers_timer64_Timer_Module_State_0_gctrl__A
00850298   ti_sysbios_timers_timer64_Timer_Module_State_0_handles__A
008502d8   ti_sysbios_timers_timer64_Timer_Module_State_0_intFreqs__A
0084eda8   ti_sysbios_timers_timer64_Timer_Module__diagsEnabled__C
0084edac   ti_sysbios_timers_timer64_Timer_Module__diagsIncluded__C
0084edb0   ti_sysbios_timers_timer64_Timer_Module__diagsMask__C
0084ef24   ti_sysbios_timers_timer64_Timer_Module__id__C
0084f9f4   ti_sysbios_timers_timer64_Timer_Module__root__V
0082ee40   ti_sysbios_timers_timer64_Timer_Module__startupDone__F
00830c80   ti_sysbios_timers_timer64_Timer_Module__startupDone__S
0084f9fc   ti_sysbios_timers_timer64_Timer_Module__state__V
00830ca0   ti_sysbios_timers_timer64_Timer_Module_startup__E
008127a0   ti_sysbios_timers_timer64_Timer_Module_startup__F
00830cc0   ti_sysbios_timers_timer64_Timer_TimerSupportProxy_enable__E
0084edb4   ti_sysbios_timers_timer64_Timer_anyMask__C
0084edb8   ti_sysbios_timers_timer64_Timer_freqDivisor__C
0082c320   ti_sysbios_timers_timer64_Timer_getCount__E
0082c320   ti_sysbios_timers_timer64_Timer_getExpiredCounts__E
00820da0   ti_sysbios_timers_timer64_Timer_getFreq__E
0082c3a0   ti_sysbios_timers_timer64_Timer_getPeriod__E
0084edbc   ti_sysbios_timers_timer64_Timer_numLocalTimers__C
0084edc0   ti_sysbios_timers_timer64_Timer_numTimerDevices__C
00830ce0   ti_sysbios_timers_timer64_Timer_setNextTick__E
00821680   ti_sysbios_timers_timer64_Timer_setPeriodMicroSecs__E
008226e0   ti_sysbios_timers_timer64_Timer_start__E
0084ef28   ti_sysbios_timers_timer64_Timer_startupNeeded__C
00828c40   ti_sysbios_timers_timer64_Timer_startup__E
0082a1a0   ti_sysbios_timers_timer64_Timer_stop__E
008306a0   ti_sysbios_xdcruntime_GateProcessSupport_query__F
0084edc4   ti_sysbios_xdcruntime_GateThreadSupport_Instance_State_gate__O
0082ee80   ti_sysbios_xdcruntime_GateThreadSupport_Instance_finalize__F
0082eec0   ti_sysbios_xdcruntime_GateThreadSupport_Instance_init__F
0084fa10   ti_sysbios_xdcruntime_GateThreadSupport_Module__root__V
0084e710   ti_sysbios_xdcruntime_GateThreadSupport_Object__DESC__C
0084e8c0   ti_sysbios_xdcruntime_GateThreadSupport_Object__PARAMS__C
0082c420   ti_sysbios_xdcruntime_GateThreadSupport_Object__create__S
0082ef00   ti_sysbios_xdcruntime_GateThreadSupport_Object__delete__S
00830d00   ti_sysbios_xdcruntime_GateThreadSupport_enter__E
0082ef40   ti_sysbios_xdcruntime_GateThreadSupport_enter__F
00830d20   ti_sysbios_xdcruntime_GateThreadSupport_leave__E
0082ef80   ti_sysbios_xdcruntime_GateThreadSupport_leave__F
00830d40   ti_sysbios_xdcruntime_GateThreadSupport_query__E
008306a0   ti_sysbios_xdcruntime_GateThreadSupport_query__F
00852648   timeAdj
00852658   timeLength
00849ff0   timerFreq
00807ad0   tsk0
008315c0   txMsgPtrs
0082c4a0   unlink
0082d300   vsprintf
0082b060   write
00805394   writeNandPage
0082d360   writemsg
0084edc8   xdc_runtime_Assert_E_assertFailed__C
0082b100   xdc_runtime_Assert_raise__I
0084edcc   xdc_runtime_Core_A_initializedParams__C
0084edd0   xdc_runtime_Core_Module__diagsEnabled__C
0084edd4   xdc_runtime_Core_Module__diagsIncluded__C
0084edd8   xdc_runtime_Core_Module__diagsMask__C
0084ef2c   xdc_runtime_Core_Module__id__C
0082c520   xdc_runtime_Core_assignLabel__I
0082c5a0   xdc_runtime_Core_assignParams__I
0081d1a0   xdc_runtime_Core_createObject__I
008277a0   xdc_runtime_Core_deleteObject__I
0084eddc   xdc_runtime_Error_E_generic__C
0084ede0   xdc_runtime_Error_E_memory__C
0084ede4   xdc_runtime_Error_Module__diagsEnabled__C
0084ede8   xdc_runtime_Error_Module__diagsIncluded__C
0084edec   xdc_runtime_Error_Module__diagsMask__C
0084ef30   xdc_runtime_Error_Module__loggerDefined__C
0084edf0   xdc_runtime_Error_Module__loggerFxn8__C
0084edf4   xdc_runtime_Error_Module__loggerObj__C
0084fa18   xdc_runtime_Error_Module__state__V
00830d80   xdc_runtime_Error_check__E
0082efc0   xdc_runtime_Error_check__F
00830da0   xdc_runtime_Error_init__E
0082f000   xdc_runtime_Error_init__F
0084ef34   xdc_runtime_Error_maxDepth__C
0084edf8   xdc_runtime_Error_policy__C
00830dc0   xdc_runtime_Error_print__E
00828d20   xdc_runtime_Error_print__F
0084edfc   xdc_runtime_Error_raiseHook__C
0082f040   xdc_runtime_Error_raiseX__E
0081d420   xdc_runtime_Error_raiseX__F
0082f080   xdc_runtime_GateNull_Handle__label__S
0084e364   xdc_runtime_GateNull_Module__FXNS__C
0084fa1c   xdc_runtime_GateNull_Module__root__V
0084e730   xdc_runtime_GateNull_Object__DESC__C
0084e8d8   xdc_runtime_GateNull_Object__PARAMS__C
0082d3c0   xdc_runtime_GateNull_Object__create__S
0082f0c0   xdc_runtime_GateNull_Object__delete__S
00850488   xdc_runtime_GateNull_Object__table__V
00830de0   xdc_runtime_GateNull_enter__E
00830e00   xdc_runtime_GateNull_enter__F
00830e20   xdc_runtime_GateNull_leave__E
00830e40   xdc_runtime_GateNull_leave__F
00830e60   xdc_runtime_GateNull_query__E
00830e80   xdc_runtime_GateNull_query__F
00830ea0   xdc_runtime_Gate_enterSystem__E
00830ec0   xdc_runtime_Gate_enterSystem__F
00830ee0   xdc_runtime_Gate_leaveSystem__E
0082f100   xdc_runtime_Gate_leaveSystem__F
0084ee00   xdc_runtime_IGateProvider_Interface__BASE__C
0084ee04   xdc_runtime_IHeap_Interface__BASE__C
0084ee08   xdc_runtime_IModule_Interface__BASE__C
0084ee0c   xdc_runtime_Log_L_error__C
0084ee10   xdc_runtime_Main_Module__diagsEnabled__C
0084ee14   xdc_runtime_Main_Module__diagsIncluded__C
0084ee18   xdc_runtime_Main_Module__diagsMask__C
0084ef38   xdc_runtime_Main_Module__id__C
00830f00   xdc_runtime_Memory_HeapProxy_alloc__E
00830f20   xdc_runtime_Memory_HeapProxy_free__E
0084ef3c   xdc_runtime_Memory_Module__id__C
0084fa24   xdc_runtime_Memory_Module__state__V
00830f40   xdc_runtime_Memory_alloc__E
00828e00   xdc_runtime_Memory_alloc__F
00830f60   xdc_runtime_Memory_calloc__E
0082d420   xdc_runtime_Memory_calloc__F
0084ee1c   xdc_runtime_Memory_defaultHeapInstance__C
00830f80   xdc_runtime_Memory_free__E
0082f1c0   xdc_runtime_Memory_free__F
00830fa0   xdc_runtime_Memory_getMaxDefaultTypeAlign__E
00830fc0   xdc_runtime_Memory_getMaxDefaultTypeAlign__F
0084fa28   xdc_runtime_Registry_Module__state__V
00830fe0   xdc_runtime_Registry_findById__E
0082f200   xdc_runtime_Registry_findById__F
00831000   xdc_runtime_Startup_Module__startupDone__S
0084fa30   xdc_runtime_Startup_Module__state__V
00000001   xdc_runtime_Startup__EXECFXN__C
00000001   xdc_runtime_Startup__RESETFXN__C
0084ee20   xdc_runtime_Startup_execImpl__C
00831020   xdc_runtime_Startup_exec__E
008278a0   xdc_runtime_Startup_exec__F
0082f240   xdc_runtime_Startup_exec__I
0084e928   xdc_runtime_Startup_firstFxns__A
0084e960   xdc_runtime_Startup_firstFxns__C
0084ee28   xdc_runtime_Startup_lastFxns__A
0084e968   xdc_runtime_Startup_lastFxns__C
0084ee24   xdc_runtime_Startup_maxPasses__C
00831040   xdc_runtime_Startup_reset__I
00831060   xdc_runtime_Startup_rtsDone__E
00831080   xdc_runtime_Startup_rtsDone__F
0084e750   xdc_runtime_Startup_sfxnRts__A
0084ee2c   xdc_runtime_Startup_sfxnRts__C
0084ded0   xdc_runtime_Startup_sfxnTab__A
0084ee30   xdc_runtime_Startup_sfxnTab__C
0084ee34   xdc_runtime_Startup_startModsFxn__C
0081d900   xdc_runtime_Startup_startMods__I
008310a0   xdc_runtime_SysStd_abort__E
0082d480   xdc_runtime_SysStd_abort__F
008310c0   xdc_runtime_SysStd_exit__E
008310e0   xdc_runtime_SysStd_exit__F
00831100   xdc_runtime_SysStd_putch__E
00831120   xdc_runtime_SysStd_putch__F
00831140   xdc_runtime_SysStd_ready__E
00831160   xdc_runtime_SysStd_ready__F
0084ee38   xdc_runtime_System_A_cannotFitIntoArg__C
00831180   xdc_runtime_System_Module_GateProxy_enter__E
008311a0   xdc_runtime_System_Module_GateProxy_leave__E
008503b8   xdc_runtime_System_Module_State_0_atexitHandlers__A
0084ee3c   xdc_runtime_System_Module__gateObj__C
0084fa38   xdc_runtime_System_Module__state__V
008311c0   xdc_runtime_System_Module_startup__E
008311e0   xdc_runtime_System_Module_startup__F
00831200   xdc_runtime_System_SupportProxy_abort__E
00831220   xdc_runtime_System_SupportProxy_exit__E
00831240   xdc_runtime_System_SupportProxy_putch__E
00831260   xdc_runtime_System_SupportProxy_ready__E
00831280   xdc_runtime_System_abort__E
0082f280   xdc_runtime_System_abort__F
0082f2c0   xdc_runtime_System_aprintf__E
0082d4e0   xdc_runtime_System_aprintf_va__F
008312a0   xdc_runtime_System_atexit__E
0082c620   xdc_runtime_System_atexit__F
0082d4e0   xdc_runtime_System_avprintf__F
00809bc0   xdc_runtime_System_doPrint__I
008312c0   xdc_runtime_System_exit__E
008312e0   xdc_runtime_System_exit__F
0084ee40   xdc_runtime_System_extendFxn__C
0082a260   xdc_runtime_System_formatNum__I
00831300   xdc_runtime_System_lastFxn__I
0084ee44   xdc_runtime_System_maxAtexitHandlers__C
00819540   xdc_runtime_System_printfExtend__I
0082f300   xdc_runtime_System_printf__E
0082d540   xdc_runtime_System_printf_va__F
0082c6a0   xdc_runtime_System_rtsExit__I
0082f340   xdc_runtime_System_sprintf__E
00831340   xdc_runtime_System_sprintf_va__F
0082d540   xdc_runtime_System_vprintf__F
00831320   xdc_runtime_System_vsprintf__E
00831340   xdc_runtime_System_vsprintf__F
0084fa44   xdc_runtime_Text_Module__state__V
0084ef40   xdc_runtime_Text_charCnt__C
0084a5d0   xdc_runtime_Text_charTab__A
0084ee48   xdc_runtime_Text_charTab__C
00831360   xdc_runtime_Text_cordText__E
0082d5a0   xdc_runtime_Text_cordText__F
0084ef44   xdc_runtime_Text_isLoaded__C
0084ee4c   xdc_runtime_Text_nameEmpty__C
0084ee50   xdc_runtime_Text_nameStatic__C
0084ee54   xdc_runtime_Text_nameUnknown__C
0084da18   xdc_runtime_Text_nodeTab__A
0084ee58   xdc_runtime_Text_nodeTab__C
0082c720   xdc_runtime_Text_printVisFxn__I
008279a0   xdc_runtime_Text_putMod__F
00831380   xdc_runtime_Text_putSite__E
00823d80   xdc_runtime_Text_putSite__F
0084ef48   xdc_runtime_Text_registryModsLastId__C
008313a0   xdc_runtime_Text_ropeText__E
0082f380   xdc_runtime_Text_ropeText__F
0084ef4c   xdc_runtime_Text_unnamedModsLastId__C
00827aa0   xdc_runtime_Text_visitRope2__I
0084ee5c   xdc_runtime_Text_visitRopeFxn__C
0082f3c0   xdc_runtime_Text_visitRope__I
0082c7a0   xdc_runtime_Text_xprintf__I
008313c0   xdc_runtime_Timestamp_SupportProxy_get32__E
008313e0   xdc_runtime_Timestamp_SupportProxy_get64__E
00831400   xdc_runtime_Timestamp_SupportProxy_getFreq__E
00831420   xdc_runtime_Timestamp_get32__E
008313c0   xdc_runtime_Timestamp_get32__F
00831440   xdc_runtime_Timestamp_get64__E
008313e0   xdc_runtime_Timestamp_get64__F
00831460   xdc_runtime_Timestamp_getFreq__E
00831400   xdc_runtime_Timestamp_getFreq__F
0082f400   xdc_runtime_knl_GateThread_Handle__label__S
0082f440   xdc_runtime_knl_GateThread_Instance_finalize__F
0082f480   xdc_runtime_knl_GateThread_Instance_init__F
0084e388   xdc_runtime_knl_GateThread_Module__FXNS__C
0084fa4c   xdc_runtime_knl_GateThread_Module__root__V
00831480   xdc_runtime_knl_GateThread_Module__startupDone__S
0084e770   xdc_runtime_knl_GateThread_Object__DESC__C
0084e8f0   xdc_runtime_knl_GateThread_Object__PARAMS__C
0082a320   xdc_runtime_knl_GateThread_Object__create__S
0082f4c0   xdc_runtime_knl_GateThread_Object__delete__S
0082f500   xdc_runtime_knl_GateThread_Proxy_Object__create__S
008314a0   xdc_runtime_knl_GateThread_Proxy_Object__delete__S
008314c0   xdc_runtime_knl_GateThread_Proxy_enter__E
008314e0   xdc_runtime_knl_GateThread_Proxy_leave__E
00831500   xdc_runtime_knl_GateThread_Proxy_query__E
00831520   xdc_runtime_knl_GateThread_enter__E
00831540   xdc_runtime_knl_GateThread_enter__F
00831560   xdc_runtime_knl_GateThread_leave__E
00831580   xdc_runtime_knl_GateThread_leave__F
008315a0   xdc_runtime_knl_GateThread_query__E
00831500   xdc_runtime_knl_GateThread_query__F
0084ee60   xdc_runtime_knl_ISync_Interface__BASE__C
00803354   xmc_setup


GLOBAL SYMBOLS: SORTED BY Symbol Address 

address    name
--------   ----
00000000   _argsize
00000001   __TI_args_main
00000001   xdc_runtime_Startup__EXECFXN__C
00000001   xdc_runtime_Startup__RESETFXN__C
00001000   __TI_STACK_SIZE
00800000   __ASM__
00800090   __ISA__
008000a8   __PLAT__
008000d0   __TARG__
008000f8   __TRDR__
00800390   serial_num_isvalid
008004a8   platform_get_info
008007b4   platform_init
008009c4   platform_get_coreid
008009d0   platform_get_emac_info
00800a64   platform_get_macaddr
00800af4   platform_get_emac_start_evt_id
00800af8   platform_get_phy_addr
00800b18   platform_get_switch_state
00800b28   platform_phy_link_status
00800b38   platform_uart_read
00800ba4   platform_uart_write
00800bc0   platform_uart_set_baudrate
00800bf4   platform_uart_init
00800c10   platform_fpgaWriteConfigReg
00800c34   platform_fpgaReadConfigReg
00800c54   platform_led
00800ca0   platform_delay
00800d00   platform_delaycycles
00800d40   platform_external_memory_test
00800dc0   platform_internal_memory_test
00800ef0   platform_write_configure
00800f28   platform_write
0080104c   platform_device_open
008011d0   platform_device_close
0080126c   platform_device_read_spare_data
0080130c   platform_device_mark_block_bad
00801420   platform_device_write_spare_data
008014c0   platform_device_read
00801620   platform_offset_to_blocknpage
00801748   platform_blocknpage_to_offset
00801840   platform_device_write
00801d6c   platform_device_erase_block
00801e30   Convert_CoreLocal2GlobalAddr
00802d24   prog_pll1_values
00802e88   CorePllcHwSetup
008030d4   CorePllcGetHwSetup
008031c0   PowerUpDomains
008031f0   SetDDR3PllConfig
00803354   xmc_setup
008033a0   DDR3Init
008037a0   ti_sdo_ipc_GateMP_Instance_init__F
00804f70   NandReadSpareArea
00805068   readNandPage
00805330   NandWriteDataBytes
00805394   writeNandPage
00805620   NandWriteSpareArea
00805738   nandFlashBlockErase
008058f8   NandGetDetails
00805a00   nandInit
00805a64   i2cEepromWriteBlock
00805d2c   i2cEepromRead
00805f30   i2cEepromWrite
00806050   i2cEepromWriteByteAddr
008061a8   i2cEepromMacWrite
00806440   i2cEepromMacRead
008067a0   getStats
0080696c   attachAll
00806a6c   detachAll
00806b54   allocateMessages
00806bd0   freeMessages
00806c34   syncSendCore
00806d88   syncReceiveCore
00806f28   sendMessages
00807094   receiveMessages
008071c4   getStartTime64
008071ec   getExecutionTime64
00807244   calculateThroughput
00807360   printStatistics
00807764   initPlatform
00807ad0   tsk0
00807b48   main
00807de0   ti_sdo_ipc_heaps_HeapMemMP_alloc__E
00808840   ti_sdo_ipc_heaps_HeapMemMP_free__E
00809220   Ipc_attach
00809bc0   xdc_runtime_System_doPrint__I
0080a560   Ipc_detach
0080b028   Osal_platformMalloc
0080b058   Osal_platformFree
0080b084   Osal_platformSpiCsEnter
0080b0a0   Osal_platformSpiCsExit
0080b0ac   Osal_qmssBeginMemAccess
0080b0ec   Osal_qmssEndMemAccess
0080b128   Osal_qmssCsEnter
0080b14c   Osal_qmssCsExit
0080b16c   Osal_qmssMalloc
0080b1a8   Osal_qmssFree
0080b1e0   Osal_cppiCsEnter
0080b204   Osal_cppiCsExit
0080b22c   Osal_cppiBeginMemAccess
0080b26c   Osal_cppiEndMemAccess
0080b2a8   Osal_cppiMalloc
0080b2e8   Osal_cppiFree
0080b324   Osal_srioMalloc
0080b360   Osal_srioFree
0080b394   Osal_dataBufferInitMemory
0080b460   Osal_srioDataBufferMalloc
0080b524   Osal_srioDataBufferFree
0080b5b8   Osal_srioLog
0080b5d0   Osal_srioCreateSem
0080b5e4   Osal_srioDeleteSem
0080b5f0   Osal_srioPendSem
0080b604   Osal_srioPostSem
0080b610   Osal_srioEnterMultipleCoreCriticalSection
0080b634   Osal_srioExitMultipleCoreCriticalSection
0080b654   Osal_srioEnterSingleCoreCriticalSection
0080b678   Osal_srioExitSingleCoreCriticalSection
0080b69c   Osal_srioBeginMemAccess
0080b6d8   Osal_srioEndMemAccess
0080b714   Osal_srioBeginDescriptorAccess
0080b758   Osal_srioEndDescriptorAccess
0080b7a0   ti_sdo_ipc_GateMP_Instance_finalize__F
0080c000   MessageQ_put
0080c840   ti_sdo_ipc_heaps_HeapMemMP_Instance_init__F
0080cfc0   ti_sysbios_family_c64p_Exception_handler__I
0080d740   pow
0080de40   UartInit
0080e198   UartSetBaudRate
0080e210   UartSetBaudRate_B
0080e280   UartReadBaudRate
0080e2f0   UartReadBaudRate_B
0080e368   UartReadData
0080e394   UartReadData_B
0080e3c4   UartWriteData
0080e420   UartWriteData_B
0080e478   UartIsDataReady
0080e4b4   UartIsDataReady_B
0080e500   ti_sdo_ipc_nsremote_NameServerRemoteNotify_Instance_init__F
0080ebc0   NameServer_add
0080f260   ti_sysbios_heaps_HeapMem_free__E
0080f8c0   Notify_sendEvent
0080fee0   ti_sysbios_heaps_HeapMem_alloc__E
00810500   Notify_registerEventSingle
00810ae0   Notify_unregisterEventSingle
008110a0   __c6xabi_divd
00811c50   spi_claim
00811df8   spi_release
00811e10   spi_xfer
00811f48   spi_cmd
00811fc0   spi_cmd_read
00812020   spi_cmd_write
00812080   spi_read_word
0081212c   spi_write_word
008121e0   ti_sdo_ipc_SharedRegion_start__F
008127a0   ti_sysbios_timers_timer64_Timer_Module_startup__F
00812d60   ti_sdo_ipc_nsremote_NameServerRemoteNotify_get__F
008132e0   MessageQ_free
00813840   NameServer_get
00813da0   ti_sdo_ipc_Ipc_procSyncStart__I
00814360   nor_get_details
008143ec   nor_init
00814470   nor_read
00814500   nor_write
008146d4   nor_erase
00814800   ti_sdo_ipc_notifyDrivers_NotifyDriverCirc_Instance_init__F
00814ce0   getBoardVersion
00814d2c   getFpgaDevID
00814d78   fpgaControlUserLEDs
00814e38   fpgaDisableNandWriteProtect
00814e80   fpgaEnableNandWriteProtect
00814ec4   fpgaDisableNorWriteProtect
00814f08   fpgaEnableNorWriteProtect
00814f4c   fpgaDisableEepromWriteProtect
00814f90   fpgaEnableEepromWriteProtect
00814fd4   fpgaGetUserSwitch
00815020   fpgaGetAMCDetect
00815064   fpgaWriteConfigurationRegister
00815110   fpgaReadConfigurationRegister
008151a0   ti_sdo_ipc_gates_GatePeterson_Instance_init__F
00815640   _printfi
00815f00   ti_sdo_ipc_GateMP_setRegion0Reserved__F
00816360   ti_sdo_ipc_Ipc_procSyncFinish__I
008167c0   ti_sdo_ipc_MessageQ_Instance_init__F
00816c20   ti_sdo_ipc_heaps_HeapMemMP_getStats__E
00817060   ti_sdo_ipc_heaps_HeapMemMP_postInit__I
008174a0   ti_sdo_ipc_Notify_Instance_init__F
008178a0   ti_sysbios_knl_Semaphore_pend__E
00817ca0   ti_sdo_ipc_SharedRegion_reserveMemory__F
00818060   ti_sysbios_knl_Task_setPri__E
00818420   fputs
008187c0   HeapMemMP_sharedMemReq
00818b40   MessageQ_alloc
00818ec0   GateMP_sharedMemReq
00819200   ti_sdo_ipc_nsremote_NameServerRemoteNotify_swiFxn__I
00819540   xdc_runtime_System_printfExtend__I
00819ba0   GateMP_openByAddr
00819ea0   ti_sysbios_family_c64p_Hwi_dispatchC__I
0081a1a0   SharedRegion_getEntry
0081a480   SharedRegion_getPtr
0081aa40   ti_sdo_ipc_notifyDrivers_NotifyDriverCirc_isr__I
0081ad20   ti_sysbios_gates_GateMutexPri_enter__E
0081b000   ti_sysbios_knl_Task_Module_startup__F
0081b2e0   MessageQ_open
0081b5a0   Ipc_start
0081b840   NameServer_getLocal
0081bd80   ti_sysbios_knl_Clock_workFunc__E
0081c020   SharedRegion_getSRPtr
0081c2a0   __c6xabi_divf
0081ca20   ti_sdo_ipc_notifyDrivers_NotifyDriverCirc_sharedMemReq__F
0081cca0   ti_sysbios_knl_Clock_Instance_init__F
0081cf20   ti_sysbios_knl_Task_exit__E
0081d1a0   xdc_runtime_Core_createObject__I
0081d420   xdc_runtime_Error_raiseX__F
0081d6a0   ti_sdo_ipc_heaps_HeapMemMP_Instance_finalize__F
0081d900   xdc_runtime_Startup_startMods__I
0081db60   __c6xabi_divull
0081e220   ti_sdo_ipc_MessageQ_Instance_finalize__F
0081e460   ti_sdo_ipc_notifyDrivers_NotifyDriverCirc_sendEvent__E
0081e6a0   ti_sysbios_family_c64p_Exception_internalHandler__I
0081e8e0   ti_sysbios_knl_Semaphore_post__E
0081eb20   MessageQ_get
0081ef60   fputc
0081f180   ti_sysbios_family_c64p_Hwi_reconfig__E
0081f3a0   ti_sysbios_knl_Swi_run__I
0081f5c0   ti_sysbios_knl_Task_schedule__I
0081f7e0   ti_sysbios_knl_Task_startup__E
0081fa00   GateMP_enter
0081fc00   GateMP_leave
00820000   ti_sysbios_family_c64p_Hwi_dispatchAlways
00820400   setvbuf
00820600   ti_sdo_ipc_family_c647x_MultiProcSetup_init__I
00820800   ti_sdo_ipc_GateMP_attach__F
008209e0   ti_sdo_ipc_GateMP_getFreeResource__I
00820bc0   ti_sysbios_knl_Task_postInit__I
00820da0   ti_sysbios_timers_timer64_Timer_getFreq__E
00820f80   HeapMemMP_openByAddr
00821300   ti_sysbios_knl_Swi_Instance_init__F
008214c0   ti_sysbios_knl_Task_checkStacks__E
00821680   ti_sysbios_timers_timer64_Timer_setPeriodMicroSecs__E
00821840   HOSTrename
008219e0   SharedRegion_getCacheLineSize
00821b80   SharedRegion_getHeap
00821d20   SharedRegion_isCacheEnabled
00821ec0   __c6xabi_divul
00822060   ti_sdo_ipc_GateMP_openRegion0Reserved__F
00822200   ti_sdo_ipc_nsremote_NameServerRemoteNotify_attach__E
008223a0   ti_sdo_ipc_transports_TransportShmNotify_put__E
00822540   ti_sysbios_gates_GateMutex_enter__E
008226e0   ti_sysbios_timers_timer64_Timer_start__E
00822880   MultiProc_getName
00822a00   MultiProc_setLocalId
00822b80   NameServer_getHandle
00822d00   Notify_intLineRegistered
00823000   frexp
00823180   ti_sysbios_family_c64p_Exception_dispatch__E
00823300   ti_sdo_ipc_MessageQ_registerTransport__F
00823480   ti_sdo_ipc_Notify_Module_startup__F
00823600   ti_sdo_ipc_gates_GatePeterson_enter__E
00823780   ti_sdo_utils_NameServer_Module_startup__F
00823900   ti_sysbios_heaps_HeapMem_Instance_init__F
00823a80   ti_sysbios_knl_Swi_schedule__I
00823c00   ti_sysbios_knl_Task_unblockI__E
00823d80   xdc_runtime_Text_putSite__F
00823f00   ldexp
00824060   sqrt
00824294   configSerdes
00824320   ti_sdo_ipc_GateMP_createLocal__F
00824480   ti_sdo_ipc_MessageQ_unregisterTransport__F
008245e0   ti_sdo_ipc_gates_GateHWSem_Instance_init__F
00824740   ti_sdo_utils_NameServer_isRegistered__E
008248a0   ti_sdo_utils_NameServer_registerRemoteDriver__E
00824a00   ti_sdo_utils_NameServer_unregisterRemoteDriver__E
00824b60   ti_sysbios_syncs_SyncSem_Instance_init__F
00824cc0   CSL_chipReadReg
00824e00   GateMP_close
00824f40   MessageQ_registerHeap
00825080   Notify_attach
008251c0   _auto_init_elf
00825580   ti_sdo_ipc_Notify_exec__F
008256c0   ti_sysbios_family_c64p_Hwi_Module_startup__F
00825800   ti_sysbios_family_c66_Cache_Module_startup__F
00825940   ti_sysbios_gates_GateSwi_enter__E
00825a80   ti_sysbios_knl_Clock_Instance_finalize__F
00825bc0   ti_sysbios_knl_Semaphore_Instance_init__F
00825d00   ti_sysbios_knl_Swi_post__E
00825e40   ti_sysbios_knl_Task_blockI__E
00825f80   ti_sysbios_knl_Task_yield__E
008260c0   _closefile
00826300   fseek
00826540   ti_sdo_ipc_MessageQ_Module_startup__F
00826660   ti_sdo_ipc_family_c647x_Interrupt_intRegister__E
00826780   ti_sdo_ipc_nsremote_NameServerRemoteNotify_Instance_finalize__F
008268a0   HOSTlseek
008269a0   _wrt_ok
00826ba0   ti_sdo_ipc_GateMP_start__F
00826ca0   ti_sdo_ipc_Notify_Instance_finalize__F
00826da0   ti_sdo_ipc_SharedRegion_attach__F
00826ea0   ti_sdo_ipc_SharedRegion_clearReservedMemory__F
00826fa0   ti_sdo_ipc_family_c647x_Interrupt_Module_startup__F
008270a0   ti_sdo_ipc_gates_GateHWSem_Module_startup__F
008271a0   ti_sdo_ipc_gates_GateMPSupportNull_enter__E
008272a0   ti_sdo_ipc_gates_GateMPSupportNull_leave__E
008273a0   ti_sdo_ipc_transports_TransportShmNotify_Instance_init__F
008274a0   ti_sysbios_gates_GateMutexPri_leave__E
008275a0   ti_sysbios_knl_Clock_startI__E
008276a0   ti_sysbios_knl_Swi_restoreHwi__E
008277a0   xdc_runtime_Core_deleteObject__I
008278a0   xdc_runtime_Startup_exec__F
008279a0   xdc_runtime_Text_putMod__F
00827aa0   xdc_runtime_Text_visitRope2__I
00827ba0   HOSTopen
00827d60   atoi
00827e40   close
00827f20   __TI_zero_init
00828000   fflush
008280e0   ltoa
008281c0   memset
008282a0   printf
00828380   ti_sdo_ipc_Notify_Object__create__S
00828460   ti_sdo_ipc_Notify_detach__F
00828540   ti_sdo_ipc_family_c647x_NotifyCircSetup_attach__E
00828620   ti_sdo_ipc_gates_GateHWSem_enter__E
00828700   ti_sdo_ipc_notifyDrivers_NotifyDriverCirc_disableEvent__E
008287e0   ti_sdo_ipc_notifyDrivers_NotifyDriverCirc_enable__E
008288c0   ti_sysbios_family_c64p_Hwi_Instance_finalize__F
008289a0   ti_sysbios_family_c64p_Hwi_Instance_init__F
00828a80   ti_sysbios_family_c64p_Hwi_Object__create__S
00828b60   ti_sysbios_knl_Clock_start__E
00828c40   ti_sysbios_timers_timer64_Timer_startup__E
00828d20   xdc_runtime_Error_print__F
00828e00   xdc_runtime_Memory_alloc__F
00828ee0   HOSTread
00828fa0   HOSTunlink
00829060   HOSTwrite
00829120   HeapMemMP_create
008292a0   __cxa_finalize
00829360   __c6xabi_divu
00829360   __divu
00829420   _doflush
008294e0   exit
008295a0   ti_sdo_ipc_GateMP_Object__create__S
00829660   ti_sdo_ipc_GateMP_getRegion0ReservedSize__F
00829720   ti_sdo_ipc_MessageQ_Object__create__S
008297e0   ti_sdo_ipc_family_c647x_Interrupt_intShmStub__I
008298a0   ti_sdo_ipc_gates_GatePeterson_Object__create__S
00829960   ti_sdo_ipc_heaps_HeapMemMP_Object__create__S
00829a20   ti_sdo_ipc_nsremote_NameServerRemoteNotify_Object__create__S
00829ae0   ti_sdo_ipc_transports_TransportShmNotifySetup_attach__E
00829ba0   ti_sdo_ipc_transports_TransportShmNotify_Object__create__S
00829c60   ti_sysbios_BIOS_errorRaiseHook__I
00829d20   ti_sysbios_gates_GateAll_leave__E
00829de0   ti_sysbios_heaps_HeapMem_getStats__E
00829ea0   ti_sysbios_knl_Clock_logTick__E
00829f60   ti_sysbios_knl_Swi_Instance_finalize__F
0082a020   ti_sysbios_knl_Swi_Object__create__S
0082a0e0   ti_sysbios_syncs_SyncSem_Object__create__S
0082a1a0   ti_sysbios_timers_timer64_Timer_stop__E
0082a260   xdc_runtime_System_formatNum__I
0082a320   xdc_runtime_knl_GateThread_Object__create__S
0082a3e0   HOSTclose
0082a480   MessageQ_create
0082a520   __c6xabi_fltulld
0082a5c0   __c6xabi_nround
0082a660   __c6xabi_remu
0082a660   __remu
0082a700   _c_int00
0082a7a0   _cleanup
0082aa20   ti_sysbios_family_c64p_Hwi_plug__E
0082ab60   lseek
0082ac00   memcpy
0082aca0   modf
0082ad40   ti_sdo_ipc_family_c647x_Interrupt_intUnregister__E
0082ade0   ti_sdo_ipc_gates_GatePeterson_leave__E
0082ae80   ti_sdo_ipc_notifyDrivers_NotifyDriverCirc_Instance_finalize__F
0082af20   ti_sysbios_heaps_HeapMem_init__I
0082afc0   ti_sysbios_syncs_SyncSem_wait__F
0082b060   write
0082b100   xdc_runtime_Assert_raise__I
0082b1a0   __c6xabi_fixdu
0082b220   __c6xabi_fixfu
0082b2a0   __c6xabi_llshl
0082b320   ti_sysbios_family_c62_TaskSupport_swap__E
0082b3a0   malloc
0082b420   readmsg
0082b4a0   strncpy
0082b520   evmI2CInit
0082b5a0   ti_sdo_ipc_gates_GateHWSem_Object__create__S
0082b620   ti_sdo_ipc_gates_GateMPSupportNull_Object__create__S
0082b6a0   ti_sdo_ipc_notifyDrivers_NotifyDriverCirc_Object__create__S
0082b720   ti_sdo_ipc_nsremote_NameServerRemoteNotify_detach__E
0082b7a0   ti_sdo_ipc_transports_TransportShmNotify_Instance_finalize__F
0082b820   ti_sdo_utils_List_Object__create__S
0082b8a0   ti_sysbios_family_c62_TaskSupport_start__E
0082b920   ti_sysbios_family_c64p_Exception_Module_startup__F
0082b9a0   ti_sysbios_family_c64p_Hwi_eventMap__E
0082ba20   ti_sysbios_family_c66_Cache_invL1pAll__E
0082baa0   ti_sysbios_gates_GateAll_Object__create__S
0082bb20   ti_sysbios_gates_GateHwi_Object__create__S
0082bba0   ti_sysbios_gates_GateMutexPri_Object__create__S
0082bc20   ti_sysbios_gates_GateMutex_Object__create__S
0082bca0   ti_sysbios_gates_GateSwi_Object__create__S
0082bd20   ti_sysbios_gates_GateSwi_leave__E
0082bda0   ti_sysbios_hal_Hwi_checkStack
0082be20   ti_sysbios_heaps_HeapMem_Object__create__S
0082bea0   ti_sysbios_knl_Clock_Module_startup__F
0082bf20   ti_sysbios_knl_Clock_Object__create__S
0082bfa0   ti_sysbios_knl_Clock_getTicks__E
0082c020   ti_sysbios_knl_Idle_loop__E
0082c0a0   ti_sysbios_knl_Queue_Object__create__S
0082c120   ti_sysbios_knl_Semaphore_Object__create__S
0082c1a0   ti_sysbios_knl_Semaphore_pendTimeout__I
0082c220   ti_sysbios_knl_Swi_startup__E
0082c2a0   ti_sysbios_knl_Task_restore__E
0082c320   ti_sysbios_timers_timer64_Timer_getCount__E
0082c320   ti_sysbios_timers_timer64_Timer_getExpiredCounts__E
0082c3a0   ti_sysbios_timers_timer64_Timer_getPeriod__E
0082c420   ti_sysbios_xdcruntime_GateThreadSupport_Object__create__S
0082c4a0   remove
0082c4a0   unlink
0082c520   xdc_runtime_Core_assignLabel__I
0082c5a0   xdc_runtime_Core_assignParams__I
0082c620   xdc_runtime_System_atexit__F
0082c6a0   xdc_runtime_System_rtsExit__I
0082c720   xdc_runtime_Text_printVisFxn__I
0082c7a0   xdc_runtime_Text_xprintf__I
0082c820   GateMP_Params_init
0082c880   HeapMemMP_Params_init
0082c8e0   Notify_numIntLines
0082c940   __c6xabi_frcmpyd_div
0082c9a0   __c6xabi_llshru
0082ca00   _subcull
0082ca60   memccpy
0082cac0   ti_sdo_ipc_MessageQ_Object__get__S
0082cb20   ti_sdo_ipc_family_c647x_NotifyCircSetup_sharedMemReq__E
0082cb80   ti_sdo_ipc_gates_GateHWSem_leave__E
0082cbe0   ti_sdo_ipc_gates_GatePeterson_Instance_finalize__F
0082cc40   ti_sdo_ipc_gates_GatePeterson_sharedMemReq__E
0082cca0   ti_sdo_ipc_transports_TransportShmNotifySetup_detach__E
0082cd00   ti_sdo_ipc_transports_TransportShmNotify_notifyFxn__I
0082cd60   ti_sdo_utils_List_Object__get__S
0082cdc0   ti_sdo_utils_NameServer_Object__get__S
0082ce20   ti_sysbios_BIOS_exitFunc__I
0082ce80   ti_sysbios_BIOS_registerRTSLock__I
0082cee0   ti_sysbios_gates_GateAll_enter__E
0082cf40   ti_sysbios_gates_GateMutex_Instance_init__F
0082cfa0   ti_sysbios_hal_Hwi_initStack
0082d000   ti_sysbios_heaps_HeapMem_Object__get__S
0082d060   ti_sysbios_knl_Clock_doTick__I
0082d0c0   ti_sysbios_knl_Queue_Object__get__S
0082d120   ti_sysbios_knl_Swi_Module_startup__F
0082d180   ti_sysbios_knl_Swi_Object__get__S
0082d1e0   ti_sysbios_knl_Task_Object__get__S
0082d240   ti_sysbios_knl_Task_allBlockedFunction__I
0082d2a0   ti_sysbios_knl_Task_enter__I
0082d300   vsprintf
0082d360   writemsg
0082d3b8   C$$IO$$
0082d3c0   xdc_runtime_GateNull_Object__create__S
0082d420   xdc_runtime_Memory_calloc__F
0082d480   xdc_runtime_SysStd_abort__F
0082d4e0   xdc_runtime_System_aprintf_va__F
0082d4e0   xdc_runtime_System_avprintf__F
0082d540   xdc_runtime_System_printf_va__F
0082d540   xdc_runtime_System_vprintf__F
0082d5a0   xdc_runtime_Text_cordText__F
0082d600   __c6xabi_isinf
0082d680   _args_main
0082d700   ti_sysbios_family_c62_TaskSupport_buildTaskStack
0082d740   ti_sysbios_family_xxx_Hwi_switchToIsrStack
0082d780   free
0082d7c0   l2_global_address
0082d840   strlen
0082d880   ti_sdo_ipc_GateMP_Object__delete__S
0082d8c0   ti_sdo_ipc_GateMP_Params__init__S
0082d900   ti_sdo_ipc_GateMP_RemoteCustom1Proxy_Object__create__S
0082d940   ti_sdo_ipc_GateMP_RemoteCustom2Proxy_Object__create__S
0082d980   ti_sdo_ipc_GateMP_RemoteSystemProxy_Object__create__S
0082d9c0   ti_sdo_ipc_MessageQ_Params__init__S
0082da00   ti_sdo_ipc_MessageQ_registerTransport__E
0082da40   ti_sdo_ipc_Notify_Object__delete__S
0082da80   ti_sdo_ipc_family_c647x_Interrupt_intClear__E
0082dac0   ti_sdo_ipc_family_c647x_Interrupt_intSend__E
0082db00   ti_sdo_ipc_gates_GateHWSem_Handle__label__S
0082db40   ti_sdo_ipc_gates_GateHWSem_Object__delete__S
0082db80   ti_sdo_ipc_gates_GateHWSem_Params__init__S
0082dbc0   ti_sdo_ipc_gates_GateMPSupportNull_Handle__label__S
0082dc00   ti_sdo_ipc_gates_GateMPSupportNull_Object__delete__S
0082dc40   ti_sdo_ipc_gates_GateMPSupportNull_Params__init__S
0082dc80   ti_sdo_ipc_gates_GatePeterson_Handle__label__S
0082dcc0   ti_sdo_ipc_gates_GatePeterson_Object__delete__S
0082dd00   ti_sdo_ipc_gates_GatePeterson_Params__init__S
0082dd40   ti_sdo_ipc_heaps_HeapMemMP_Handle__label__S
0082dd80   ti_sdo_ipc_heaps_HeapMemMP_Object__delete__S
0082ddc0   ti_sdo_ipc_heaps_HeapMemMP_Params__init__S
0082de00   ti_sdo_ipc_notifyDrivers_NotifyDriverCirc_Handle__label__S
0082de40   ti_sdo_ipc_notifyDrivers_NotifyDriverCirc_InterruptProxy_intRegister__E
0082de80   ti_sdo_ipc_notifyDrivers_NotifyDriverCirc_Object__delete__S
0082dec0   ti_sdo_ipc_notifyDrivers_NotifyDriverCirc_Params__init__S
0082df00   ti_sdo_ipc_notifyDrivers_NotifyDriverCirc_disable__E
0082df40   ti_sdo_ipc_notifyDrivers_NotifyDriverCirc_enableEvent__E
0082df80   ti_sdo_ipc_notifyDrivers_NotifyDriverCirc_registerEvent__E
0082dfc0   ti_sdo_ipc_notifyDrivers_NotifyDriverCirc_unregisterEvent__E
0082e000   ti_sdo_ipc_nsremote_NameServerRemoteNotify_Handle__label__S
0082e040   ti_sdo_ipc_nsremote_NameServerRemoteNotify_Object__delete__S
0082e080   ti_sdo_ipc_nsremote_NameServerRemoteNotify_Object__first__S
0082e0c0   ti_sdo_ipc_nsremote_NameServerRemoteNotify_Object__next__S
0082e100   ti_sdo_ipc_nsremote_NameServerRemoteNotify_Params__init__S
0082e140   ti_sdo_ipc_nsremote_NameServerRemoteNotify_get__E
0082e180   ti_sdo_ipc_nsremote_NameServerRemoteNotify_sharedMemReq__E
0082e1c0   ti_sdo_ipc_transports_TransportShmNotify_Handle__label__S
0082e200   ti_sdo_ipc_transports_TransportShmNotify_Object__delete__S
0082e240   ti_sdo_ipc_transports_TransportShmNotify_Params__init__S
0082e280   ti_sdo_utils_List_Object__destruct__S
0082e2c0   ti_sdo_utils_NameServer_Module__startupDone__F
0082e300   ti_sdo_utils_NameServer_Object__first__S
0082e340   ti_sdo_utils_NameServer_Object__next__S
0082e380   ti_sysbios_BIOS_startFunc__I
0082e3c0   ti_sysbios_BIOS_start__E
0082e400   ti_sysbios_family_c64p_Hwi_Module__startupDone__F
0082e440   ti_sysbios_family_c64p_Hwi_Object__delete__S
0082e480   ti_sysbios_family_c64p_Hwi_Params__init__S
0082e4c0   ti_sysbios_family_c64p_Hwi_disableInterrupt__E
0082e500   ti_sysbios_family_c64p_Hwi_enableInterrupt__E
0082e540   ti_sysbios_family_c66_Cache_wait__E
0082e580   ti_sysbios_gates_GateAll_Handle__label__S
0082e5c0   ti_sysbios_gates_GateAll_Object__delete__S
0082e600   ti_sysbios_gates_GateHwi_Handle__label__S
0082e640   ti_sysbios_gates_GateHwi_Object__delete__S
0082e680   ti_sysbios_gates_GateMutexPri_Handle__label__S
0082e6c0   ti_sysbios_gates_GateMutexPri_Instance_finalize__F
0082e700   ti_sysbios_gates_GateMutexPri_Instance_init__F
0082e740   ti_sysbios_gates_GateMutexPri_Object__delete__S
0082e780   ti_sysbios_gates_GateMutexPri_Object__destruct__S
0082e7c0   ti_sysbios_gates_GateMutex_Handle__label__S
0082e800   ti_sysbios_gates_GateMutex_Instance_finalize__F
0082e840   ti_sysbios_gates_GateMutex_Object__delete__S
0082e880   ti_sysbios_gates_GateMutex_leave__E
0082e8c0   ti_sysbios_gates_GateSwi_Handle__label__S
0082e900   ti_sysbios_gates_GateSwi_Object__delete__S
0082e940   ti_sysbios_hal_Cache_CacheProxy_inv__E
0082e940   ti_sysbios_hal_Cache_inv__E
0082e980   ti_sysbios_hal_Cache_CacheProxy_wbInv__E
0082e980   ti_sysbios_hal_Cache_wbInv__E
0082e9c0   ti_sysbios_hal_Cache_CacheProxy_wb__E
0082e9c0   ti_sysbios_hal_Cache_wb__E
0082ea00   ti_sysbios_hal_Timer_Module__startupDone__F
0082ea40   ti_sysbios_heaps_HeapMem_Handle__label__S
0082ea80   ti_sysbios_heaps_HeapMem_Object__delete__S
0082eac0   ti_sysbios_knl_Clock_Object__destruct__S
0082eb00   ti_sysbios_knl_Clock_Params__init__S
0082eb40   ti_sysbios_knl_Queue_Object__destruct__S
0082eb80   ti_sysbios_knl_Semaphore_Instance_finalize__F
0082ebc0   ti_sysbios_knl_Semaphore_Object__delete__S
0082ec00   ti_sysbios_knl_Semaphore_Object__destruct__S
0082ec40   ti_sysbios_knl_Semaphore_Params__init__S
0082ec80   ti_sysbios_knl_Swi_Object__destruct__S
0082ecc0   ti_sysbios_knl_Swi_Params__init__S
0082ed00   ti_sysbios_knl_Task_Object__first__S
0082ed40   ti_sysbios_knl_Task_Object__next__S
0082ed80   ti_sysbios_syncs_SyncSem_Handle__label__S
0082edc0   ti_sysbios_syncs_SyncSem_Instance_finalize__F
0082ee00   ti_sysbios_syncs_SyncSem_Object__delete__S
0082ee40   ti_sysbios_timers_timer64_Timer_Module__startupDone__F
0082ee80   ti_sysbios_xdcruntime_GateThreadSupport_Instance_finalize__F
0082eec0   ti_sysbios_xdcruntime_GateThreadSupport_Instance_init__F
0082ef00   ti_sysbios_xdcruntime_GateThreadSupport_Object__delete__S
0082ef40   ti_sysbios_xdcruntime_GateThreadSupport_enter__F
0082ef80   ti_sysbios_xdcruntime_GateThreadSupport_leave__F
0082efc0   xdc_runtime_Error_check__F
0082f000   xdc_runtime_Error_init__F
0082f040   xdc_runtime_Error_raiseX__E
0082f080   xdc_runtime_GateNull_Handle__label__S
0082f0c0   xdc_runtime_GateNull_Object__delete__S
0082f100   xdc_runtime_Gate_leaveSystem__F
0082f1c0   xdc_runtime_Memory_free__F
0082f200   xdc_runtime_Registry_findById__F
0082f240   xdc_runtime_Startup_exec__I
0082f280   xdc_runtime_System_abort__F
0082f2c0   xdc_runtime_System_aprintf__E
0082f300   xdc_runtime_System_printf__E
0082f340   xdc_runtime_System_sprintf__E
0082f380   xdc_runtime_Text_ropeText__F
0082f3c0   xdc_runtime_Text_visitRope__I
0082f400   xdc_runtime_knl_GateThread_Handle__label__S
0082f440   xdc_runtime_knl_GateThread_Instance_finalize__F
0082f480   xdc_runtime_knl_GateThread_Instance_init__F
0082f4c0   xdc_runtime_knl_GateThread_Object__delete__S
0082f500   xdc_runtime_knl_GateThread_Proxy_Object__create__S
0082f540   GateMP_getDefaultRemote
0082f560   MultiProc_getBaseIdOfCluster
0082f580   MultiProc_getNumProcessors
0082f5a0   MultiProc_self
0082f5c0   __c6xabi_errno_addr
0082f5e0   __c6xabi_negll
0082f600   __c6xabi_trunc
0082f620   __cxa_atexit
0082f640   __cxa_ia64_exit
0082f660   __xdc__init
0082f680   _nop
0082f700   _register_lock
0082f720   _register_unlock
0082f740   ti_sysbios_family_c62_TaskSupport_glue
0082f760   ti_sysbios_family_xxx_Hwi_switchToTaskStack
0082f780   C$$EXIT
0082f780   abort
0082f7a0   atexit
0082f7c0   __TI_decompress_none
0082f7e0   __TI_decompress_rle24
0082f820   putc
0082f840   putchar
0082f860   ti_sdo_ipc_GateMP_RemoteCustom1Proxy_Object__delete__S
0082f880   ti_sdo_ipc_GateMP_RemoteCustom1Proxy_Params__init__S
0082f8a0   ti_sdo_ipc_GateMP_RemoteCustom1Proxy_Proxy__abstract__S
0082f8c0   ti_sdo_ipc_GateMP_RemoteCustom1Proxy_Proxy__delegate__S
0082f8e0   ti_sdo_ipc_GateMP_RemoteCustom1Proxy_getReservedMask__E
0082f900   ti_sdo_ipc_GateMP_RemoteCustom1Proxy_sharedMemReq__E
0082f920   ti_sdo_ipc_GateMP_RemoteCustom2Proxy_Object__delete__S
0082f940   ti_sdo_ipc_GateMP_RemoteCustom2Proxy_Params__init__S
0082f960   ti_sdo_ipc_GateMP_RemoteCustom2Proxy_Proxy__abstract__S
0082f980   ti_sdo_ipc_GateMP_RemoteCustom2Proxy_Proxy__delegate__S
0082f9a0   ti_sdo_ipc_GateMP_RemoteCustom2Proxy_getReservedMask__E
0082f9c0   ti_sdo_ipc_GateMP_RemoteCustom2Proxy_sharedMemReq__E
0082f9e0   ti_sdo_ipc_GateMP_RemoteSystemProxy_Object__delete__S
0082fa00   ti_sdo_ipc_GateMP_RemoteSystemProxy_Params__init__S
0082fa20   ti_sdo_ipc_GateMP_RemoteSystemProxy_Proxy__abstract__S
0082fa40   ti_sdo_ipc_GateMP_RemoteSystemProxy_Proxy__delegate__S
0082fa60   ti_sdo_ipc_GateMP_RemoteSystemProxy_getReservedMask__E
0082fa80   ti_sdo_ipc_GateMP_RemoteSystemProxy_sharedMemReq__E
0082faa0   ti_sdo_ipc_GateMP_attach__E
0082fac0   ti_sdo_ipc_GateMP_getRegion0ReservedSize__E
0082fae0   ti_sdo_ipc_GateMP_getSharedAddr__E
0082fb00   ti_sdo_ipc_GateMP_getSharedAddr__F
0082fb20   ti_sdo_ipc_GateMP_start__E
0082fb40   ti_sdo_ipc_MessageQ_Module_startup__E
0082fb60   ti_sdo_ipc_MessageQ_SetupTransportProxy_attach__E
0082fb80   ti_sdo_ipc_MessageQ_SetupTransportProxy_detach__E
0082fba0   ti_sdo_ipc_MessageQ_SetupTransportProxy_isRegistered__E
0082fbc0   ti_sdo_ipc_MessageQ_SetupTransportProxy_sharedMemReq__E
0082fbe0   ti_sdo_ipc_MessageQ_unregisterTransport__E
0082fc00   ti_sdo_ipc_Notify_Module_GateProxy_enter__E
0082fc20   ti_sdo_ipc_Notify_Module_GateProxy_leave__E
0082fc40   ti_sdo_ipc_Notify_Module_startup__E
0082fc60   ti_sdo_ipc_Notify_SetupProxy_attach__E
0082fc80   ti_sdo_ipc_Notify_SetupProxy_numIntLines__E
0082fca0   ti_sdo_ipc_Notify_SetupProxy_sharedMemReq__E
0082fcc0   ti_sdo_ipc_Notify_detach__E
0082fce0   ti_sdo_ipc_Notify_exec__E
0082fd00   ti_sdo_ipc_SharedRegion_attach__E
0082fd20   ti_sdo_ipc_SharedRegion_clearReservedMemory__E
0082fd40   ti_sdo_ipc_SharedRegion_reserveMemory__E
0082fd60   ti_sdo_ipc_SharedRegion_start__E
0082fd80   ti_sdo_ipc_family_c647x_Interrupt_Module_startup__E
0082fda0   ti_sdo_ipc_family_c647x_Interrupt_intDisable__E
0082fdc0   ti_sdo_ipc_family_c647x_Interrupt_intEnable__E
0082fde0   ti_sdo_ipc_family_c647x_NotifyCircSetup_numIntLines__E
0082fe00   ti_sdo_ipc_gates_GateHWSem_Module_startup__E
0082fe20   ti_sdo_ipc_gates_GateHWSem_getReservedMask__E
0082fe40   ti_sdo_ipc_gates_GateHWSem_query__E
0082fe60   ti_sdo_ipc_gates_GateHWSem_query__F
0082fe80   ti_sdo_ipc_gates_GateHWSem_sharedMemReq__E
0082fea0   ti_sdo_ipc_gates_GateMPSupportNull_Instance_init__F
0082fec0   ti_sdo_ipc_gates_GateMPSupportNull_getReservedMask__E
0082fee0   ti_sdo_ipc_gates_GateMPSupportNull_query__E
0082ff00   ti_sdo_ipc_gates_GateMPSupportNull_query__F
0082ff20   ti_sdo_ipc_gates_GateMPSupportNull_sharedMemReq__E
0082ff40   ti_sdo_ipc_gates_GatePeterson_getReservedMask__E
0082ff60   ti_sdo_ipc_gates_GatePeterson_query__E
0082ff80   ti_sdo_ipc_gates_GatePeterson_query__F
0082ffa0   ti_sdo_ipc_heaps_HeapMemMP_isBlocking__E
0082ffc0   ti_sdo_ipc_heaps_HeapMemMP_isBlocking__F
0082ffe0   ti_sdo_ipc_notifyDrivers_NotifyDriverCirc_InterruptProxy_intClear__E
00830000   ti_sdo_ipc_notifyDrivers_NotifyDriverCirc_InterruptProxy_intDisable__E
00830020   ti_sdo_ipc_notifyDrivers_NotifyDriverCirc_InterruptProxy_intEnable__E
00830040   ti_sdo_ipc_notifyDrivers_NotifyDriverCirc_InterruptProxy_intSend__E
00830060   ti_sdo_ipc_notifyDrivers_NotifyDriverCirc_InterruptProxy_intUnregister__E
00830080   ti_sdo_ipc_notifyDrivers_NotifyDriverCirc_setNotifyHandle__E
008300a0   ti_sdo_ipc_notifyDrivers_NotifyDriverCirc_sharedMemReq__E
008300c0   ti_sdo_ipc_nsremote_NameServerRemoteNotify_cbFxn__I
008300e0   ti_sdo_ipc_transports_TransportShmNotifySetup_isRegistered__E
00830100   ti_sdo_ipc_transports_TransportShmNotifySetup_sharedMemReq__E
00830120   ti_sdo_ipc_transports_TransportShmNotify_control__E
00830140   ti_sdo_ipc_transports_TransportShmNotify_getStatus__E
00830160   ti_sdo_ipc_transports_TransportShmNotify_setErrFxn__E
00830180   ti_sdo_ipc_transports_TransportShmNotify_setErrFxn__F
008301a0   ti_sdo_utils_List_Instance_init__F
008301c0   ti_sdo_utils_MultiProc_getClusterId__E
008301e0   ti_sdo_utils_MultiProc_getClusterId__F
00830200   ti_sdo_utils_NameServer_Module__startupDone__S
00830220   ti_sdo_utils_NameServer_Module_startup__E
00830240   ti_sdo_utils_NameServer_SetupProxy_attach__E
00830260   ti_sdo_utils_NameServer_SetupProxy_detach__E
00830280   ti_sdo_utils_NameServer_SetupProxy_sharedMemReq__E
008302a0   ti_sysbios_BIOS_RtsGateProxy_enter__E
008302c0   ti_sysbios_BIOS_RtsGateProxy_leave__E
008302e0   ti_sysbios_BIOS_getCpuFreq__E
008302e0   ti_sysbios_family_c64p_TimestampProvider_getFreq__E
00830300   ti_sysbios_BIOS_getThreadType__E
00830320   ti_sysbios_BIOS_setThreadType__E
00830340   ti_sysbios_family_c62_TaskSupport_Module__startupDone__S
00830360   ti_sysbios_family_c62_TaskSupport_checkStack__E
00830380   ti_sysbios_family_c64p_Exception_Module_startup__E
008303a0   ti_sysbios_family_c64p_Hwi_Module__startupDone__S
008303c0   ti_sysbios_family_c64p_Hwi_Module_startup__E
008303e0   ti_sysbios_family_c64p_Hwi_clearInterrupt__E
00830400   ti_sysbios_family_c64p_Hwi_getHandle__E
00830420   ti_sysbios_family_c64p_Hwi_startup__E
00830440   ti_sysbios_family_c64p_Hwi_switchFromBootStack__E
00830460   ti_sysbios_family_c64p_Hwi_unPluggedInterrupt__I
00830480   ti_sysbios_family_c64p_TimestampProvider_Module_startup__E
008304a0   ti_sysbios_family_c64p_TimestampProvider_Module_startup__F
008304c0   ti_sysbios_family_c64p_TimestampProvider_get32__E
008304e0   ti_sysbios_family_c64p_TimestampProvider_get64__E
00830500   ti_sysbios_family_c64p_tci6488_TimerSupport_enable__E
00830520   ti_sysbios_family_c66_Cache_Module_startup__E
00830540   ti_sysbios_family_c66_Cache_inv__E
00830560   ti_sysbios_family_c66_Cache_wbInv__E
00830580   ti_sysbios_family_c66_Cache_wb__E
008305a0   ti_sysbios_gates_GateAll_Instance_init__F
008305c0   ti_sysbios_gates_GateAll_query__E
008305e0   ti_sysbios_gates_GateAll_query__F
00830600   ti_sysbios_gates_GateHwi_Instance_init__F
00830620   ti_sysbios_gates_GateHwi_enter__E
00830640   ti_sysbios_gates_GateHwi_leave__E
00830660   ti_sysbios_gates_GateHwi_query__E
00830680   ti_sysbios_gates_GateHwi_query__F
008306a0   ti_sysbios_gates_GateMutexPri_query__E
008306a0   ti_sysbios_xdcruntime_GateProcessSupport_query__F
008306a0   ti_sysbios_xdcruntime_GateThreadSupport_query__F
008306c0   ti_sysbios_gates_GateMutexPri_query__F
008306e0   ti_sysbios_gates_GateMutex_query__E
00830700   ti_sysbios_gates_GateMutex_query__F
00830720   ti_sysbios_gates_GateSwi_Instance_init__F
00830740   ti_sysbios_gates_GateSwi_query__E
00830760   ti_sysbios_gates_GateSwi_query__F
00830780   ti_sysbios_hal_Cache_CacheProxy_wait__E
00830780   ti_sysbios_hal_Cache_wait__E
008307a0   ti_sysbios_hal_Hwi_HwiProxy_Module__startupDone__S
008307c0   ti_sysbios_hal_Hwi_HwiProxy_clearInterrupt__E
008307c0   ti_sysbios_hal_Hwi_clearInterrupt__E
008307e0   ti_sysbios_hal_Hwi_HwiProxy_disableInterrupt__E
008307e0   ti_sysbios_hal_Hwi_disableInterrupt__E
00830800   ti_sysbios_hal_Hwi_HwiProxy_enableInterrupt__E
00830800   ti_sysbios_hal_Hwi_enableInterrupt__E
00830820   ti_sysbios_hal_Hwi_HwiProxy_startup__E
00830820   ti_sysbios_hal_Hwi_startup__E
00830840   ti_sysbios_hal_Hwi_HwiProxy_switchFromBootStack__E
00830840   ti_sysbios_hal_Hwi_switchFromBootStack__E
00830860   ti_sysbios_hal_Hwi_Module_startup__E
00830880   ti_sysbios_hal_Hwi_Module_startup__F
008308a0   ti_sysbios_hal_Timer_Module__startupDone__S
008308c0   ti_sysbios_hal_Timer_Module_startup__E
008308e0   ti_sysbios_hal_Timer_Module_startup__F
00830900   ti_sysbios_hal_Timer_TimerProxy_Module__startupDone__S
00830920   ti_sysbios_hal_Timer_TimerProxy_getExpiredCounts__E
00830940   ti_sysbios_hal_Timer_TimerProxy_getPeriod__E
00830960   ti_sysbios_hal_Timer_TimerProxy_setNextTick__E
00830980   ti_sysbios_hal_Timer_TimerProxy_startup__E
00830980   ti_sysbios_hal_Timer_startup__E
008309a0   ti_sysbios_heaps_HeapMem_Module_GateProxy_enter__E
008309c0   ti_sysbios_heaps_HeapMem_Module_GateProxy_leave__E
008309e0   ti_sysbios_heaps_HeapMem_Module_GateProxy_query__E
00830a00   ti_sysbios_heaps_HeapMem_isBlocking__E
00830a40   ti_sysbios_knl_Clock_Module_startup__E
00830a60   ti_sysbios_knl_Queue_Instance_init__F
00830a80   ti_sysbios_knl_Queue_empty__E
00830aa0   ti_sysbios_knl_Swi_Module_startup__E
00830ac0   ti_sysbios_knl_Swi_disable__E
00830ae0   ti_sysbios_knl_Task_Module_startup__E
00830b00   ti_sysbios_knl_Task_SupportProxy_Module__startupDone__S
00830b20   ti_sysbios_knl_Task_SupportProxy_checkStack__E
00830b40   ti_sysbios_knl_Task_SupportProxy_start__E
00830b60   ti_sysbios_knl_Task_SupportProxy_swap__E
00830b80   ti_sysbios_knl_Task_disable__E
00830ba0   ti_sysbios_knl_Task_getPri__E
00830bc0   ti_sysbios_knl_Task_self__E
00830be0   ti_sysbios_syncs_SyncSem_query__E
00830c00   ti_sysbios_syncs_SyncSem_query__F
00830c20   ti_sysbios_syncs_SyncSem_signal__E
00830c40   ti_sysbios_syncs_SyncSem_signal__F
00830c60   ti_sysbios_syncs_SyncSem_wait__E
00830c80   ti_sysbios_timers_timer64_Timer_Module__startupDone__S
00830ca0   ti_sysbios_timers_timer64_Timer_Module_startup__E
00830cc0   ti_sysbios_timers_timer64_Timer_TimerSupportProxy_enable__E
00830ce0   ti_sysbios_timers_timer64_Timer_setNextTick__E
00830d00   ti_sysbios_xdcruntime_GateThreadSupport_enter__E
00830d20   ti_sysbios_xdcruntime_GateThreadSupport_leave__E
00830d40   ti_sysbios_xdcruntime_GateThreadSupport_query__E
00830d80   xdc_runtime_Error_check__E
00830da0   xdc_runtime_Error_init__E
00830dc0   xdc_runtime_Error_print__E
00830de0   xdc_runtime_GateNull_enter__E
00830e00   xdc_runtime_GateNull_enter__F
00830e20   xdc_runtime_GateNull_leave__E
00830e40   xdc_runtime_GateNull_leave__F
00830e60   xdc_runtime_GateNull_query__E
00830e80   xdc_runtime_GateNull_query__F
00830ea0   xdc_runtime_Gate_enterSystem__E
00830ec0   xdc_runtime_Gate_enterSystem__F
00830ee0   xdc_runtime_Gate_leaveSystem__E
00830f00   xdc_runtime_Memory_HeapProxy_alloc__E
00830f20   xdc_runtime_Memory_HeapProxy_free__E
00830f40   xdc_runtime_Memory_alloc__E
00830f60   xdc_runtime_Memory_calloc__E
00830f80   xdc_runtime_Memory_free__E
00830fa0   xdc_runtime_Memory_getMaxDefaultTypeAlign__E
00830fc0   xdc_runtime_Memory_getMaxDefaultTypeAlign__F
00830fe0   xdc_runtime_Registry_findById__E
00831000   xdc_runtime_Startup_Module__startupDone__S
00831020   xdc_runtime_Startup_exec__E
00831040   xdc_runtime_Startup_reset__I
00831060   xdc_runtime_Startup_rtsDone__E
00831080   xdc_runtime_Startup_rtsDone__F
008310a0   xdc_runtime_SysStd_abort__E
008310c0   xdc_runtime_SysStd_exit__E
008310e0   xdc_runtime_SysStd_exit__F
00831100   xdc_runtime_SysStd_putch__E
00831120   xdc_runtime_SysStd_putch__F
00831140   xdc_runtime_SysStd_ready__E
00831160   xdc_runtime_SysStd_ready__F
00831180   xdc_runtime_System_Module_GateProxy_enter__E
008311a0   xdc_runtime_System_Module_GateProxy_leave__E
008311c0   xdc_runtime_System_Module_startup__E
008311e0   xdc_runtime_System_Module_startup__F
00831200   xdc_runtime_System_SupportProxy_abort__E
00831220   xdc_runtime_System_SupportProxy_exit__E
00831240   xdc_runtime_System_SupportProxy_putch__E
00831260   xdc_runtime_System_SupportProxy_ready__E
00831280   xdc_runtime_System_abort__E
008312a0   xdc_runtime_System_atexit__E
008312c0   xdc_runtime_System_exit__E
008312e0   xdc_runtime_System_exit__F
00831300   xdc_runtime_System_lastFxn__I
00831320   xdc_runtime_System_vsprintf__E
00831340   xdc_runtime_System_sprintf_va__F
00831340   xdc_runtime_System_vsprintf__F
00831360   xdc_runtime_Text_cordText__E
00831380   xdc_runtime_Text_putSite__E
008313a0   xdc_runtime_Text_ropeText__E
008313c0   xdc_runtime_Timestamp_SupportProxy_get32__E
008313c0   xdc_runtime_Timestamp_get32__F
008313e0   xdc_runtime_Timestamp_SupportProxy_get64__E
008313e0   xdc_runtime_Timestamp_get64__F
00831400   xdc_runtime_Timestamp_SupportProxy_getFreq__E
00831400   xdc_runtime_Timestamp_getFreq__F
00831420   xdc_runtime_Timestamp_get32__E
00831440   xdc_runtime_Timestamp_get64__E
00831460   xdc_runtime_Timestamp_getFreq__E
00831480   xdc_runtime_knl_GateThread_Module__startupDone__S
008314a0   xdc_runtime_knl_GateThread_Proxy_Object__delete__S
008314c0   xdc_runtime_knl_GateThread_Proxy_enter__E
008314e0   xdc_runtime_knl_GateThread_Proxy_leave__E
00831500   xdc_runtime_knl_GateThread_Proxy_query__E
00831500   xdc_runtime_knl_GateThread_query__F
00831520   xdc_runtime_knl_GateThread_enter__E
00831540   xdc_runtime_knl_GateThread_enter__F
00831560   xdc_runtime_knl_GateThread_leave__E
00831580   xdc_runtime_knl_GateThread_leave__F
008315a0   xdc_runtime_knl_GateThread_query__E
008315c0   txMsgPtrs
008392c0   rxMsgPtrs
00840fc0   ti_sdo_utils_NameServer_Module_State_0_nsRemoteHandle__A
00840fc8   ti_sysbios_heaps_HeapMem_Instance_State_0_buf__A
00848fc8   ti_sysbios_knl_Task_Instance_State_0_hookEnv__A
00848fd0   ti_sysbios_knl_Task_Instance_State_1_hookEnv__A
00848fd8   ti_sysbios_knl_Task_Instance_State_0_stack__A
008497d8   ti_sysbios_knl_Task_Instance_State_1_stack__A
00849fd8   localQueueName
00849fe0   nextQueueName
00849fe8   prevQueueName
00849ff0   timerFreq
00849ff8   cpuFreq
0084a000   rawtimestamps
0084a190   latencies
0084a320   latencyStats
0084a348   _tmpnams
0084a488   gDataBufferMemMgr
0084a578   gI2cBlock
0084a5c8   _lock
0084a5cc   _unlock
0084a5d0   xdc_runtime_Text_charTab__A
0084d618   ti_sysbios_family_c66_Cache_marvalues__C
0084da18   xdc_runtime_Text_nodeTab__A
0084db8c   ti_sdo_ipc_GateMP_A_invalidClose__C
0084db90   _ctypes_
0084ded0   xdc_runtime_Startup_sfxnTab__A
0084df10   ti_sdo_ipc_notifyDrivers_NotifyDriverCirc_Module__FXNS__C
0084df48   ti_sdo_ipc_GateMP_Object__PARAMS__C
0084df7c   ti_sdo_ipc_notifyDrivers_NotifyDriverCirc_Object__PARAMS__C
0084dfb0   ti_sdo_ipc_heaps_HeapMemMP_Object__PARAMS__C
0084dfe0   ti_sysbios_family_c64p_Hwi_Object__PARAMS__C
0084e03c   ti_sdo_ipc_gates_GateHWSem_Module__FXNS__C
0084e068   ti_sdo_ipc_gates_GateMPSupportNull_Module__FXNS__C
0084e094   ti_sdo_ipc_gates_GatePeterson_Module__FXNS__C
0084e110   ti_sdo_ipc_heaps_HeapMemMP_Module__FXNS__C
0084e138   ti_sdo_ipc_nsremote_NameServerRemoteNotify_Module__FXNS__C
0084e160   ti_sdo_ipc_transports_TransportShmNotify_Module__FXNS__C
0084e188   ti_sysbios_heaps_HeapMem_Module__FXNS__C
0084e1b0   ti_sysbios_knl_Swi_Object__PARAMS__C
0084e1d8   ti_sdo_ipc_gates_GateHWSem_Object__PARAMS__C
0084e1fc   ti_sdo_ipc_gates_GateMPSupportNull_Object__PARAMS__C
0084e220   ti_sdo_ipc_gates_GatePeterson_Object__PARAMS__C
0084e244   ti_sysbios_gates_GateAll_Module__FXNS__C
0084e268   ti_sysbios_gates_GateHwi_Module__FXNS__C
0084e28c   ti_sysbios_gates_GateMutexPri_Module__FXNS__C
0084e2b0   ti_sysbios_gates_GateMutex_Module__FXNS__C
0084e2d4   ti_sysbios_gates_GateSwi_Module__FXNS__C
0084e2f8   ti_sysbios_knl_Clock_Object__PARAMS__C
0084e31c   ti_sysbios_knl_Semaphore_Object__PARAMS__C
0084e340   ti_sysbios_syncs_SyncSem_Module__FXNS__C
0084e364   xdc_runtime_GateNull_Module__FXNS__C
0084e388   xdc_runtime_knl_GateThread_Module__FXNS__C
0084e3f0   ti_sdo_ipc_GateMP_Object__DESC__C
0084e410   ti_sdo_ipc_MessageQ_Object__DESC__C
0084e430   ti_sdo_ipc_Notify_Object__DESC__C
0084e450   ti_sdo_ipc_gates_GateHWSem_Object__DESC__C
0084e470   ti_sdo_ipc_gates_GateMPSupportNull_Object__DESC__C
0084e490   ti_sdo_ipc_gates_GatePeterson_Object__DESC__C
0084e4b0   ti_sdo_ipc_heaps_HeapMemMP_Object__DESC__C
0084e4d0   ti_sdo_ipc_notifyDrivers_NotifyDriverCirc_Object__DESC__C
0084e4f0   ti_sdo_ipc_nsremote_NameServerRemoteNotify_Object__DESC__C
0084e510   ti_sdo_ipc_nsremote_NameServerRemoteNotify_Object__PARAMS__C
0084e530   ti_sdo_ipc_transports_TransportShmNotify_Object__DESC__C
0084e550   ti_sdo_utils_List_Object__DESC__C
0084e570   ti_sysbios_family_c64p_Hwi_Object__DESC__C
0084e590   ti_sysbios_gates_GateAll_Object__DESC__C
0084e5b0   ti_sysbios_gates_GateHwi_Object__DESC__C
0084e5d0   ti_sysbios_gates_GateMutexPri_Object__DESC__C
0084e5f0   ti_sysbios_gates_GateMutex_Object__DESC__C
0084e610   ti_sysbios_gates_GateSwi_Object__DESC__C
0084e630   ti_sysbios_heaps_HeapMem_Object__DESC__C
0084e650   ti_sysbios_heaps_HeapMem_Object__PARAMS__C
0084e670   ti_sysbios_knl_Clock_Object__DESC__C
0084e690   ti_sysbios_knl_Queue_Object__DESC__C
0084e6b0   ti_sysbios_knl_Semaphore_Object__DESC__C
0084e6d0   ti_sysbios_knl_Swi_Object__DESC__C
0084e6f0   ti_sysbios_syncs_SyncSem_Object__DESC__C
0084e710   ti_sysbios_xdcruntime_GateThreadSupport_Object__DESC__C
0084e730   xdc_runtime_GateNull_Object__DESC__C
0084e750   xdc_runtime_Startup_sfxnRts__A
0084e770   xdc_runtime_knl_GateThread_Object__DESC__C
0084e790   ti_sdo_ipc_MessageQ_Object__PARAMS__C
0084e7ac   ti_sdo_ipc_transports_TransportShmNotify_Object__PARAMS__C
0084e7c8   ti_sysbios_syncs_SyncSem_Object__PARAMS__C
0084e7e4   ti_sdo_ipc_Notify_Object__PARAMS__C
0084e7fc   ti_sdo_utils_List_Object__PARAMS__C
0084e814   ti_sysbios_gates_GateAll_Object__PARAMS__C
0084e82c   ti_sysbios_gates_GateHwi_Object__PARAMS__C
0084e844   ti_sysbios_gates_GateMutexPri_Object__PARAMS__C
0084e85c   ti_sysbios_gates_GateMutex_Object__PARAMS__C
0084e874   ti_sysbios_gates_GateSwi_Object__PARAMS__C
0084e88c   ti_sysbios_knl_Queue_Object__PARAMS__C
0084e8a4   ti_sdo_ipc_GateMP_A_invalidDelete__C
0084e8a8   ti_sysbios_knl_Task_hooks__A
0084e8c0   ti_sysbios_xdcruntime_GateThreadSupport_Object__PARAMS__C
0084e8d8   xdc_runtime_GateNull_Object__PARAMS__C
0084e8f0   xdc_runtime_knl_GateThread_Object__PARAMS__C
0084e924   ti_sdo_ipc_GateMP_E_gateUnavailable__C
0084e928   xdc_runtime_Startup_firstFxns__A
0084e938   ti_sysbios_family_c66_Cache_initSize__C
0084e944   ti_sdo_ipc_GateMP_E_localGate__C
0084e948   ti_sdo_utils_MultiProc_nameList__A
0084e950   ti_sysbios_knl_Idle_funcList__C
0084e958   ti_sysbios_knl_Task_hooks__C
0084e960   xdc_runtime_Startup_firstFxns__C
0084e968   xdc_runtime_Startup_lastFxns__C
0084e974   ti_sdo_ipc_GateMP_LM_create__C
0084e97c   ti_sdo_ipc_GateMP_LM_delete__C
0084e980   ti_sdo_ipc_GateMP_LM_enter__C
0084e984   ti_sdo_ipc_GateMP_LM_leave__C
0084e988   ti_sdo_ipc_GateMP_LM_open__C
0084e98c   ti_sdo_ipc_GateMP_Module__diagsEnabled__C
0084e990   ti_sdo_ipc_GateMP_Module__diagsIncluded__C
0084e994   ti_sdo_ipc_GateMP_Module__diagsMask__C
0084e998   ti_sdo_ipc_GateMP_Module__loggerFxn2__C
0084e99c   ti_sdo_ipc_GateMP_Module__loggerFxn4__C
0084e9a0   ti_sdo_ipc_GateMP_Module__loggerObj__C
0084e9a4   ti_sdo_ipc_Ipc_A_addrNotCacheAligned__C
0084e9a8   ti_sdo_ipc_Ipc_A_addrNotInSharedRegion__C
0084e9ac   ti_sdo_ipc_Ipc_A_internal__C
0084e9b0   ti_sdo_ipc_Ipc_A_invArgument__C
0084e9b4   ti_sdo_ipc_Ipc_A_invParam__C
0084e9b8   ti_sdo_ipc_Ipc_A_nullArgument__C
0084e9bc   ti_sdo_ipc_Ipc_E_internal__C
0084e9c0   ti_sdo_ipc_Ipc_E_nameFailed__C
0084e9c4   ti_sdo_ipc_Ipc_E_versionMismatch__C
0084e9c8   ti_sdo_ipc_Ipc_Module__diagsEnabled__C
0084e9cc   ti_sdo_ipc_Ipc_Module__diagsIncluded__C
0084e9d0   ti_sdo_ipc_Ipc_Module__diagsMask__C
0084e9d4   ti_sdo_ipc_Ipc_numUserFxns__C
0084e9d8   ti_sdo_ipc_Ipc_procSync__C
0084e9dc   ti_sdo_ipc_Ipc_userFxns__C
0084e9e0   ti_sdo_ipc_MessageQ_A_cannotFreeStaticMsg__C
0084e9e4   ti_sdo_ipc_MessageQ_A_heapIdInvalid__C
0084e9e8   ti_sdo_ipc_MessageQ_A_invalidMsg__C
0084e9ec   ti_sdo_ipc_MessageQ_A_invalidObj__C
0084e9f0   ti_sdo_ipc_MessageQ_A_invalidParam__C
0084e9f4   ti_sdo_ipc_MessageQ_A_invalidQueueId__C
0084e9f8   ti_sdo_ipc_MessageQ_A_procIdInvalid__C
0084e9fc   ti_sdo_ipc_MessageQ_A_unregisteredTransport__C
0084ea00   ti_sdo_ipc_MessageQ_E_maxReached__C
0084ea04   ti_sdo_ipc_MessageQ_E_nameFailed__C
0084ea08   ti_sdo_ipc_MessageQ_Instance_State_highList__O
0084ea0c   ti_sdo_ipc_MessageQ_Instance_State_normalList__O
0084ea10   ti_sdo_ipc_MessageQ_LM_alloc__C
0084ea14   ti_sdo_ipc_MessageQ_LM_free__C
0084ea18   ti_sdo_ipc_MessageQ_LM_get__C
0084ea1c   ti_sdo_ipc_MessageQ_LM_putLocal__C
0084ea20   ti_sdo_ipc_MessageQ_Module__diagsEnabled__C
0084ea24   ti_sdo_ipc_MessageQ_Module__diagsIncluded__C
0084ea28   ti_sdo_ipc_MessageQ_Module__diagsMask__C
0084ea2c   ti_sdo_ipc_MessageQ_Module__loggerFxn4__C
0084ea30   ti_sdo_ipc_MessageQ_Module__loggerObj__C
0084ea34   ti_sdo_ipc_MessageQ_Object__count__C
0084ea38   ti_sdo_ipc_MessageQ_Object__heap__C
0084ea3c   ti_sdo_ipc_MessageQ_Object__table__C
0084ea40   ti_sdo_ipc_MessageQ_maxRuntimeEntries__C
0084ea44   ti_sdo_ipc_Notify_A_alreadyRegistered__C
0084ea48   ti_sdo_ipc_Notify_A_internal__C
0084ea4c   ti_sdo_ipc_Notify_A_invArgument__C
0084ea50   ti_sdo_ipc_Notify_A_notRegistered__C
0084ea54   ti_sdo_ipc_Notify_A_reservedEvent__C
0084ea58   ti_sdo_ipc_Notify_Module__diagsEnabled__C
0084ea5c   ti_sdo_ipc_Notify_Module__diagsIncluded__C
0084ea60   ti_sdo_ipc_Notify_Module__diagsMask__C
0084ea64   ti_sdo_ipc_Notify_Module__gateObj__C
0084ea68   ti_sdo_ipc_Notify_Object__heap__C
0084ea6c   ti_sdo_ipc_Notify_numEvents__C
0084ea70   ti_sdo_ipc_SharedRegion_A_addrOutOfRange__C
0084ea74   ti_sdo_ipc_SharedRegion_A_idTooLarge__C
0084ea78   ti_sdo_ipc_SharedRegion_A_noHeap__C
0084ea7c   ti_sdo_ipc_SharedRegion_A_region0Invalid__C
0084ea80   ti_sdo_ipc_SharedRegion_A_regionInvalid__C
0084ea84   ti_sdo_ipc_SharedRegion_A_reserveTooMuch__C
0084ea88   ti_sdo_ipc_SharedRegion_INVALIDSRPTR__C
0084ea8c   ti_sdo_ipc_SharedRegion_Module__diagsEnabled__C
0084ea90   ti_sdo_ipc_SharedRegion_Module__diagsIncluded__C
0084ea94   ti_sdo_ipc_SharedRegion_Module__diagsMask__C
0084ea98   ti_sdo_ipc_SharedRegion_cacheLineSize__C
0084ea9c   ti_sdo_ipc_SharedRegion_numOffsetBits__C
0084eaa0   ti_sdo_ipc_SharedRegion_offsetMask__C
0084eaa4   ti_sdo_ipc_family_c647x_Interrupt_INTERDSPINT__C
0084eaa8   ti_sdo_ipc_family_c647x_Interrupt_IPCAR0__C
0084eaac   ti_sdo_ipc_family_c647x_Interrupt_IPCGR0__C
0084eab0   ti_sdo_ipc_family_c647x_Interrupt_KICK0__C
0084eab4   ti_sdo_ipc_family_c647x_Interrupt_KICK1__C
0084eab8   ti_sdo_ipc_family_c647x_MultiProcSetup_A_invalidProcessor__C
0084eabc   ti_sdo_ipc_family_c647x_MultiProcSetup_Module__diagsEnabled__C
0084eac0   ti_sdo_ipc_family_c647x_MultiProcSetup_Module__diagsIncluded__C
0084eac4   ti_sdo_ipc_family_c647x_MultiProcSetup_Module__diagsMask__C
0084eac8   ti_sdo_ipc_family_c647x_MultiProcSetup_procMap__A
0084eacc   ti_sdo_ipc_family_c647x_MultiProcSetup_procMap__C
0084ead0   ti_sdo_ipc_family_c647x_NotifyCircSetup_dspIntVectId__C
0084ead4   ti_sdo_ipc_gates_GateHWSem_A_invSemNum__C
0084ead8   ti_sdo_ipc_gates_GateHWSem_Module__diagsEnabled__C
0084eadc   ti_sdo_ipc_gates_GateHWSem_Module__diagsIncluded__C
0084eae0   ti_sdo_ipc_gates_GateHWSem_Module__diagsMask__C
0084eae4   ti_sdo_ipc_gates_GateHWSem_baseAddr__C
0084eae8   ti_sdo_ipc_gates_GateHWSem_numSems__C
0084eaec   ti_sdo_ipc_gates_GateHWSem_reservedMaskArr__C
0084eaf0   ti_sdo_ipc_gates_GateHWSem_reservedMaskArr__A
0084eaf4   ti_sdo_ipc_gates_GateMPSupportNull_A_invalidAction__C
0084eaf8   ti_sdo_ipc_gates_GateMPSupportNull_Module__diagsEnabled__C
0084eafc   ti_sdo_ipc_gates_GateMPSupportNull_Module__diagsIncluded__C
0084eb00   ti_sdo_ipc_gates_GateMPSupportNull_Module__diagsMask__C
0084eb04   ti_sdo_ipc_gates_GateMPSupportNull_action__C
0084eb08   ti_sdo_ipc_gates_GatePeterson_E_gateRemotelyOpened__C
0084eb0c   ti_sdo_ipc_gates_GatePeterson_Module__diagsEnabled__C
0084eb10   ti_sdo_ipc_gates_GatePeterson_Module__diagsIncluded__C
0084eb14   ti_sdo_ipc_gates_GatePeterson_Module__diagsMask__C
0084eb18   ti_sdo_ipc_gates_GatePeterson_numInstances__C
0084eb1c   ti_sdo_ipc_heaps_HeapMemMP_A_align__C
0084eb20   ti_sdo_ipc_heaps_HeapMemMP_A_heapSize__C
0084eb24   ti_sdo_ipc_heaps_HeapMemMP_A_invalidFree__C
0084eb28   ti_sdo_ipc_heaps_HeapMemMP_A_zeroBlock__C
0084eb2c   ti_sdo_ipc_heaps_HeapMemMP_E_memory__C
0084eb30   ti_sdo_ipc_heaps_HeapMemMP_Module__diagsEnabled__C
0084eb34   ti_sdo_ipc_heaps_HeapMemMP_Module__diagsIncluded__C
0084eb38   ti_sdo_ipc_heaps_HeapMemMP_Module__diagsMask__C
0084eb3c   ti_sdo_ipc_interfaces_IGateMPSupport_Interface__BASE__C
0084eb40   ti_sdo_ipc_interfaces_IMessageQTransport_Interface__BASE__C
0084eb44   ti_sdo_ipc_interfaces_INotifyDriver_Interface__BASE__C
0084eb48   ti_sdo_ipc_notifyDrivers_NotifyDriverCirc_A_notSupported__C
0084eb4c   ti_sdo_ipc_notifyDrivers_NotifyDriverCirc_Module__diagsEnabled__C
0084eb50   ti_sdo_ipc_notifyDrivers_NotifyDriverCirc_Module__diagsIncluded__C
0084eb54   ti_sdo_ipc_notifyDrivers_NotifyDriverCirc_Module__diagsMask__C
0084eb58   ti_sdo_ipc_notifyDrivers_NotifyDriverCirc_maxIndex__C
0084eb5c   ti_sdo_ipc_notifyDrivers_NotifyDriverCirc_modIndex__C
0084eb60   ti_sdo_ipc_notifyDrivers_NotifyDriverCirc_numMsgs__C
0084eb64   ti_sdo_ipc_nsremote_NameServerRemoteNotify_A_invalidValueLen__C
0084eb68   ti_sdo_ipc_nsremote_NameServerRemoteNotify_Instance_State_semMultiBlock__O
0084eb6c   ti_sdo_ipc_nsremote_NameServerRemoteNotify_Instance_State_semRemoteWait__O
0084eb70   ti_sdo_ipc_nsremote_NameServerRemoteNotify_Instance_State_swiObj__O
0084eb74   ti_sdo_ipc_nsremote_NameServerRemoteNotify_Module__diagsEnabled__C
0084eb78   ti_sdo_ipc_nsremote_NameServerRemoteNotify_Module__diagsIncluded__C
0084eb7c   ti_sdo_ipc_nsremote_NameServerRemoteNotify_Module__diagsMask__C
0084eb80   ti_sdo_ipc_nsremote_NameServerRemoteNotify_notifyEventId__C
0084eb84   ti_sdo_ipc_nsremote_NameServerRemoteNotify_timeout__C
0084eb88   ti_sdo_ipc_transports_TransportShmNotifySetup_priority__C
0084eb8c   ti_sdo_utils_INameServerRemote_Interface__BASE__C
0084eb90   ti_sdo_utils_List_Object__count__C
0084eb94   ti_sdo_utils_List_Object__table__C
0084eb98   ti_sdo_utils_MultiProc_A_invalidMultiProcId__C
0084eb9c   ti_sdo_utils_MultiProc_Module__diagsEnabled__C
0084eba0   ti_sdo_utils_MultiProc_Module__diagsIncluded__C
0084eba4   ti_sdo_utils_MultiProc_Module__diagsMask__C
0084eba8   ti_sdo_utils_MultiProc_nameList__C
0084ebac   ti_sdo_utils_NameServer_A_invArgument__C
0084ebb0   ti_sdo_utils_NameServer_A_invalidLen__C
0084ebb4   ti_sdo_utils_NameServer_E_entryExists__C
0084ebb8   ti_sdo_utils_NameServer_E_maxReached__C
0084ebbc   ti_sdo_utils_NameServer_Instance_State_freeList__O
0084ebc0   ti_sdo_utils_NameServer_Instance_State_nameList__O
0084ebc4   ti_sdo_utils_NameServer_Module__diagsEnabled__C
0084ebc8   ti_sdo_utils_NameServer_Module__diagsIncluded__C
0084ebcc   ti_sdo_utils_NameServer_Module__diagsMask__C
0084ebd0   ti_sdo_utils_NameServer_Object__count__C
0084ebd4   ti_sdo_utils_NameServer_Object__table__C
0084ebd8   ti_sysbios_BIOS_Module__diagsEnabled__C
0084ebdc   ti_sysbios_BIOS_Module__diagsIncluded__C
0084ebe0   ti_sysbios_BIOS_Module__diagsMask__C
0084ebe4   ti_sysbios_BIOS_installedErrorHook__C
0084ebe8   ti_sysbios_family_c64p_Exception_E_exceptionMin__C
0084ebec   ti_sysbios_family_c64p_Exception_exceptionHook__C
0084ebf0   ti_sysbios_family_c64p_Exception_externalHook__C
0084ebf4   ti_sysbios_family_c64p_Exception_internalHook__C
0084ebf8   ti_sysbios_family_c64p_Exception_nmiHook__C
0084ebfc   ti_sysbios_family_c64p_Hwi_E_alreadyDefined__C
0084ec00   ti_sysbios_family_c64p_Hwi_E_handleNotFound__C
0084ec04   ti_sysbios_family_c64p_Hwi_LD_end__C
0084ec08   ti_sysbios_family_c64p_Hwi_LM_begin__C
0084ec0c   ti_sysbios_family_c64p_Hwi_Module__diagsEnabled__C
0084ec10   ti_sysbios_family_c64p_Hwi_Module__diagsIncluded__C
0084ec14   ti_sysbios_family_c64p_Hwi_Module__diagsMask__C
0084ec18   ti_sysbios_family_c64p_Hwi_Module__loggerFxn1__C
0084ec1c   ti_sysbios_family_c64p_Hwi_Module__loggerFxn8__C
0084ec20   ti_sysbios_family_c64p_Hwi_Module__loggerObj__C
0084ec24   ti_sysbios_family_c66_Cache_atomicBlockSize__C
0084ec28   ti_sysbios_gates_GateMutexPri_A_badContext__C
0084ec2c   ti_sysbios_gates_GateMutexPri_Instance_State_pendQ__O
0084ec30   ti_sysbios_gates_GateMutexPri_Module__diagsEnabled__C
0084ec34   ti_sysbios_gates_GateMutexPri_Module__diagsIncluded__C
0084ec38   ti_sysbios_gates_GateMutexPri_Module__diagsMask__C
0084ec3c   ti_sysbios_gates_GateMutex_A_badContext__C
0084ec40   ti_sysbios_gates_GateMutex_Instance_State_sem__O
0084ec44   ti_sysbios_gates_GateMutex_Module__diagsEnabled__C
0084ec48   ti_sysbios_gates_GateMutex_Module__diagsIncluded__C
0084ec4c   ti_sysbios_gates_GateMutex_Module__diagsMask__C
0084ec50   ti_sysbios_gates_GateSwi_A_badContext__C
0084ec54   ti_sysbios_gates_GateSwi_Module__diagsEnabled__C
0084ec58   ti_sysbios_gates_GateSwi_Module__diagsIncluded__C
0084ec5c   ti_sysbios_gates_GateSwi_Module__diagsMask__C
0084ec60   ti_sysbios_hal_Hwi_E_stackOverflow__C
0084ec64   ti_sysbios_heaps_HeapMem_A_align__C
0084ec68   ti_sysbios_heaps_HeapMem_A_heapSize__C
0084ec6c   ti_sysbios_heaps_HeapMem_A_invalidFree__C
0084ec70   ti_sysbios_heaps_HeapMem_A_zeroBlock__C
0084ec74   ti_sysbios_heaps_HeapMem_E_memory__C
0084ec78   ti_sysbios_heaps_HeapMem_Module__diagsEnabled__C
0084ec7c   ti_sysbios_heaps_HeapMem_Module__diagsIncluded__C
0084ec80   ti_sysbios_heaps_HeapMem_Module__diagsMask__C
0084ec84   ti_sysbios_heaps_HeapMem_Module__gateObj__C
0084ec88   ti_sysbios_heaps_HeapMem_Object__count__C
0084ec8c   ti_sysbios_heaps_HeapMem_Object__table__C
0084ec90   ti_sysbios_heaps_HeapMem_reqAlignMask__C
0084ec94   ti_sysbios_heaps_HeapMem_reqAlign__C
0084ec98   ti_sysbios_knl_Clock_A_badThreadType__C
0084ec9c   ti_sysbios_knl_Clock_LM_begin__C
0084eca0   ti_sysbios_knl_Clock_LM_tick__C
0084eca4   ti_sysbios_knl_Clock_LW_delayed__C
0084eca8   ti_sysbios_knl_Clock_Module_State_clockQ__O
0084ecac   ti_sysbios_knl_Clock_Module__diagsEnabled__C
0084ecb0   ti_sysbios_knl_Clock_Module__diagsIncluded__C
0084ecb4   ti_sysbios_knl_Clock_Module__diagsMask__C
0084ecb8   ti_sysbios_knl_Clock_Module__loggerFxn1__C
0084ecbc   ti_sysbios_knl_Clock_Module__loggerFxn2__C
0084ecc0   ti_sysbios_knl_Clock_Module__loggerObj__C
0084ecc4   ti_sysbios_knl_Clock_tickMode__C
0084ecc8   ti_sysbios_knl_Clock_tickPeriod__C
0084eccc   ti_sysbios_knl_Clock_tickSource__C
0084ecd0   ti_sysbios_knl_Idle_funcList__A
0084ecd4   ti_sysbios_knl_Queue_Object__count__C
0084ecd8   ti_sysbios_knl_Queue_Object__table__C
0084ecdc   ti_sysbios_knl_Semaphore_A_badContext__C
0084ece0   ti_sysbios_knl_Semaphore_A_noEvents__C
0084ece4   ti_sysbios_knl_Semaphore_A_overflow__C
0084ece8   ti_sysbios_knl_Semaphore_Instance_State_pendQ__O
0084ecec   ti_sysbios_knl_Semaphore_LM_pend__C
0084ecf0   ti_sysbios_knl_Semaphore_LM_post__C
0084ecf4   ti_sysbios_knl_Semaphore_Module__diagsEnabled__C
0084ecf8   ti_sysbios_knl_Semaphore_Module__diagsIncluded__C
0084ecfc   ti_sysbios_knl_Semaphore_Module__diagsMask__C
0084ed00   ti_sysbios_knl_Semaphore_Module__loggerFxn2__C
0084ed04   ti_sysbios_knl_Semaphore_Module__loggerFxn4__C
0084ed08   ti_sysbios_knl_Semaphore_Module__loggerObj__C
0084ed0c   ti_sysbios_knl_Swi_A_badPriority__C
0084ed10   ti_sysbios_knl_Swi_LD_end__C
0084ed14   ti_sysbios_knl_Swi_LM_begin__C
0084ed18   ti_sysbios_knl_Swi_LM_post__C
0084ed1c   ti_sysbios_knl_Swi_Module__diagsEnabled__C
0084ed20   ti_sysbios_knl_Swi_Module__diagsIncluded__C
0084ed24   ti_sysbios_knl_Swi_Module__diagsMask__C
0084ed28   ti_sysbios_knl_Swi_Module__loggerFxn1__C
0084ed2c   ti_sysbios_knl_Swi_Module__loggerFxn4__C
0084ed30   ti_sysbios_knl_Swi_Module__loggerObj__C
0084ed34   ti_sysbios_knl_Swi_Object__count__C
0084ed38   ti_sysbios_knl_Swi_Object__table__C
0084ed3c   ti_sysbios_knl_Task_A_badPriority__C
0084ed40   ti_sysbios_knl_Task_E_spOutOfBounds__C
0084ed44   ti_sysbios_knl_Task_E_stackOverflow__C
0084ed48   ti_sysbios_knl_Task_LD_block__C
0084ed4c   ti_sysbios_knl_Task_LD_exit__C
0084ed50   ti_sysbios_knl_Task_LD_ready__C
0084ed54   ti_sysbios_knl_Task_LM_setPri__C
0084ed58   ti_sysbios_knl_Task_LM_switch__C
0084ed5c   ti_sysbios_knl_Task_LM_yield__C
0084ed60   ti_sysbios_knl_Task_Module_State_inactiveQ__O
0084ed64   ti_sysbios_knl_Task_Module_State_terminatedQ__O
0084ed68   ti_sysbios_knl_Task_Module__diagsEnabled__C
0084ed6c   ti_sysbios_knl_Task_Module__diagsIncluded__C
0084ed70   ti_sysbios_knl_Task_Module__diagsMask__C
0084ed74   ti_sysbios_knl_Task_Module__loggerFxn2__C
0084ed78   ti_sysbios_knl_Task_Module__loggerFxn4__C
0084ed7c   ti_sysbios_knl_Task_Module__loggerObj__C
0084ed80   ti_sysbios_knl_Task_Object__count__C
0084ed84   ti_sysbios_knl_Task_Object__table__C
0084ed88   ti_sysbios_knl_Task_allBlockedFunc__C
0084ed8c   ti_sysbios_knl_Task_numConstructedTasks__C
0084ed90   ti_sysbios_knl_Task_numPriorities__C
0084ed94   ti_sysbios_syncs_SyncSem_Module__diagsEnabled__C
0084ed98   ti_sysbios_syncs_SyncSem_Module__diagsIncluded__C
0084ed9c   ti_sysbios_syncs_SyncSem_Module__diagsMask__C
0084eda0   ti_sysbios_timers_timer64_Timer_A_notAvailable__C
0084eda4   ti_sysbios_timers_timer64_Timer_E_cannotSupport__C
0084eda8   ti_sysbios_timers_timer64_Timer_Module__diagsEnabled__C
0084edac   ti_sysbios_timers_timer64_Timer_Module__diagsIncluded__C
0084edb0   ti_sysbios_timers_timer64_Timer_Module__diagsMask__C
0084edb4   ti_sysbios_timers_timer64_Timer_anyMask__C
0084edb8   ti_sysbios_timers_timer64_Timer_freqDivisor__C
0084edbc   ti_sysbios_timers_timer64_Timer_numLocalTimers__C
0084edc0   ti_sysbios_timers_timer64_Timer_numTimerDevices__C
0084edc4   ti_sysbios_xdcruntime_GateThreadSupport_Instance_State_gate__O
0084edc8   xdc_runtime_Assert_E_assertFailed__C
0084edcc   xdc_runtime_Core_A_initializedParams__C
0084edd0   xdc_runtime_Core_Module__diagsEnabled__C
0084edd4   xdc_runtime_Core_Module__diagsIncluded__C
0084edd8   xdc_runtime_Core_Module__diagsMask__C
0084eddc   xdc_runtime_Error_E_generic__C
0084ede0   xdc_runtime_Error_E_memory__C
0084ede4   xdc_runtime_Error_Module__diagsEnabled__C
0084ede8   xdc_runtime_Error_Module__diagsIncluded__C
0084edec   xdc_runtime_Error_Module__diagsMask__C
0084edf0   xdc_runtime_Error_Module__loggerFxn8__C
0084edf4   xdc_runtime_Error_Module__loggerObj__C
0084edf8   xdc_runtime_Error_policy__C
0084edfc   xdc_runtime_Error_raiseHook__C
0084ee00   xdc_runtime_IGateProvider_Interface__BASE__C
0084ee04   xdc_runtime_IHeap_Interface__BASE__C
0084ee08   xdc_runtime_IModule_Interface__BASE__C
0084ee0c   xdc_runtime_Log_L_error__C
0084ee10   xdc_runtime_Main_Module__diagsEnabled__C
0084ee14   xdc_runtime_Main_Module__diagsIncluded__C
0084ee18   xdc_runtime_Main_Module__diagsMask__C
0084ee1c   xdc_runtime_Memory_defaultHeapInstance__C
0084ee20   xdc_runtime_Startup_execImpl__C
0084ee24   xdc_runtime_Startup_maxPasses__C
0084ee28   xdc_runtime_Startup_lastFxns__A
0084ee2c   xdc_runtime_Startup_sfxnRts__C
0084ee30   xdc_runtime_Startup_sfxnTab__C
0084ee34   xdc_runtime_Startup_startModsFxn__C
0084ee38   xdc_runtime_System_A_cannotFitIntoArg__C
0084ee3c   xdc_runtime_System_Module__gateObj__C
0084ee40   xdc_runtime_System_extendFxn__C
0084ee44   xdc_runtime_System_maxAtexitHandlers__C
0084ee48   xdc_runtime_Text_charTab__C
0084ee4c   xdc_runtime_Text_nameEmpty__C
0084ee50   xdc_runtime_Text_nameStatic__C
0084ee54   xdc_runtime_Text_nameUnknown__C
0084ee58   xdc_runtime_Text_nodeTab__C
0084ee5c   xdc_runtime_Text_visitRopeFxn__C
0084ee60   xdc_runtime_knl_ISync_Interface__BASE__C
0084ee64   ti_sdo_ipc_GateMP_Module__id__C
0084ee68   ti_sdo_ipc_GateMP_Module__loggerDefined__C
0084ee6c   ti_sdo_ipc_Ipc_Module__id__C
0084ee70   ti_sdo_ipc_Ipc_generateSlaveDataForHost__C
0084ee74   ti_sdo_ipc_MessageQ_Module__id__C
0084ee78   ti_sdo_ipc_MessageQ_Module__loggerDefined__C
0084ee7c   ti_sdo_ipc_Notify_Module__id__C
0084ee80   ti_sdo_ipc_Notify_numLines__C
0084ee84   ti_sdo_ipc_Notify_reservedEvents__C
0084ee88   ti_sdo_ipc_SharedRegion_Module__id__C
0084ee8c   ti_sdo_ipc_SharedRegion_numEntries__C
0084ee90   ti_sdo_ipc_SharedRegion_translate__C
0084ee94   ti_sdo_ipc_family_c647x_Interrupt_enableKick__C
0084ee98   ti_sdo_ipc_family_c647x_MultiProcSetup_Module__id__C
0084ee9c   ti_sdo_ipc_gates_GateHWSem_Module__id__C
0084eea0   ti_sdo_ipc_gates_GateMPSupportNull_Module__id__C
0084eea4   ti_sdo_ipc_gates_GatePeterson_Module__id__C
0084eea8   ti_sdo_ipc_heaps_HeapMemMP_Module__id__C
0084eeac   ti_sdo_ipc_notifyDrivers_NotifyDriverCirc_Module__id__C
0084eeb0   ti_sdo_ipc_notifyDrivers_NotifyDriverCirc_enableStats__C
0084eeb4   ti_sdo_ipc_nsremote_NameServerRemoteNotify_Module__id__C
0084eeb8   ti_sdo_ipc_transports_TransportShmNotify_alwaysWriteBackMsg__C
0084eebc   ti_sdo_ipc_transports_TransportShmNotify_notifyEventId__C
0084eec0   ti_sdo_utils_MultiProc_Module__id__C
0084eec4   ti_sdo_utils_MultiProc_numProcessors__C
0084eec8   ti_sdo_utils_MultiProc_numProcsInCluster__C
0084eecc   ti_sdo_utils_NameServer_Module__id__C
0084eed0   ti_sdo_utils_NameServer_singleProcessor__C
0084eed4   ti_sysbios_BIOS_Module__id__C
0084eed8   ti_sysbios_family_c64p_Exception_Module__id__C
0084eedc   ti_sysbios_family_c64p_Hwi_Module__id__C
0084eee0   ti_sysbios_family_c64p_Hwi_Module__loggerDefined__C
0084eee4   ti_sysbios_gates_GateMutexPri_Module__id__C
0084eee8   ti_sysbios_gates_GateMutex_Module__id__C
0084eeec   ti_sysbios_gates_GateSwi_Module__id__C
0084eef0   ti_sysbios_hal_Hwi_Module__id__C
0084eef4   ti_sysbios_heaps_HeapMem_Module__id__C
0084eef8   ti_sysbios_knl_Clock_Module__id__C
0084eefc   ti_sysbios_knl_Clock_Module__loggerDefined__C
0084ef00   ti_sysbios_knl_Semaphore_Module__id__C
0084ef04   ti_sysbios_knl_Semaphore_Module__loggerDefined__C
0084ef08   ti_sysbios_knl_Swi_Module__id__C
0084ef0c   ti_sysbios_knl_Swi_Module__loggerDefined__C
0084ef10   ti_sysbios_knl_Task_Module__id__C
0084ef14   ti_sysbios_knl_Task_Module__loggerDefined__C
0084ef18   ti_sysbios_knl_Task_deleteTerminatedTasks__C
0084ef1c   ti_sysbios_knl_Task_initStackFlag__C
0084ef20   ti_sysbios_syncs_SyncSem_Module__id__C
0084ef24   ti_sysbios_timers_timer64_Timer_Module__id__C
0084ef28   ti_sysbios_timers_timer64_Timer_startupNeeded__C
0084ef2c   xdc_runtime_Core_Module__id__C
0084ef30   xdc_runtime_Error_Module__loggerDefined__C
0084ef34   xdc_runtime_Error_maxDepth__C
0084ef38   xdc_runtime_Main_Module__id__C
0084ef3c   xdc_runtime_Memory_Module__id__C
0084ef40   xdc_runtime_Text_charCnt__C
0084ef44   xdc_runtime_Text_isLoaded__C
0084ef48   xdc_runtime_Text_registryModsLastId__C
0084ef4c   xdc_runtime_Text_unnamedModsLastId__C
0084ef50   ti_sdo_ipc_GateMP_Module_State_0_remoteCustom1Gates__A
0084f750   ti_sdo_ipc_GateMP_Module__root__V
0084f758   ti_sdo_ipc_GateMP_Module__state__V
0084f7a0   ti_sdo_ipc_Ipc_Module__state__V
0084f7ac   ti_sdo_ipc_MessageQ_Module__root__V
0084f7b4   ti_sdo_ipc_MessageQ_Module__state__V
0084f7d0   ti_sdo_ipc_Notify_Module__root__V
0084f7d8   ti_sdo_ipc_Notify_Module__state__V
0084f7e0   ti_sdo_ipc_SharedRegion_Module__state__V
0084f7e4   ti_sdo_ipc_family_c647x_Interrupt_Module__state__V
0084f7ec   ti_sdo_ipc_gates_GateHWSem_Module__root__V
0084f7f4   ti_sdo_ipc_gates_GateMPSupportNull_Module__root__V
0084f7fc   ti_sdo_ipc_gates_GatePeterson_Module__root__V
0084f804   ti_sdo_ipc_heaps_HeapMemMP_Module__root__V
0084f80c   ti_sdo_ipc_heaps_HeapMemMP_Module__state__V
0084f810   ti_sdo_ipc_notifyDrivers_NotifyDriverCirc_Module__root__V
0084f818   ti_sdo_ipc_nsremote_NameServerRemoteNotify_Module__root__V
0084f820   ti_sdo_ipc_transports_TransportShmNotify_Module__root__V
0084f828   ti_sdo_ipc_transports_TransportShmNotifySetup_Module__state__V
0084f82c   ti_sdo_utils_List_Module__root__V
0084f834   ti_sdo_utils_MultiProc_Module__state__V
0084f838   ti_sdo_utils_NameServer_Module__root__V
0084f840   ti_sdo_utils_NameServer_Module__state__V
0084f848   ti_sdo_utils_NameServerRemoteNull_Module__root__V
0084f850   ti_sysbios_BIOS_Module__state__V
0084f86c   ti_sysbios_family_c64p_Exception_Module__state__V
0084f898   ti_sysbios_family_c64p_Hwi_Module__root__V
0084f8a0   ti_sysbios_family_c64p_Hwi_Module__state__V
0084f908   ti_sysbios_gates_GateAll_Module__root__V
0084f910   ti_sysbios_gates_GateHwi_Module__root__V
0084f918   ti_sysbios_gates_GateMutex_Module__root__V
0084f920   ti_sysbios_gates_GateMutexPri_Module__root__V
0084f928   ti_sysbios_gates_GateSwi_Module__root__V
0084f930   ti_sysbios_hal_Hwi_Module__root__V
0084f938   ti_sysbios_hal_Timer_Module__root__V
0084f940   ti_sysbios_heaps_HeapMem_Module__root__V
0084f948   ti_sysbios_knl_Clock_Module__root__V
0084f950   ti_sysbios_knl_Clock_Module__state__V
0084f97c   ti_sysbios_knl_Queue_Module__root__V
0084f984   ti_sysbios_knl_Semaphore_Module__root__V
0084f98c   ti_sysbios_knl_Swi_Module__root__V
0084f994   ti_sysbios_knl_Swi_Module__state__V
0084f9b0   ti_sysbios_knl_Task_Module__root__V
0084f9b8   ti_sysbios_knl_Task_Module__state__V
0084f9ec   ti_sysbios_syncs_SyncSem_Module__root__V
0084f9f4   ti_sysbios_timers_timer64_Timer_Module__root__V
0084f9fc   ti_sysbios_timers_timer64_Timer_Module__state__V
0084fa10   ti_sysbios_xdcruntime_GateThreadSupport_Module__root__V
0084fa18   xdc_runtime_Error_Module__state__V
0084fa1c   xdc_runtime_GateNull_Module__root__V
0084fa24   xdc_runtime_Memory_Module__state__V
0084fa28   xdc_runtime_Registry_Module__state__V
0084fa30   xdc_runtime_Startup_Module__state__V
0084fa38   xdc_runtime_System_Module__state__V
0084fa44   xdc_runtime_Text_Module__state__V
0084fa4c   xdc_runtime_knl_GateThread_Module__root__V
0084fa54   __xdc__init__addr
0084fa58   _ftable
0084fc38   ti_sysbios_timers_timer64_Timer_Module_State_0_device__A
0084fcf8   ti_sdo_utils_NameServer_Object__table__V
0084fe40   ti_sdo_ipc_SharedRegion_Module_State_0_regions__A
0084ff58   ti_sysbios_knl_Task_Object__table__V
0084ff9c   TSK_idle
0084ffe0   ti_sdo_ipc_GateMP_Module_State_0_remoteSystemGates__A
00850060   ti_sysbios_knl_Swi_Module_State_0_readyQ__A
008500e0   ti_sysbios_knl_Task_Module_State_0_readyQ__A
00850218   ti_sysbios_gates_GateMutex_Object__table__V
00850258   ti_sysbios_timers_timer64_Timer_Module_State_0_gctrl__A
00850298   ti_sysbios_timers_timer64_Timer_Module_State_0_handles__A
008502d8   ti_sysbios_timers_timer64_Timer_Module_State_0_intFreqs__A
00850350   ti_sdo_ipc_Ipc_Module_State_0_procEntry__A
00850398   ti_sdo_ipc_MessageQ_Module_State_0_heaps__A
008503b8   xdc_runtime_System_Module_State_0_atexitHandlers__A
008503d8   ti_sysbios_gates_GateMutexPri_Object__table__V
008503f0   ti_sysbios_heaps_HeapMem_Object__table__V
00850404   _ft_end
00850408   ti_sdo_ipc_MessageQ_Module_State_0_transports__A
00850418   ti_sdo_ipc_family_c647x_Interrupt_Module_State_0_fxnTable__A
00850428   ti_sysbios_gates_GateAll_Object__table__V
00850438   _cleanup_ptr
0085043c   _dtors_ptr
00850440   __TI_enable_exit_profile_output
00850448   ti_sysbios_gates_GateSwi_Object__table__V
00850454   __errno
00850454   errno
00850458   ti_sdo_ipc_Notify_Module_State_0_notifyHandles__A
00850460   ti_sdo_ipc_transports_TransportShmNotifySetup_Module_State_0_handles__A
00850468   ti_sdo_ipc_GateMP_Module_State_0_remoteCustom2Gates__A
00850470   ti_sdo_ipc_Notify_Module_State_0_notifyHandles_0__A
00850478   ti_sdo_ipc_Notify_Module_State_0_notifyHandles_1__A
00850480   ti_sysbios_gates_GateHwi_Object__table__V
00850488   xdc_runtime_GateNull_Object__table__V
00850490   _stack
00851490   __TI_STACK_END
00851d28   gDeviceNandBBlist
00852144   gDeviceNand
0085217c   gDeviceNor
008521b4   gDeviceEeprom0
008521ec   gDeviceEeprom1
00852228   emac_port_mode
00852230   __CIOBUF_
00852400   ti_sysbios_family_c64p_Hwi0
00852420   ti_sysbios_family_c64p_Hwi1
00852440   ti_sysbios_family_c64p_Hwi2
00852460   ti_sysbios_family_c64p_Hwi3
00852480   ti_sysbios_family_c64p_Hwi4
008524a0   ti_sysbios_family_c64p_Hwi5
008524c0   ti_sysbios_family_c64p_Hwi6
008524e0   ti_sysbios_family_c64p_Hwi7
00852500   ti_sysbios_family_c64p_Hwi8
00852520   ti_sysbios_family_c64p_Hwi9
00852540   ti_sysbios_family_c64p_Hwi10
00852560   ti_sysbios_family_c64p_Hwi11
00852580   ti_sysbios_family_c64p_Hwi12
008525a0   ti_sysbios_family_c64p_Hwi13
008525c0   ti_sysbios_family_c64p_Hwi14
008525e0   ti_sysbios_family_c64p_Hwi15
00852600   __TI_STATIC_BASE
00852600   prevCoreId
00852602   selfId
00852604   nextQueueId
00852608   prevQueueId
0085260c   cpuTimerFreqRatio
00852610   Ipc_sr0MemorySetup
00852618   gDataBufferMemMgrMaxSize
0085261c   qmssMallocCounter
00852620   qmssFreeCounter
00852624   cppiMallocCounter
00852628   cppiFreeCounter
0085262c   srioMallocCounter
00852630   srioFreeCounter
00852634   srioDataBufferMallocCounter
00852638   srioDataBufferFreeCounter
00852640   numCores
00852648   timeAdj
00852650   messageQ
00852658   timeLength
00852660   platform_errno
00852664   platform_init_return_code
00852e40   __TI_Handler_Table_Base
00852e4c   __TI_Handler_Table_Limit
00852e70   __TI_CINIT_Base
00852ea8   __TI_CINIT_Limit
ffffffff   __TI_pprof_out_hndl
ffffffff   __TI_prof_data_size
ffffffff   __TI_prof_data_start
ffffffff   __binit__
ffffffff   __c_args__
ffffffff   binit
UNDEFED    __TI_INITARRAY_Base
UNDEFED    __TI_INITARRAY_Limit

[1490 symbols]
